:020000040000FA
:10000000021F4E022003FFFFFFFFFF02200BFFFF36
:10001000FFFFFF022013FFFFFFFFFF02201BFFFF78
:10002000FFFFFF022023FFFFFFFFFF02202BFFFF48
:10003000FFFFFF022033FFFFFFFFFF02203BFFFF18
:10004000FFFFFF022043FFFFFFFFFF02204BFFFFE8
:10005000FFFFFF022053FFFFFFFFFF02205BFFFFB8
:10006000FFFFFF022063FFFFFFFFFF02206BFFFF88
:10007000FFFFFF022073FFFFFFFFFF02207BFFFF58
:10008000FFFFFF022083FFFFFFFFFF02208BFFFF28
:10009000FFFF70DFFFFF040000000002000000C847
:1000A000030002030369A5020269A532730000017F
:1000B00000000000000400FFFFFFFFFFFFFFFF0440
:1000C00003090424035400650078006100730020D4
:1000D0000049006E0073007400720075006D0065C9
:1000E000006E007400730024035400490020004394
:1000F000004300320035003300310020005500532A
:10010000004200200043004400430000035F005F02
:100110000030005800000000000000000000000057
:1001200000000000000000000000000000000000CF
:100130000000000000303132333435363738394171
:1001400042434445463C1C911C911C911C911C99B6
:100150001C74F8121BD6900391E060159003027492
:10016000FEF0900304744DF0A37405F07A011207B9
:100170000C7F01021D7B74F8121BD674FF121EC582
:100180007E00801F851882851983E064FE700690CA
:1001900003877401F0851882851983E0F890038441
:1001A000E068F07901AA18AB191210DFE9700302B8
:1001B000027E851882851983E064EF70027E07E075
:1001C000C0E0900387E0F8900385E0FAE82AF8E4BD
:1001D000340012075BD0E0F0900387E060A6146063
:1001E0000E14602A14603A14605014606680A69061
:1001F0000384E4F0851882851983E0900386F0C3B8
:1002000094809003874003E4808A74028086851876
:1002100082851983E0900382F090038774030201C2
:1002200094851882851983E0900383F0900386E01B
:1002300060199003877404020194900385E004F030
:10024000F8900386E06860030201959003877405C7
:10025000020194900385E4F0900387F0900384E01A
:10026000F8851882851983E0686003020195900380
:1002700082E0644D60030201951203B68002EEF93C
:100280007401121E4602017174F7121BD674FB1220
:100290001EC5EAFEEBFF7508047509007808121EFA
:1002A000DF7402121F467A907B0079041218F274F0
:1002B00002121E461206FE121F97E0687003A3E0AA
:1002C000697012851882851983E0F47003A3E0F445
:1002D00060030203917404121F3E1207678A088BA1
:1002E00009A808A9097402121F97E8F0A3E9F0749D
:1002F00004121F97E0600879011201510203AA85D8
:100300001882851983E0687003A3E0697076851808
:1003100082851983E0F47003A3E0F470197402126B
:100320001F977410F0A37420F085188285198374C8
:1003300010F0A37420F07508017509007808121EEA
:10034000DF7402121F467A247B0812197774021296
:100350001E467508047808121EDF7402121F467AC2
:10036000907B0079041218F27402121E461206FEE7
:10037000121F97E0687003A3E06970047902800699
:100380007904800279031201518E828F83741E805A
:10039000058E828F83E4F01206FE121F97E06870CC
:1003A00003A3E06970047901800279007405121ECC
:1003B000467F02021D7B74ED121BD674F8121EC517
:1003C000900307E0FA900306E0FB8B08EAF8E4C824
:1003D000F9EB28FEE93408FF751001880C750D064D
:1003E0008F0974027808121F2BC39508F8E4950949
:1003F000F9740228F50E740339F50F8E088F09740D
:10040000097808121F5DE508F511EE2410F508E4DF
:100410003FF509EEF50AEF5401F50B900383E01464
:1004200060541470030204EB147003020566146038
:100430001024FE70030206211470030206D1020686
:10044000E1750D03794E1213B29003071206F4748E
:1004500002F0A374401206F274081206F2F0A3F040
:10046000751012AA10A90C12070CA90D7408121EFF
:10047000467F0C021D7B750D04794E1213B2EE45BA
:100480000B7005A9111219DDC3EE9425EF940850E5
:100490003CC3E5089424E50994084031E50E249610
:1004A000F8E50F3420F988828983E0701BA3AA82C3
:1004B000AB83E070139003887401F08882898374A1
:1004C000A5F08A828B838004900388E4F07508107D
:1004D0007509007808121EDF7C087D03EEFAEFFB39
:1004E0001219777402121E46020463750D05E51198
:1004F000C394794006750C010204637512407513AC
:10050000007812121EDF7C097D037402780A121F24
:100510002BAA0AAB0BA9111218F27402121E4690F4
:100520000307E0A3F0900306E0A3F0751043C3EEC9
:100530009425EF94084003020463C3E5089424E57E
:100540000994085003020463900388E070030204D6
:1005500063E50E2497F8E50F3420F988828983E457
:10056000F0A3F00204637508047509007808121EF0
:10057000DF7402121F467A907B0079041218F2741D
:1005800002121E467402121F97E0F8A3E0F98518C4
:1005900082851983E0687003A3E069851882851954
:1005A00083700BE0F47003A3E0F470578009E0F46B
:1005B0007003A3E0F4700D8518828519837410F020
:1005C000A37420F01206FE121F97E8F0A3E9F0755D
:1005D00008017808121EDF7402121F467A247B0875
:1005E0001219777402121E467508047808121EDF6D
:1005F0007402121F467A907B0079041218F274027A
:10060000121E461206FE121F97E0687003A3E069EF
:100610007006750D01020463750D02750C07020466
:10062000639003D6E0600764026003020463EAFF9C
:100630007A01790012070CE060030206C5800312FC
:10064000117B121162E970F77404121F971206E60B
:100650007404121F977808121F7B85080C85090DFA
:10066000850A0E850B0F9003C2780C121F057404C7
:10067000121F97780C121F6CE5084509450A450BB7
:1006800070CE8EC2E5C554E04FF5C57404121F97B5
:100690001206E67404121F977808121F7B85080C57
:1006A00085090D850A0E850B0F9003C2780C121F69
:1006B000057404121F97780C121F6CE50845094554
:1006C0000A450B70CE7A01790012070C79080204F2
:1006D0006CEB900391F07003020463750D09020442
:1006E00063790602046CE4F0A37426F0A3E4F0A39B
:1006F000F022F0A3E4F0A3F0A3F0A3F0A322851866
:1007000082851983E0F8A3E0F974022274F6121BC3
:10071000D6EAFE900305E0D2E7F0E9A3F0EE9003FD
:1007200003F08E0A74042AFE7A028004E0620A0A48
:10073000EAF83395E012075B8E08C3E89508E99460
:1007400000A2D265D03340E4E50AF0740128F97ABA
:10075000027B0312111D7F03021D7BF9740228F531
:1007600082740339F5832274E9121BD675820075F1
:1007700083FE121E288A168B177514007515008AC1
:10078000828B83E4F09003D6E07006D2AAD2AF80C9
:1007900004640270057900120151750C00750D207A
:1007A000750E00750F009003D6E0600464027015AA
:1007B00012117B120176E9F874096860030208A33C
:1007C0007900120151E064027007A292400302080E
:1007D0007E7508007509027808121EDF7402121F68
:1007E00046850C08850D09AA08E5095407FB850E06
:1007F0000A850F0B740B7808121E96A9081218F2BE
:100800007402121E467E007F009003CAC0828E10C2
:10081000EFF5113395E0F512F513850C08850D09F8
:10082000850E0A850F0B78087910121F189003C6E1
:100830007808121F05758303D0827808121E0950AC
:100840001D851882851983E5822EF582E5833FF5A3
:1008500083E0F9AA14AB151208D28A148B150EEE98
:1008600070010FC3EF940240A09003CE780C121FCA
:10087000059003D2780C121E0940030207A67900E6
:10088000AA14AB151208D279001208D28B15900366
:10089000D6E07004C2AFC2AAEA451570277AA57BDC
:1008A000A58021E870030207C5740668700302077B
:1008B000C574076870030207C5851682851783749F
:1008C00001F080BA758200758302121E287F100223
:1008D0001D7BC008C0097C088A088B09740F780842
:1008E000121F5DEA25E0FAEB33FBE9A2E75004743E
:1008F000014AFAE508A2E0500874216AFA74106B04
:10090000FBE9C333F91CEC70CFD009D0082274F78F
:10091000121BD6120F2860030209E9A3E0F8A3E036
:1009200060030209E9A3E064027002A3E06003022D
:1009300009E99003B8E02480600914604F14605CFA
:100940000209E9E860030209E99003B2E060047873
:1009500001800278009003C0E8F0A3E4F09003B1B6
:10096000E0600A9003C0E04402F0A3E4F09003A624
:10097000E0640460149003B374C0F0A37403F0A3A4
:10098000E4F0A37402120F8AF002100A90039FE0B1
:10099000640470559003C0E4F0A380D0E8547FF560
:1009A0000890039FE064047040E508C39406503942
:1009B000749F2508F582E43403F583E854806018B9
:1009C000A3A3A3A3A3A3A3E06403700478018002FC
:1009D00078009003C0E88091E582240CF5825002F3
:1009E0000583E0640370E980E39003A674048098B3
:1009F00074F7121BD6E9FE9003BE120F2B600302A0
:100A00000AD190039FE06404600B9003BC120F2B8B
:100A10006003020AD19003B8E0541F6009146030EB
:100A2000146020020AD19003BAE064017022EE90B3
:100A300003B1F060047905800279067A00121BD4B4
:100A4000020AD79003BCE0547FFA9003BAE0600535
:100A50007900020AD9EAC394065076EA90620EF051
:100A6000749F2AF8E43403F99003BCE05480602CAE
:100A7000EE6004741080027440906211F0EE600425
:100A800074038001E488828983A3A3A3A3A3A3A3FF
:100A9000F0EE6004790880307907802CEE600474F1
:100AA0002080027480906214F0EE60047403800170
:100AB000E4C0E0E8240CF582E439F583D0E0F0EE00
:100AC0006004790A80027909121BD490620EE480D6
:100AD000059003A67404F0790102100A7900120946
:100AE000F0E97003121BC32279011209F0E97003C7
:100AF000121BD222C082C0839003BC120F2B701530
:100B0000A3120F2B700F9003BA120CD05480FAE985
:100B1000FBEA4B60079003A67404801AE890620019
:100B2000F090039F6009E06402700C74038007E09A
:100B3000640370037402F0D083D0822274F3121B1A
:100B4000D69003BAE0FAA3E01460081460101460B1
:100B500039805712175F120CADA37B80804179005A
:100B6000121781120CAD7B80E92402F9E43AFA12E3
:100B70001E7CFC1919E0FAA3E92403F9E43AFA12FD
:100B80001E7CF9ECA3F0A3E9801CEAF91217EF90A0
:100B900003B3EAF0A3EBF0A3E4120CBCA37B0012B6
:100BA0001E7CA3F0A3E4F0020C679003B3E4F0A36F
:100BB000F0A3F0F50B90047DE0FAA3E0FB020C42F9
:100BC00075090074037808121F2BEA2508F8EB3525
:100BD00009F99003BA120CC6E493C0E0EFFCD0E030
:100BE0006C705DA3E4936E70579003BC120CC6A3A7
:100BF000A3E493C0E0EFFCD0E06C7044888289836A
:100C0000A3A3A3E4936E703888828983A3A3A3A3CC
:100C1000E493F508740193F5099003B3E508F0A394
:100C2000E509F0A37480F088828983A3A3A3A3A31A
:100C3000A3E493F8740193F99003B6E8F0A3E9F004
:100C4000050B850B0890047F120CD0C39AF50CE9B4
:100C50009BF50D7403780C121F5DC3E508950CE439
:100C6000950D5003020BC09003B3E0FCA3E0FDA37D
:100C7000E0FEEC4D4E9003A6700474048029E064FD
:100C80000460259003BEE0FAA3E0FB9003B6E0F811
:100C9000A3E0F9C3EA98EB9950089003B6EAF0A3F1
:100CA000EBF09003A67401F07F06021D7B9003B366
:100CB000EAF0A3EBF0A37480120CBC22F09003B313
:100CC000E0F9A3E0FA22E0FEA3E0FF888289832214
:100CD000E0F8A3E0F9E82274EE121BD6EA2404F847
:100CE000E43BF9880889098882F583E493602590BC
:100CF0000481120CD0FEE9FF8007EE2404FE5001AF
:100D00000F8E828F83E493F8740193F9EA6870027E
:100D1000EB6970E6750C00803F9062147490F0747B
:100D200010120E2A7003750D408E828F83A3A3A329
:100D3000E49355106006E50DD2E0F50DE50D9062E7
:100D400015F0EA906213F0EC240CF582E43DF58393
:100D5000E4F090620EF0050C850882850983E49327
:100D6000F8E50CC3984003020E257A0079051216A7
:100D7000F28A0E8B0FEA450F60DCEA2402F8E435B4
:100D80000FF9880A890B8882F583E493540FF512D2
:100D900090620EF0750D008A828B83A3A3A3A3E457
:100DA000932407F510A3E4933400F511740378102D
:100DB000121F5DAA10851210749F2510F8E43403E9
:100DC000F9E8FCE9FD751001751100E512781012C3
:100DD0001F2BE50E2403F8E4350FF9850A82850BF5
:100DE00083E493A2E74003020D199062117448F066
:100DF0007408120E2A7003750D408E828F83A3A390
:100E0000E49355106006E50DD2E0F50DE50D906216
:100E100012F0EA906210F08C828D83A3A3A3A3A3A7
:100E2000A3A3020D507F0B021D7BF088828983E40F
:100E3000935403640122C082C083120F287010A350
:100E4000120F2B700AA3E064017002A3E060079008
:100E500003A67404800C9003B374A0F0A37403126F
:100E60000F80F0020B3774F4121BD690039FE064DE
:100E70000260149003BC120F2B700CA3120F2B7086
:100E8000069003BBE060099003A67404F0020F23F0
:100E90007A007901121BD49003BAE060717A00F9EC
:100EA0001217818A088B09EA4509605A90039F74DA
:100EB00004F09003BAE09003A0F0750C008508825E
:100EC000850983A3A3A3A3E493F8E50CC398504C2E
:100ED000850C0A74A1250AF8E43403F9E8FEE9FF59
:100EE0008E828F83E4F07A0079041216F28A828B64
:100EF00083A3A3A3E493F88E828F83E06870E71244
:100F00000CD7050C80B79003A67404F0800E9003F4
:100F1000A0F090039F7403F0F91216587A0079023A
:100F2000121BD47F05021D7B9003BAE0F8A3E0F901
:100F3000E8492274F6121BD690039FE064047019EE
:100F40009003B8E064817011120F28700C9003BEFA
:100F5000E064017002A3E060079003A67404801AA5
:100F60009003BCE024A1F508A3E03403F509900345
:100F7000B3E508F0A3E509120F80F07F03021D7BA3
:100F8000F0A3E4F0A304120F8A22F0A3E4F090038C
:100F9000A6042274F7121BD690039FE064047064C9
:100FA0009003B8E06401705C9003BE120F2B705484
:100FB0009003BAE0FB9003BCE0FA9003A0E0F912C2
:100FC00017B98A088B09AE08AF09EE4F6036900357
:100FD000BCE0FA7903121BD49003BAE0C0E090039E
:100FE000BCE024A1F8A3E03403F988828983D0E02F
:100FF000F0EEFAEFFB120CD79003BCE0FA79041282
:101000001BD480069003A67404F07F02021D7BC0EF
:1010100082C0838003121A39A2E840F9A823E85459
:101020000460097823E654FBF6121402A823E8545E
:101030001060097823E654EFF6121420A823E8A2E2
:10104000E05005782354FCF690620EE0FA7404F048
:10105000906214E0A2E0503AE5A8F8C2AF906216A0
:10106000E0F9A3E0E9FBE8A2E792AF8017906228DD
:10107000E0C0E0900393E0F8121112D0E0F090038A
:1010800093E004F0EBFC74FF2C1B0470E0906214FE
:10109000E4F0EA90620EF0E0FD7404F0906211E07A
:1010A000A2E04031900395E0F8900394E068602559
:1010B0007A40900394121155E0906228F0900394C6
:1010C000E004F008900395E06860041AEA70E39089
:1010D00062117401F0ED90620EF0D083D082227420
:1010E000F8121BD6E9FE79008012121112E08A82F2
:1010F0008B83F0900392E00412114A09900392E06E
:10110000F8900393E0686005E9C39E40DD7F01022B
:101110001D7B748528F582E43404F58322C082C0E7
:1011200083E9FC80188A828B83E0C0E090039512EB
:101130001155D0E012114A900395E004F0ECF874D8
:10114000FF281C0470DF79018090F08A828B83A3D2
:10115000AA82AB8322E0F8748528F582E43405F591
:101160008322C082C083900395E0F8900394E068E6
:1011700060047901800279000210DA02100F74FB1A
:10118000121EC57E009006857808121F7B794A12D0
:1011900013B29006857401F0A3F0A37469F0A374F0
:1011A000A5F09003D77808121EF070030E801590FA
:1011B00003DB7808121EF06008E59D541864107077
:1011C00003022000EEF9121329C280D291EEA2E0B0
:1011D00050030212DCAA18AB19120288E97003024C
:1011E00012DCC291851882851983E0C3943C500EAD
:1011F000E0F8743CC398F50895E0F5098006750899
:1012000000750900E4F50AF50B9003DF780C121F56
:101210007B7808790C121ADA790612015112100F34
:10122000120176E9F8740968700779061201518095
:10123000277407686016A2935012E8600874066865
:1012400060030212DCA292400F0212DC75080075E6
:101250000900750A00750B0085080C85090D850AC3
:101260000E850B0F9003C27808121F05E50C450D83
:10127000450E450F70A7D2807907120151800312E5
:10128000100F121162E970F77E007F007401121FC7
:1012900097E4F0A37426F0A3E4F0A3F07401121F06
:1012A000977808121F7B85080C85090D850A0E8525
:1012B0000B0F9003C2780C121F057401121F977850
:1012C0000C121F6CE5084509450A450B70CEA29229
:1012D00050FCA29350F81213AD022000D280D2919C
:1012E000794E1213B2750800750900750A00750B66
:1012F00000790512015112100F120176E9F87409F4
:101300006860EE74016870EE12100F9003E37808C5
:10131000121F059003E77808121E0950EB1213AD57
:101320000220007405121E462274F8121BD6E9FE34
:1013300053BEFBE59DA2E650FA0078F8790100E87B
:1013400024FF18E934FFF9E84970F375C68074800A
:10135000659E70FA43BE049062707408F01213A286
:10136000EE700853F4FEC29043FE017403F5D57588
:10137000D489900396E4F0A374C2F0A37401F0A39F
:10138000E4F0A3F0A3F0A37408F01213C87AFF7B73
:10139000FF1219F453F4FED29043FE011213A2027D
:1013A000110DD28043FD01C29143FE0222D280C2C0
:1013B0009122781075B60FE5B4A2E750FAE5BBC3E9
:1013C0009940F118E870ED22C082C0837A0079015B
:1013D0001217818A828B83A3A3A3A3A3A3A3E4935D
:1013E000A2E69003B2500474018001E4F09003B1CE
:1013F000E4F090620F7403F0E0A2E750FBD083D0DA
:101400008222C082C08390039F7402F0A3E4F09014
:1014100003A6F0790312165875210075220080DDAD
:1014200074F6121BD690620EE0FEE4F0906211E0BA
:10143000FFA2E4501D7480F09003A67407F0E5212C
:1014400045226009852182852283121FA69003A66A
:10145000E4F0EFA2E2500B906211E4F09003A6F0EA
:1014600080669003A6E0F87402687045906216E00A
:10147000FF9003B3121DBBEFF97A207B6212168C2A
:101480007403121E468F089003B612163C121634CF
:101490002F121647E0F8A3E0F9E849600474408091
:1014A000027448906211F0E849600302162A02169D
:1014B000067406687009852182852283121FA69012
:1014C00003A6E060030215B1EFA2E0400302162A72
:1014D0007508B8750903750A007808121EDB7908CB
:1014E0007A207B6212168C7403121E4675210075D9
:1014F00022009003B8E054E0601D24E07003021560
:101500008D24E0607224C0604824E07003021598C6
:1015100024E0606E0215A3A3E014602624FE601D83
:1015200024FE600A24FC601F24FE60208075120ADD
:10153000F49003A6E06404707274608070120AE88C
:1015400080EF120ADC80EA120E6680E5120F9380AB
:10155000E0A3E0600E24FA600F24FE601024FE6019
:1015600011804012090E80C9120B3C80C4120E3645
:1015700080BF120F3380BA7521BF75221B121BBFAB
:1015800080AF7521C175221B121BC180A475215A21
:1015900075221B121B5A809975218A75221B121BFA
:1015A0008A808E9003A67404F0808E74409062113D
:1015B000F09003A6E0F874016870617F029003B6B2
:1015C000E0F8A3E0F9C3E89420E994005007E8F5B7
:1015D0000A7F0A8003750A209003B3121DBBA90A73
:1015E0007A207B621216B77403121E46850A08120F
:1015F0001634250812164712163CEF906211F0E5DA
:101600000AC394205024E521452260098521828562
:101610002283121FA69003A6E4F0800E7405687062
:1016200009852182852283121FA6EE90620EF07F2B
:1016300003021D7B9003B31216E4E922C3E0950870
:10164000F0A3E09400F022F9E43AFA9003B3E9F051
:10165000A3EAF0A3EBF0A32274F7121BD678007470
:10166000A728F582E43403F583E9F008E8C394057C
:1016700040ED780074AC28F582E43403F583E9F09A
:1016800008E8C3940540ED7F02021D7B74F8121B2D
:10169000D6EAFCEBFDE9F87408121F971216DF601A
:1016A000118C828D83E0121EAFE9240109E43AFA1D
:1016B000D8EF7F01021D7B74F8121BD6EAFCEBFD0C
:1016C000E9F87408121F971216DF6011121E7C8C45
:1016D000828D83F0E9240109E43AFAD8EF80D3122D
:1016E00016E4E822E0F9A3E0FAA3E0FB22D083D0DD
:1016F0008222C082C083E9FCEAFD7A007B0080037D
:1017000012173D90039DE0F8A3E0F990047BE06898
:101710007003A3E069602490039EE0F5838882A3B0
:10172000E493F8EC68700D90039DE0FAA3E0FB12DF
:10173000173D8007ED6870C8ED60C580B090039DCF
:10174000E0F8A3E0F5838882E493F890039DE02815
:10175000F8A3E03400F990039DE8F0A3E9F022C07B
:1017600082C0831217707A0079011216F20216ED08
:10177000900479E0F8A3E0F990039DE8F0A3E9F084
:101780002274F7121BD6E9FEEAFF1217707A00796D
:10179000021216F2EA4B601CEE60108A828B83A361
:1017A000A3A3A3A3E4936E70E48009EFF874FF2869
:1017B0001F0470D97F02021D7B74F5121BD6EAFF4D
:1017C0008B087A001217817A0279041216F2EA4B1A
:1017D00060188A828B83A3A3E4936F70EA8A828B5A
:1017E00083A3A3A3E493650870DD7F04021D7B74CB
:1017F000F7121BD674F0121EC5E97A007B00600C4C
:101800001460101460141460180218DB7AF37B0360
:101810000218DB7AF77B030218DB7A1B7B040218C1
:10182000DB90043FE060030218D79003EB740812CA
:101830001F467408121DE8750808F5097808121E7D
:10184000DF7402121F467AE87B07797F1218F27460
:1018500002121E467808121EDF740A121F46740216
:10186000121F3E121C997402121E468B09EA45098A
:1018700070197509007808121EDF7C0C7D787402DF
:10188000121F3E121D357402121E467C287D0085F3
:101890001882851983E5822DF582E43583F583E08E
:1018A000FF743F2CF8E43404F9EF1218E3888289BE
:1018B00083F0EFC41218E3C0E0E824FEF582E934B7
:1018C000FFF583D0E0F00D74FC2CFCEDC3940840D0
:1018D000BE90043F742AF07A3F7B047410121E46B7
:1018E0000217B4540FFA74692AF582E43404F583BC
:1018F000E02274F5121BD68908740F5508F50A7595
:101900000B00740B780A121F2BEA2400F8EB3480CA
:10191000F9E82400E9350BF9E5C7F509A2AFE4338E
:10192000F50AC2AFE508C4540FFAE5C754F84AF502
:10193000C7740B121F97E0FAA3E0FB801C88828912
:1019400083E08C828D83F088828983A3A882A98317
:101950008C828D83A3AC82AD83EAFEEBFFEE24FF85
:101960001AEF34FFFBEE4F70D48509C7E50AA2E0F9
:1019700092AF7F04021D7B74F7121BD6ED90038992
:10198000F0ECA3F0A37462F0A37473F0A3E0541F0F
:10199000F07409121F97E0F508A3E0F509E5083394
:1019A0003354FC90038EF074067808121F5DE5082E
:1019B00090038DF090038F7412F0A37442F075D1F0
:1019C000FE75D601EA906271F0EBA3F0906270E0D0
:1019D000D2E1F0E0A2E740FB7F02021D7BC082C0A3
:1019E00083E9C333906272F0906270E0D2E0F0D08D
:1019F00083D0822274F7121BD675230075240075DC
:101A000025008A268B27EA90620BF08A088B0974DE
:101A1000047808121F5DE508906207F08A088B09B8
:101A200074097808121F5DE508543E906209F0754C
:101A30008B00C2E87F02021D7B74F7121BD6E59D66
:101A4000A2E650FA906206E0FAA2E25035A826E833
:101A500090620BF0F50885270974047808121F5D61
:101A6000E508906207F0852608852709740978083B
:101A7000121F5DE508543E906209F0906201E0D2C9
:101A8000E0F07823EA46F6906202E0F50875090076
:101A900074047808121F2B7823E50846F608E50938
:101AA00046F6906204E0F50875090074097808129A
:101AB0001F2B7824E50946F6EAA2E05003752501BC
:101AC00074065A6003752500E58BA2E55006758BF8
:101AD000DF752500121BD5021A2F080808EAC0E09E
:101AE000EBC0E086F0E7A4FA180986F0E7A42AFA2A
:101AF000180986F0E7A42AFA180986F0E7A42AFA5A
:101B00001986F0E7A4FBE5F02AFA190886F0E7A4A5
:101B10002BFBE5F03AFA190886F0E7A42BFBE5F079
:101B20003AFA18180986F0E7A4C5F02BFBE43AFA54
:101B30001908E7C5F0C6A426F6E5F03BFBE43AFA3F
:101B40001886F0E7A4F6E5F00826F6E43B08F6E48C
:101B50003A08F6D0E0FBD0E0FA22C082C0839003BE
:101B6000B9E0F874226870089003A6E0701A80113A
:101B70007420689003A6700DE0700D121BB19003E5
:101B8000A6740280027404F08043C082C083900374
:101B9000B9E064219003A67013E07013121BB1A387
:101BA0007407F0A3E4F09003A60480027404F080AC
:101BB0001C9003B37496F0A37403F0A3E4F02280A6
:101BC000028000C082C0839003A67404F0D083D04A
:101BD000822280EF22222518C582C0E0E51934FF59
:101BE000C583C0E0E518C3958224F910AF0885834A
:101BF000198582188008858319858218D2AFCEF0A6
:101C0000A3E520F0A37808E608F0A3DEFAEFF0A33E
:101C1000E58124FBF8E608F0A3E608F0A30808E64F
:101C200008F0A3E608F0A315811581D0E0FED0E00E
:101C3000F815811581E8C0E0EEC0E0221201000233
:101C4000020000205104A816090001020301090244
:101C50004300020100801909040000010202010092
:101C600005240010010424020205240600010524B5
:101C70000100010705820340004009040100020A37
:101C80000000000705840240000007050402400030
:101C900000571C00007A1C000074F5121BD6740B50
:101CA000121F97E0F8A3E08015A3AA82AB838C8271
:101CB0008D83A3AC82AD83E824FF18E934FFF9E8F3
:101CC00049601F8C828D83E0F5088A828B83E0F562
:101CD0000AE508650A60D2E50AC39508FA95E0FBB3
:101CE00080047A007B007F04021D7BE47921780761
:101CF000B800028004F709D8FCE490030278C179A7
:101D0000018002F0A3D8FCD9FA7AC27B0390008E3E
:101D100078C479018015E493A3AD82AE838A828B67
:101D200083F0A3AA82AB838D828E83D8E9D9E71290
:101D3000117E121FA174F7121BD6EAF8EBF9740991
:101D4000121F97E0FEA3E0FF80188C828D83E0884D
:101D5000828983F0A3A882A9838C828D83A3AC821D
:101D6000AD838E088F09E50824FF1EE50934FFFFC7
:101D7000E508450970D47F02021D7B85198385180B
:101D800082E0A3FEE0A3F5207808E0A3F608DFFADE
:101D9000E0A3FFE0A3C0E0E0A3C0E0E0A3C0E0E078
:101DA000A3C0E010AF08858218858319800885825A
:101DB00018858319D2AFD083D0822274038000CCDF
:101DC000C0E0EDC0E0E518C39CCCAD1950011D107A
:101DD000AF068C188D1980068C188D19D2AF121D84
:101DE000E8D0E0FDD0E0FC22CAC0E0E0A3C582CC90
:101DF000C582C583CDC583F0A3C582CCC582C5830A
:101E0000CDC583DAE6D0E0CA22C008C3E096F50863
:101E100008A3E096420808A3E096420808A3E096CB
:101E200045087001D3D00822C5822518C582C58314
:101E3000351910AF07F5198582188007F5198582C5
:101E400018D2AFC5832200C0D0251810AF08F518EE
:101E5000500C05198008F51850020519D2AFD0D0E2
:101E6000222518F58210AF08F518400C15198008C6
:101E7000F51840021519D2AF85198322BB0102E77C
:101E800022C082C08389828A83BB0003E08002E48F
:101E900093D083D082226016080808C6C313C618E0
:101EA000C613C618C613C618C613C6D5E0EA22BBA9
:101EB000000EC082C0838A838982F0D083D08222C0
:101EC000BB0101F722251810AF08F518400C1519B1
:101ED0008008F51840021519D2AF227403800474EB
:101EE000028000C0E0F404121E61D0E0121F8A22BA
:101EF000E066701008A3E066700A08A3E06670044C
:101F000008A3E06622E026F608A3E036F608A3E080
:101F100036F608A3E036F622E627F60809E637F695
:101F20000809E637F60809E637F622700422600D44
:101F300018C6C333C608C633C6D5E0F41822251820
:101F4000FAE43519FB222518FCE43519FD2275D079
:101F50000075813F751802751903021CEB600C08AF
:101F6000C6C313C618C613C6D5E0F422E6F008A30C
:101F7000E6F008A3E6F008A3E6F022E0F608A3E006
:101F8000F608A3E0F608A3E0F622CAC0E0E6F0A354
:101F900008DAFAD0E0FA222518F582E43519F5833B
:101FA0002200000080FBE473FFFFFFFFFFFFFFFF45
:101FB000FFFFFFFFFFFFFFFFFFFFFFFFFFFFFFFF31
:101FC000FFFFFFFFFFFFFFFFFFFFFFFFFFFFFFFF21
:101FD000FFFFFFFFFFFFFFFFFFFFFFFFFFFFFFFF11
:101FE000FFFFFFFFFFFFFFFFFFFFFFFFFFFFFFFF01
:0A1FF600850609433886000000004C
:020000040003F7
:01FFF000F020
:020000040000FA
:10200000022DA8022220FFFFFFFFFFFFFFFFFFFFBF
:10201000FFFFFFFFFFFFFFFFFFFFFFFFFFFFFFFFD0
:10202000FFFFFFFFFFFFFFFFFFFFFF022A6CFFFF25
:10203000FFFFFF022243FFFFFFFFFFFFFFFFFFFF46
:10204000FFFFFFFFFFFFFFFFFFFFFFFFFFFFFFFFA0
:10205000FFFFFF02215CFFFFFFFFFFFFFFFFFFFF0E
:10206000FFFFFFFFFFFFFFFFFFFFFF022A44FFFF0D
:10207000FFFFFFFFFFFFFFFFFFFFFF022895FFFFAE
:10208000FFFFFF0221BC01FFFFFFFFFFFFFFFFFF7C
:102090001020102001FF01010503010F10FEFFF4C5
:1020A0004E000000008C4E00000000FF000000FF0A
:1020B00000010000153B00000000673A5F3CAF3AAA
:1020C000C93B00009D3A0000000000000000000035
:1020D0000000000000000000000000000000FF0100
:1020E0000100A907000000E803FFFF2408E80364DB
:1020F000006400B8010202000800000502070101A7
:10210000051E02051E020A0A0103B80B02803E01E9
:1021100002FEFFE8030A050001FFFF0A01E00020BC
:10212000FD000206FFFF00035F005F003000580063
:10213000000000000000000000000000000000009F
:10214000000000000000000000000000000000008F
:10215000B42609270927092709271127C0E074F2A7
:10216000122655A2AFE433FED2AFE5A7FFE5A1F5F5
:10217000085F541060061245CB75A1EFE5085F5467
:102180000860081245D175A1F78024E508A2E09205
:10219000F0EFA2E082F05017906198E0F89009818A
:1021A000E0C398A2D265D0335002E8F075A1FE7565
:1021B0001A00EEA2E092AF7F01022711C0E074F294
:1021C000122655A2AFE433FED2AF9061A4E0F875B9
:1021D0009B00E59158540860087591F712461980E4
:1021E00023E59158541060087591EF12461F801432
:1021F000E591A2E092F0E8A2E082F05007E0C2E0B0
:10220000F01247759061A3E0F8E5E9585404600EB8
:1022100012474B75E9FB906193E0A2E640F2808F94
:10222000C0E074F2122655A2AFE433FED2AF906143
:10223000A5E0F8E5BF585404600675BFFB12478D52
:102240000221AFC0E074F1122655E59DA2E650FAD6
:10225000906206E0FAA2E25035A82CE890620BF0FA
:10226000F508852D0974047808122DB8E5089062E8
:1022700007F0852C08852D0974097808122DB8E51A
:1022800008543E906209F0906201E0D2E0F07829B3
:10229000EA46F6906202E0F50875090074047808D1
:1022A000122D447829E50846F608E50946F69062BD
:1022B00004E0F50875090074097808122D44782A9D
:1022C000E50946F6EAA2E05003752B0174065A6050
:1022D00003752B00E58BA2E55006758BDF752B008F
:1022E00012493D758B00C2E87F02022711C3E498B2
:1022F000F8E499F912232E8026C3E49AFAE49BFBB2
:10230000E920E7E912232EE498F8E499F922C3E4DE
:1023100098F8E499F912232EE498F8E499F9C3E4C3
:102320009AFAE49BFB22EB20E7CFE920E7E0B90033
:1023300010BB0008E88AF084F8AAF022E4FBC8FA8F
:1023400022EB70227B10C833C8C933C9335007C38E
:102350009AC3DBF280069A50012ADBEAC833F4C83C
:10236000C933F4C9FA2275F008E4C833C8C933C9BF
:1023700033C99AC99B5004C92AC93BD5F0ECFBC8A4
:1023800033F4C8E4C9FA2274F51225EF74FA122C5A
:10239000187508047509007808122B567404122B5E
:1023A000FA7AF87B0779031244A57402122B849001
:1023B00080FC7808122DD67402122E2D7808122C6B
:1023C0004470497508027509007808122B5674028A
:1023D000122BFA7AF67B0779031244A57402122BAA
:1023E00084851882851983E0F47003A3E0F4601CEF
:1023F000851882851983E0F8A3E0F98882898374BF
:1024000002F0A3F0A37469F0A374A5F0C2AF75D66F
:102410009F0200007406122B847F040228D808084B
:1024200008EAC0E0EBC0E086F0E7A4FA180986F0FD
:10243000E7A42AFA180986F0E7A42AFA180986F010
:10244000E7A42AFA1986F0E7A4FBE5F02AFA1908AE
:1024500086F0E7A42BFBE5F03AFA190886F0E7A42A
:102460002BFBE5F03AFA18180986F0E7A4C5F02B23
:10247000FBE43AFA1908E7C5F0C6A426F6E5F03BF6
:10248000FBE43AFA1886F0E7A4F6E5F00826F6E44D
:102490003B08F6E43A08F6D0E0FBD0E0FA22122E30
:1024A00022B900030224FEE47921780DB8000280ED
:1024B00004F709D8FCE49004D17865790C8002F027
:1024C000A3D8FCD9FA781A9020867A01BA00028043
:1024D00007E493A3F608DAF97A357B109020947814
:1024E000C979018015E493A3AD82AE838A828B8380
:1024F000F0A3AA82AB838D828E83D8E9D9E7758257
:10250000DC7583987406122B3075821F75834C74AA
:1025100000122B30E4CFC0E0E4CEC0E0E4CDC0E058
:10252000E4CCC0E075F020E626F608E633F608E6CF
:1025300033F608E633F6181818EC33FCED33FDEEED
:1025400033FEEF33FFC3EC9709ED9709EE9709EFE0
:1025500097191919400FFFEC97FC09ED97FD09EE4B
:1025600097FE191906D5F0BFECF709EDF709EEF75C
:1025700009EFF7191919D0E0FCD0E0FDD0E0FED04A
:10258000E0FF222518C582C0E0E51934FFC583C0ED
:10259000E0E518C3958224F810AF08858319858279
:1025A000188008858319858218D2AFCEF0A3E52064
:1025B000F0A37808E608F0A3DEFAEFF0A3E58124A3
:1025C000FAF8E608F0A3E608F0A3E608F0A3080886
:1025D000E608F0A3E608F0A315811581D0E0FED04F
:1025E000E0F8158115811581E8C0E0EEC0E02225F4
:1025F00018C582C0E0E51934FFC583C0E0E518C303
:10260000958224F910AF0885831985821880088582
:102610008319858218D2AFCEF0A3E520F0A3780805
:10262000E608F0A3DEFAEFF0A3E58124FBF8E60864
:10263000F0A3E608F0A30808E608F0A3E608F0A374
:1026400015811581D0E0FED0E0F815811581E8C034
:10265000E0EEC0E022C0D02518C582C0E0E5193404
:10266000FFC583C0E0E518C3958224F310AF088549
:1026700083198582188008858319858218D2AFC88E
:10268000F0A3E9F0A3EAF0A3EBF0A37908E709F0DF
:10269000A3D8FAECF0A3EDF0A3EEF0A3EFF0A3D0F3
:1026A000E0F0A3D0E0F0A3D0E0F0A3E520F0A3E5B4
:1026B000F0F0A32212010002020000205104A8162B
:1026C0000900010203010902430002010080190907
:1026D000040000010202010005240010010424028C
:1026E00002052406000105240100010705820340BC
:1026F000004009040100020A0000000705840240AE
:10270000000007050402400000CF260000F226006A
:1027100000851983851882E0C0E0A3E0F9A3E0FA00
:10272000A3E0FBA37808E0F608A3DFFAE0FCA3E04F
:10273000FDA3E0FEA3E0FFA3E0C0E0A3E0C0E0A3B0
:10274000E0F5D0A3E0F520A3E0A3F5F010AF0885F5
:1027500083198582188008858319858218D2AFD0A5
:1027600082D083D0E0F8D0E032E4730875F0108EA8
:10277000218F22858226858325851882851983E00D
:10278000CEA3E0CF852682852583EBC9EAC8EDCBB1
:10279000ECCAC3E833C8E933C9EA33CAEB33CBC365
:1027A000EA9EF524EB9FF523B35004AB23AA24EC57
:1027B00033CCED33CDD5F0DAAE21AF2222D083D0A9
:1027C00082ECC0E0EDC0E0E493A3FCE493A3FDED54
:1027D0004C600D122918EC24FFFCED34FFFD80EF56
:1027E000E493A3FCE493A3FDED4C600D1229EFEC00
:1027F00024FFFCED34FFFD80EFD0E0FDD0E0FCE4F1
:1028000093A3C0E0E493C0E022851983851882E099
:10281000A3FEE0A3F5207808E0A3F608DFFAE0A322
:10282000FFE0A3C0E0E0A3C0E0E0A3C0E0E0A3C0FD
:10283000E0E0A3C0E010AF08858218858319800806
:10284000858218858319D2AFD083D082022B36D0EF
:1028500083D082E9C0E0E493A3C386F0C5F095F08D
:10286000F908E493A386F0C5F095F0700BE493A308
:10287000C3994005E9048002A3E475F002A425820F
:10288000F582E5F03583F583D0E0F9E493A3C0E069
:10289000E493C0E022C0E074F2122655A2AFE43304
:1028A000FED2AFE58AA2E25007900942E0D2E0F002
:1028B000E58AA2E35007900942E0D2E1F0758A0070
:1028C000C2EB7A107B0090093EE0F9123DF1EEA2D6
:1028D000E092AF7F01022711851983851882E0A35A
:1028E000FEE0A3F5207808E0A3F608DFFAE0A3FFF6
:1028F000E0A3C0E0E0A3C0E0E0A3C0E0E0A3C0E04C
:1029000010AF088582188583198008858218858311
:1029100019D2AFD083D08222C0E0C3E4939608746A
:1029200001939618400FE49366700808740193664B
:102930001870007019A3A3C3E493960874019396CA
:1029400018A3A3400DD0E0D0E0D0E00227F9A3A364
:10295000A3A3A3A3D0E022D083D082C5F0E493A3A5
:10296000C5F0C395F0F5F0E493A3C395F04005E5F9
:10297000F0048001E475F002A42582F582E5F035CB
:1029800083F583E493A3C0E0E493C0E02274048061
:10299000087403800474028000CCC0E0EDC0E0E560
:1029A00018C39CCCAD1950011D10AF068C188D19A1
:1029B00080068C188D19D2AF122AB2D0E0FDD0E07B
:1029C000FC2274028000CCC0E0EDC0E0E518C39C9E
:1029D000CCAD1950011D10AF068C188D1980068CD6
:1029E000188D19D2AF122A90D0E0FDD0E0FC22C0A1
:1029F000E0C0F088F0E493667008087401936618EC
:102A00007000A8F0A3A3700BD0F0D0E0D0E0D0E02D
:102A10000227F9A3A3D0F0D0E022D083D082CCC08B
:102A2000E0E493A36006122AD31470FAE493A3603F
:102A300006122C021470FAD0E0FCE493A3C0E0E488
:102A400093C0E022C0E074F2122655758900C2C519
:102A500090102DE0700E7A007B1090071DE0F912A7
:102A60003DF18003124A817F01022711C0E0C0D0EE
:102A7000E8C0E0E9C0E0E5A8D2AFC2C7751A00A27D
:102A8000E7A2E792AFD0E0F9D0E0F8D0D0D0E032C2
:102A9000CAC0E0E493A3C582CCC582C583CDC583FB
:102AA000F0A3C582CCC582C583CDC583DAE5D0E06D
:102AB000CA22CAC0E0E0A3C582CCC582C583CDC509
:102AC00083F0A3C582CCC582C583CDC583DAE6D0A9
:102AD000E0CA22C0E0E493A3D39C5010E493A3C3C4
:102AE0009C400AD0E0D0E0D0E0022A37A3A3A3D0D4
:102AF000E0227009080808226016181818C6C333A7
:102B0000C608C633C608C633C608C633C6D5E0EA0B
:102B100022C008C3E096F50808A3E096420808A37F
:102B2000E096420808A3E09645087001D3D0082239
:102B3000C09FF59FE473D09F22D083D082C09FE4D2
:102B400093C0E0740193C0E0740293F59F22740473
:102B5000800A74038006740280027401C0E0F404E9
:102B6000122B69D0E0122DE5222518F58210AF084E
:102B7000F518400C15198008F51840021519D2AF48
:102B80008519832200C0D0251810AF08F518500C05
:102B900005198008F51850020519D2AFD0D022BB14
:102BA0000102E722C082C08389828A83BB0003E0DE
:102BB0008002E493D083D082226016080808C6C33E
:102BC00013C618C613C618C613C618C613C6D5E052
:102BD000EA22C3E0C696F608A3E0C696F608A3E08C
:102BE000C696F608A3E0C696F6222518F8E435192D
:102BF000F9222518FAE43519FB222518FCE43519C9
:102C0000FD22C0E0E493A36C7009D0E0D0E0D0E0F6
:102C1000022A37A3A3D0E022251810AF08F51840E8
:102C20000C15198008F51840021519D2AF22BB0007
:102C30000EC082C0838A838982F0D083D08222BB77
:102C40000101F722E066701008A3E066700A08A38D
:102C5000E066700408A3E06622C3E09608A3E0964D
:102C600008A3E09608A3E096A2D265D03322E766D7
:102C700070100809E766700A0809E7667004080919
:102C8000E76622C3E096F008A3E096F008A3E0967A
:102C9000F008A3E096F022C3E4939608740193969B
:102CA0000874029396087403939622C3E697F60875
:102CB00009E697F60809E697F60809E697F622E08E
:102CC00026F608A3E036F608A3E036F608A3E036B9
:102CD000F622E657F60809E657F60809E657F60819
:102CE00009E657F622E056F608A3E056F608A3E0F8
:102CF00056F608A3E056F622E056F008A3E056F098
:102D000008A3E056F008A3E056F022E627F60809EB
:102D1000E637F60809E637F60809E637F622E02630
:102D2000F008A3E036F008A3E036F008A3E036F0A0
:102D300022E647F60809E647F60809E647F60809D5
:102D4000E647F622700422600D18C6C333C608C6D3
:102D500033C6D5E0F41822E4C396F608E496F608E4
:102D6000E496F608E496F622C6F4C608C6F4C60849
:102D7000C6F4C608C6F4C622600D08C6A2E713C68C
:102D800018C613C6D5E0F322C3E7960809E79608EC
:102D900009E7960809E79622C3E09608A3E096089B
:102DA000A3E09608A3E0962275D00075813F7518C0
:102DB000D17519040002249E600C08C6C313C618FE
:102DC000C613C6D5E0F422E6F008A3E6F008A3E6B1
:102DD000F008A3E6F022E0F608A3E0F608A3E0F688
:102DE00008A3E0F622CAC0E0E6F0A308DAFAD0E0D1
:102DF000FA22EAF0A3EBF0A3ECF0A3EDF022E0FA64
:102E0000A3E0FBA3E0FCA3E0FD22E0F8A3E0F9A32C
:102E1000E0FAA3E0FB22E8F0A3E9F0A3EAF0A3EBD9
:102E2000F022E5C754F84401F5C77901222518F5C9
:102E300082E43519F58322122B39D9A903122B39D3
:102E40003AAA03122B3979AC03122B394DAE031277
:102E50002B392CAF03122B3965B003122B3918B361
:102E600003122B392BB603122B393AB603122B3926
:102E7000C6B603122B397CB703122B39C3B7031222
:102E80002B390CB803122B3948B803122B39BEB8B2
:102E900003122B392AB903122B3946B903122B39E5
:102EA00077B903122B39B6B903122B39B7BA03120B
:102EB0002B3966BB03122B39F7BD03122B3950BFD8
:102EC00003122B39E3BF03122B396DC003122B39C8
:102ED000D3C003122B3912C103122B3988C103123C
:102EE0002B39DDC203122B3980C303122B3998C34F
:102EF00003122B393BC403122B39C5C603122B39DD
:102F000066C803122B3984C803122B3900800212C1
:102F10002B395A8002122B39C48002122B394D8171
:102F200002122B39098202122B39518202122B39DB
:102F30008C8202122B39E28202122B394A8302124E
:102F40002B39CE8302122B39E78302122B390C84E2
:102F500002122B394A8402122B39998402122B391E
:102F6000C28402122B39118502122B39BD8502123F
:102F70002B39858602122B39EA8602122B39B78744
:102F800002122B39FD8702122B39198802122B39B4
:102F90004B8802122B39F38902122B39CA8A02128A
:102FA0002B39F68A02122B392C8B02122B394D8BBE
:102FB00002122B395C8B02122B39678B02122B39D0
:102FC0001B8C02122B398E8C02122B39008D0212AF
:102FD0002B39088D02122B39838D02122B39DC8D8F
:102FE00002122B391F8E02122B39B19002122B398B
:102FF000F79102122B39879402122B396F95021226
:103000002B39A29502122B39649602122B39139791
:1030100002122B395B9702122B39BD9702122B3902
:10302000E29702122B39F39702122B396B98021296
:103030002B39F39802122B39579902122B393C9AEB
:1030400002122B39619A02122B39829B02122B3900
:10305000A09B02122B39B39B02122B39269C021221
:103060002B39359C02122B39BD9C02122B39059D40
:1030700002122B39129D02122B391B9D02122B3981
:103080001B9F02122B396FA002122B397FA0021254
:103090002B399BA102122B3914A202122B394AA3FD
:1030A00002122B398CA302122B39C8A302122B391E
:1030B0009CA502122B3901A802122B3915A8021265
:1030C0002B391FA802122B3929A802122B3933A839
:1030D00002122B393DA802122B3956A802122B39A5
:1030E00060A802122B396AA802122B3974A80212A6
:1030F0002B39A3A802122B39CBA802122B39D6A840
:1031000002122B3920A902122B392AA902122B39BB
:1031100035A902122B3959A902122B397DA90212A5
:103120002B39DEA902122B3929AA02122B3945AA02
:1031300002122B39AFAA02122B39FBAA02122B3929
:1031400043AB02122B39BEAB02122B3958AC021220
:103150002B391CAE02122B398AAE02122B39BCAFAE
:1031600002122B39E2AF02122B3952B102122B3963
:1031700006B502122B3906B702122B39DEB802123D
:103180002B3977B902122B3989BB02122B394BBC70
:1031900002122B3997BC02122B39FDBC02122B39BB
:1031A0000FBD02122B395FBF02122B394EC0021223
:1031B0002B398DC102122B39DFC102122B3984C287
:1031C00002122B393FC402122B3970C502122B395F
:1031D0008EC502122B39E3C502122B39E1C6021249
:1031E0002B3909C702122B396CC702122B396DC853
:1031F00002122B39E0C802122B390ECA02122B39E7
:1032000079CA02122B3969CB02122B39CFCD0212A7
:103210002B39FDCD02122B39F8CE02122B3996D064
:1032200002122B39E6D002122B399ED102122B3911
:1032300053D202122B39B7D202122B3970D3021299
:103240002B3910D402122B3974D402122B39BED46C
:1032500002122B39FBD402122B3963D602122B39FE
:103260006D8101122B39AF8101122B39AA84011211
:103270002B39FD8401122B39438501122B398486A9
:1032800001122B39E98601122B39298701122B39BA
:103290006C8801122B39AE8B01122B39D78C01129D
:1032A0002B39189801122B39B89801122B39AB9B86
:1032B00001122B39E29C01122B39589D01122B3936
:1032C000829E01122B39D29F01122B39B9A0011213
:1032D0002B3922A301122B3930A501122B39C1A59C
:1032E00001122B3995A601122B3921A701122B3976
:1032F0002BA701122B3953A701122B3900A8011259
:103300002B39EBA801122B39BEA901122B394BAA7C
:1033100001122B3961AA01122B39C5AA01122B39CE
:10332000EEAA01122B391BAB01122B3960AD011231
:103330002B393BAE01122B397FAE01122B39F0AE87
:1033400001122B39A9AF01122B39DBAF01122B3936
:1033500022B001122B3955B001122B39BAB001122B
:103360002B3909B101122B390EB101122B3962B17F
:1033700001122B39ACB101122B39A8B201122B3931
:103380000DB301122B396BB301122B39B5B60112F3
:103390002B3989B701122B3916B901122B39F0BB21
:1033A00001122B39A3BC01122B39CABE01122B39D1
:1033B0006FBF01122B39ADBF01122B397DC1011234
:1033C0002B3990C101122B3999C101122B39A2C19D
:1033D00001122B39B7C101122B39D6C101122B3979
:1033E0000BC401122B395EC401122B3968C40112BF
:1033F0002B3972C401122B39CDC401122B3929C5C6
:1034000001122B3941C601122B39A2C601122B39E8
:10341000F1C701122B393AC801122B3912C9011216
:103420002B393DCA01122B39F3CA01122B39F5CBC6
:1034300001122B39F7CC01122B39DCCD01122B39BB
:10344000F3CD01122B3930CE01122B393ACE0112B5
:103450002B3944CE01122B394FCE01122B396DCEB0
:1034600001122B39AFCE01122B390DCF01122B399E
:1034700032CF01122B394CCF01122B39D9CF011287
:103480002B3912D001122B3962D101122B39B9D14B
:1034900001122B39D3D201122B3909D301122B3946
:1034A000A5D301122B3921D401122B3991D5011248
:1034B0002B39ACD601122B3972D701122B391CD8FB
:1034C00001122B39A1D801122B3909D901122B393C
:1034D000BED901122B3910DA01122B3985DA01120B
:1034E0002B394EDB01122B3971DB01122B3935DC04
:1034F00001122B3959DC01122B397BDC01122B39DB
:10350000DCDC01122B3927DF01122B3902E001121A
:103510002B39ACE001122B39EDE201122B393BE3E0
:1035200001122B397EE301122B39D6E301122B391C
:1035300034E401122B395EE401122B3982E40112CA
:103540002B39B3E401122B39DDE401122B3924E5C8
:1035500001122B3982E501122B39DEE501122B39DC
:10356000DFE601122B3949E801122B3987E80112F5
:103570002B39B0E801122B3941E901122B398BE9C3
:1035800001122B39AFE901122B3905EA01122B394F
:1035900020EA01122B39DBEA01122B3905EB01126B
:1035A0002B3948EB01122B399EEB01122B39A3EE7C
:1035B00001122B39D6EE01122B3993EF01122B3960
:1035C0006EF001122B39FEF001122B393FF101127E
:1035D0002B39C2A605122B39FAA605122B391BA7C7
:1035E00005122B395DA705122B39C1A705122B39FE
:1035F000CBA705122B39DBA705122B3912A8051210
:103600002B39BBAB05122B3983AD05122B3977AFA4
:1036100005122B3915B005122B399CB005122B3928
:103620004D8004122B39F68004122B39D5810412F7
:103630002B39F08204122B39108304122B39328477
:1036400004122B39CF8504122B393C8604122B39F6
:10365000128704122B39188804122B397D88041222
:103660002B39B98804122B39128904122B394B8952
:1036700004122B39948904122B39268A04122B390F
:10368000C38A04122B39988B04122B39658C0412CF
:103690002B39F28C04122B39188D04122B39458DDD
:1036A00004122B39768D04122B394B8E04122B39D0
:1036B0005B8E04122B39AE8E04122B39BB8E041292
:1036C0002B39C88E04122B39D18E04122B39358F29
:1036D00004122B39938F04122B39DE8F04122B39ED
:1036E000F98F04122B39209004122B393D900412CB
:1036F0002B39499004122B39ED9104122B39069283
:1037000004122B39829204122B39959204122B3910
:10371000A59204122B394B9304122B39BB9404123B
:103720002B39CE9504122B396E9604122B397896CC
:1037300004122B39E69604122B39F79604122B3912
:10374000369704122B39649704122B3931980412DE
:103750002B39889804122B39CD9804122B392399D0
:1037600004122B39419904122B398F9904122B39E9
:103770005D9A04122B39AB9A04122B39ED9A04127C
:103780002B39709B04122B399A9B04122B39D09B36
:1037900004122B39DF9B04122B393D9C04122B3968
:1037A000B59C04122B39F69C04122B39459D04124A
:1037B0002B39709D04122B398A9D04122B39A49D3C
:1037C00004122B39799E04122B39839E04122B3953
:1037D000BE9E04122B39CE9E04122B39D79E0412A2
:1037E0002B39289F04122B393C9F04122B395AA0E5
:1037F00004122B396DA004122B3984A004122B392A
:1038000099A004122B3933A104122B39B2A104124E
:103810002B3955A204122B3960A204122B39ADA307
:1038200004122B39C9A304122B3921A404122B39F9
:103830008FA404122B39DBA404122B39F5A4041233
:103840002B3955A504122B39F3A504122B393EA6AA
:1038500004122B39A1A804122B3939A904122B39CF
:10386000B0A904122B39F6AB04122B390EAC04129A
:103870002B3911AC04122B391DAC04122B3931AC8D
:1038800004122B3939AC04122B3970AC04122B39C9
:1038900064AD04122B39EEAD04122B3970AE041254
:1038A0002B39E5AE04122B39BDAF04122B39DFAF33
:1038B00004122B3976B004122B3982B004122B3942
:1038C000DFB004122B39E2B004122B390FB104120D
:1038D0002B3924B104122B3993B104122B39DFB2E6
:1038E00004122B39F2B304122B397DB404122B3994
:1038F00090B504122B395AB604122B398BB6041228
:103900002B39B1B604122B39BAB604122B39E9B6E9
:1039100004122B3999B704122B3949B804122B39E8
:10392000BCB804122B396EB904122B39E1B9041258
:103930002B3920BA04122B3969BA04122B399EBADA
:1039400004122B390F8E05122B397A8E05122B3962
:10395000C18E05122B39378F05122B39878F05122F
:103960002B390B9005122B394F9205122B397A9473
:1039700005122B39579805122B39D49805122B397B
:103980000F9905122B392D9905122B398D99051296
:103990002B39B59905122B39E59905122B39169A51
:1039A00005122B39439A05122B399C9A05122B3993
:1039B000E79A05122B3900F201122B397CF2011221
:1039C0002B39A2F201122B39D9F201122B3932F420
:1039D00001122B394EF401122B3993F401122B39B9
:1039E00023F501122B397BF501122B3950F6011208
:1039F0002B392EF701122B3978F701122B39D9F711
:103A000001122B395DF801122B3986F801122B397E
:103A1000C7F801122B3975FA01122B3945FB011237
:103A20002B390CFC01122B39DFFC01122B3919FD4B
:103A300001122B3971FD01122B3993FD01122B3923
:103A400027FE01122B39DAFE01122B390BF2051277
:103A50002B3970F205122B3917F305122B394FF35E
:103A600005122B39008005122B39AB8005122B393A
:103A7000488205122B39C48205122B39FC820512AB
:103A80002B39E78505122B39798705122B39E38706
:103A900005122B391B8B05122B39BC8C05122B39C7
:103AA000B5A006122B39DDA006122B39C9A10612CA
:103AB0002B398FCF05122B3912D005122B3929D073
:103AC00005122B399CD005122B3902D105122B3946
:103AD0002BD105122B39B0D105122B3952D2051238
:103AE0002B39B5D205122B391AD305122B393AD3FB
:103AF00005122B396AD305122B3986D305122B39BF
:103B0000B5D305122B39E5D305122B391BD4051279
:103B10002B397BD405122B391E9B05122B39EE9BBA
:103B200005122B39139C05122B39339C05122B39A6
:103B3000479C05122B39AF9C05122B39D39C0512DB
:103B40002B39519E05122B39779F05122B3958A01E
:103B500005122B39BCA005122B39E8A005122B3910
:103B60006CA105122B39BDA105122B39DEA105125E
:103B70002B3956A205122B397BA205122B39DEA256
:103B800005122B396EA405122B393BA505122B39D2
:103B900072A505122B3997A505122B39B7A5051269
:103BA0002B39DDA505122B39F1A505122B395AA6A3
:103BB00005122B39AEA605122B39A0FD05122B39A3
:103BC000AAFD05122B39CBFD05122B3938E9041259
:103BD0002B3952EC04122B397FED04122B395AEF9A
:103BE00004122B39E4EF04122B3998F004122B390C
:103BF000C1F004122B39F6F004122B39A4F104128F
:103C00002B3934F204122B39A7F204122B3929F381
:103C100004122B392CF304122B392FF304122B39F5
:103C200032F304122B3952F304122B3955F30412D8
:103C30002B396EF304122B39D2F304122B39C4F44E
:103C400004122B39F9F504122B3946F604122B39DC
:103C50004DF704122B391FF804122B39BDA403129F
:103C60002B390ED702122B39CCDB02122B399EDCFA
:103C700002122B3925DD02122B3956DD02122B39A7
:103C800084DD02122B39D8DD02122B3906DE021236
:103C90002B3927DF02122B3955DF02122B3983DF34
:103CA00002122B39B9DF02122B3966E002122B39CE
:103CB0008CE002122B39EBE002122B3961E2021286
:103CC0002B39FBE202122B3980A903122B39C9E4EC
:103CD00002122B3913E502122B3962E502122B393D
:103CE000CEE502122B3936E602122B3983E6021298
:103CF0002B39F3E602122B3904E802122B39F8E8CB
:103D000002122B39A9E902122B39DEE902122B39F2
:103D100033EA02122B39D5EA02122B3903EB0212D5
:103D20002B3988EC02122B390DED02122B394DED97
:103D300002122B398CED02122B39A5ED02122B3910
:103D400054EE02122B391EEF02122B39C5EF02126C
:103D50002B3959F002122B39FFF002122B3969F17D
:103D600002122B39F4F102122B3987F202122B398D
:103D7000A5F202122B3978F302122B3936F4021213
:103D80002B39ECF402122B398AF502122B3925C992
:103D900005122B3966C905122B39CFC905122B39EB
:103DA000F0C905122B3909CA05122B39C3CA0512ED
:103DB0002B39CCCA05122B391DCB05122B3946CB1A
:103DC00005122B395DCB05122B39C1CB05122B39CE
:103DD00053CC05122B3984CC05122B39E0CC0512BB
:103DE0002B3946CD05122B397ACD05122B39EDCD65
:103DF00005122B392FCE05122B396FCE05122B3918
:103E0000A7CE05122B39B9CE05122B39CBCE051210
:103E10002B39FCCE05122B393CCF05122B3965CF3F
:103E200005122B39B7DA05122B39FADB05122B39BB
:103E300020DC05122B3931DC05122B3949DE051245
:103E40002B3968DE05122B399C9406122B39D2943B
:103E500006122B391D9506122B39699606122B393D
:103E60000CD504122B394AD604122B3986D60412EB
:103E70002B394BD804122B3975D804122B39FBDAA5
:103E800004122B393BDB04122B39D0DC04122B3902
:103E900065DD04122B39C3DD04122B3954DE041204
:103EA0002B398CDE04122B39CEDE04122B3948E07C
:103EB00004122B39D1E104122B3907E404122B39F7
:103EC00035E404122B3961E404122B396AE404123C
:103ED0002B39C0E404122B3950E504122B3957E872
:103EE00004122B39DBE804122B39AEA906122B3948
:103EF000C4A906122B39CEA906122B391EAA061206
:103F00002B398FE905122B39A8E905122B394DEA17
:103F100005122B398DEA05122B39A6EA05122B3929
:103F2000DAEA05122B3927EB05122B395BEB051268
:103F30002B399DEB05122B3973ED05122B39DEED74
:103F400005122B39FAA106122B394FA206122B3972
:103F5000A8A206122B3910A906122B3952A9061253
:103F60002B3994A906122B39A4A906122B39BDC8E6
:103F700003122B3918C903122B39B8C903122B3974
:103F8000D0CA03122B39BCCB03122B3989CC0312B4
:103F90002B399ECC03122B39E8CC03122B393FCDA1
:103FA00003122B39ABCD03122B39BECD03122B39A3
:103FB00016CE03122B3985CE03122B399DCE031258
:103FC0002B3938D103122B3934D203122B398FD22B
:103FD00003122B39D5D203122B39F3D403122B3908
:103FE00043D503122B39C4D503122B3996D60312AD
:103FF0002B39CFD603122B39EED603122B3939D7F2
:1040000003122B394FD703122B3966D703122B39E2
:1040100095D703122B39A7D703122B397DD803125A
:104020002B3988D803122B390DD903122B3965D9B6
:1040300003122B39B1D903122B39E8DA03122B39C9
:1040400019DB03122B3995DD03122B39C6DD031260
:104050002B39E1DE03122B3910DF03122B3988DFF5
:1040600003122B394AE003122B397EE003122B395D
:10407000EEE003122B39CBE103122B3904E20312D9
:104080002B390EE203122B3911E203122B391BE2FA
:1040900003122B3937E203122B39B3E203122B3907
:1040A000ECE203122B3908E303122B3934E3031239
:1040B0002B396FE303122B398AE303122B3994E374
:1040C00003122B39C3E303122B39D9E303122B3923
:1040D000F5E303122B3924E403122B3944E40312D1
:1040E0002B398DE403122B39D6E403122B39E0E58A
:1040F00003122B3933A506122B3944A506122B398E
:10410000CDA506122B39CDF804122B391CF9041257
:104110002B39DAFA04122B39ADFC04122B39EBFCE3
:1041200004122B39C1FD04122B39C6FE04122B399F
:10413000E8FE04122B3944FF04122B39C5FF041288
:104140002B39D95100122B39FB5100122B394D5309
:1041500000122B39965300122B390F5400122B39B1
:104160008A5400122B39F35400122B393A5500129D
:104170002B39A85500122B394D5600122B39D35626
:1041800000122B390F5700122B39635B00122B39A9
:10419000715D00122B39A45D00122B39E35D001212
:1041A0002B39F05E00122B39D96100122B39836252
:1041B00000122B392E6400122B39616500122B3945
:1041C000776600122B39EC6600122B39B8670012A3
:1041D0002B394F6800122B395F6800122B39166992
:1041E00000122B394C6A00122B39906C00122B39BB
:1041F000336F00122B39117000122B394E710012DF
:104200002B39937400122B39A37400122B39DA75F1
:1042100000122B398D7600122B39BE7700122B3904
:104220002C7800122B39637900122B39B8790012DF
:104230002B3906BB04122B39ADBB04122B391FBC22
:1042400004122B392FBC04122B39B1BC04122B39A8
:1042500008BD04122B39FDBD04122B3924BE0412F3
:104260002B39C9BE04122B3918BF04122B3976BF63
:1042700004122B39D1BF04122B39ACC204122B39D2
:1042800065C304122B39CAC304122B395DC504124D
:104290002B39FDC504122B3996C604122B39F3C6EF
:1042A00004122B3969C704122B3965C804122B3943
:1042B00058C904122B39B1C904122B39C7C90412C9
:1042C0002B39E8C904122B3927CA04122B39B7CA73
:1042D00004122B39FACB04122B39B7CD04122B3927
:1042E00001CF04122B393BD004122B3946D10412D2
:1042F0002B39E6D104122B3955D204122B3972D343
:1043000004122B392BE703122B3996E703122B39B2
:10431000DEE703122B3945E803122B39A1E803121B
:104320002B39DCE803122B3978E903122B39D2E957
:1043300003122B393EEB03122B39B7EB03122B3947
:10434000EEEC03122B3916ED03122B39F4ED0312A8
:104350002B3905EE03122B391BEE03122B390DEF0F
:1043600003122B3930EF03122B39F8EF03122B39DC
:1043700020F003122B3937F003122B3951F00312BE
:104380002B397DF003122B399DF003122B39C3F02A
:1043900003122B39DAF003122B39AFF103122B3948
:1043A00009F203122B39E1F203122B395DF30312E8
:1043B0002B3974F303122B39EEF303122B3936F435
:1043C00003122B395CF403122B39B9F503122B3984
:1043D000BEF503122B39FBF503122B3972F60312CB
:1043E0002B39DEF603122B39D9F703122B39B3F828
:1043F00003122B39FFF803122B3917FA03122B394A
:1044000011FB03122B39B3FB03122B39FCFB0312F4
:104410002B3911FC03122B3923FD03122B39C4FD58
:1044200003122B3922FE03122B39747A00122B3916
:10443000B17A00122B394A7B00122B39557C0012BD
:104440002B399D7E00122B39197F00122B390080E9
:1044500006122B392E8106122B39F68106122B39C2
:104460004B8206122B39CE8206122B39589906122E
:104470002B392EFF01122B393FFF01122B39DFFFA1
:1044800001122B39F5FF04122B39E57F00122B396D
:1044900026A606122B3936A606122B394EA6061270
:1044A0002B3902A706122B392FA406122B39B4A4DC
:1044B00006122B391AA506122B39C3A706122B395F
:1044C000C6A706122B39FFA706122B3952A80612CF
:1044D0002B3964A806122B3967A806122B3909F666
:1044E00005122B3917F605122B3990F605122B39C8
:1044F00065F705122B3924F905122B3989F90512B4
:104500002B39ECF905122B39F87F00122B39CC9698
:1045100006122B39049706122B39559806122B399F
:10452000D99806122B39F79106122B399892061258
:104530002B39C99206122B39149306122B39D893B2
:1045400006122B390B9406122B39319406122B3993
:10455000439406122B39579406122B396594061290
:104560002B392FD505122B395BD505122B3902D8E3
:1045700005122B3957D805122B3993D805122B3930
:10458000A7D805122B39C0D805122B39B3D905127B
:104590002B398FDA05122B39A3DA05122B39E59D59
:1045A00006122B39099E06122B39229E06122B3930
:1045B000619E06122B39949E06122B39C49E061258
:1045C0002B39CE9E06122B39369F06122B39399F76
:1045D00006122B39439F06122B39509F06122B3996
:1045E000518F06122B39798F06122B39BA8F06128A
:1045F0002B39D88F06122B39F38F06122B395B908B
:1046000006122B39679006122B39C69006122B39E9
:10461000EA9006122B39AB9106122B39B89106128B
:104620002B39C99106122B39CCAA06122B39E4AAD0
:1046300006122B390AAB06122B3900E005122B3972
:1046400049E105122B394FE105122B3966E10512BC
:104650002B3987E105122B399DE105122B39B1E188
:1046600005122B3930E205122B3995E205122B3950
:104670001DE305122B3996E305122B396FE4051261
:104680002B397FE405122B398EE405122B3977A8DC
:1046900006122B399BA806122B39C3A806122B39F8
:1046A000EBA806122B39928C06122B39FE8C0612BF
:1046B0002B391D8D06122B39838D06122B39C98992
:1046C00006122B39E28906122B39F98906122B3989
:1046D000028A06122B39208A06122B392A8A0612E0
:1046E0002B39348A06122B39478A06122B39D48A81
:1046F00006122B39438B06122B39718B06122B397C
:10470000C28B06122B390E8C06122B39298C0612FD
:104710002B39338C06122B39448C06122B39878C9B
:1047200006122B3953AB06122B399EAB06122B39CE
:104730004FF602122B397BF602122B3999F6021230
:104740002B39ACF602122B39C7F602122B3926F799
:1047500002122B3954F702122B3960FB02122B394B
:10476000A2FC02122B39D4FC02122B393FFD02129B
:104770002B39C3FE02122B39EBFE02122B3900FF3C
:1047800002122B3910FF02122B3950FF02122B3963
:1047900092FF02122B39A2FF02122B39C3FE031221
:1047A0002B39D3FE03122B39F1FE03122B390CFFE8
:1047B00003122B3933FF03122B3954FF03122B3909
:1047C0006EFF03122B39A6FF03122B39C9FF031208
:1047D0002B390FA706122B3955A706122B3900FAD1
:1047E00005122B3910FA05122B392EFB05122B3925
:1047F00060FB05122B3982FB05122B39AAFB05122F
:104800002B39C3FB05122B39FFFB05122B3968FC32
:1048100005122B39A4FC05122B39EBFC05122B39A0
:1048200018FD05122B3944FD05122B39569C061232
:104830002B398D9C06122B39B59D06122B39B89D4C
:1048400006122B391CA306122B398EA306122B3904
:10485000CCA306122B390DA406122B39C5B90512AB
:104860002B39CBB905122B3912BA05122B391EBCC4
:1048700005122B394EBC05122B39B8BC05122B3949
:1048800073BD05122B39BABD05122B39EDBD0512CA
:104890002B3977BE05122B398EBE05122B399BBEE4
:1048A00005122B39A5BE05122B3945C005122B392F
:1048B00037C105122B3995C105122B3948B10512A4
:1048C0002B395EB105122B3910B205122B393AB3D0
:1048D00005122B392FB405122B39C6B405122B390A
:1048E00001B505122B3973B505122B39D1B5051257
:1048F0002B39E1B505122B3908B605122B395AB6FA
:1049000005122B39C9B705122B39CEB705122B3931
:10491000F0B705122B394CAA06122B397AAA0612C7
:104920002B39AFAA06122B39B1AA06122B39B3AA1A
:1049300006122B39C4AA06122B39C6AA06122B3925
:10494000C9AA06122B39CD9A06122B393B9B0612A7
:104950002B395D9B06122B39959B06122B39CB9B6D
:1049600006122B39A08606122B39E38606122B3944
:10497000018706122B39348906122B3968890612F1
:104980002B39938906122B399A7F00122B39CEC10D
:1049900005122B39B1C205122B3999C305122B39D7
:1049A000AAC305122B39BBC305122B3907C4051244
:1049B0002B39F6C505122B3951C705122B3981C782
:1049C00005122B394CC805122B39A9C805122B39F1
:1049D000EBED05122B3909EE05122B394DEE0512C0
:1049E0002B3973EE05122B3995EE05122B39ADEEEE
:1049F00005122B39C5EE05122B39DDEE05122B39C8
:104A000083EF05122B39C5EF05122B39CFEF0512B5
:104A10002B39E4EF05122B39EBF005122B3906F197
:104A200005122B390FF105122B3918F105122B390C
:104A300021F105122B392BF105122B39A8F10512A2
:104A40002B39BFE405122B3904E905122B3920E973
:104A500005122B3925E905122B39608306122B39F3
:104A6000768306122B39F78406122B39218506121C
:104A70002B39688506122B39718606122B395A9FFD
:104A800006122B39CDAB06122B39D2FF02122B396D
:104A9000A9A403122B3995A403122B3981A4031264
:104AA0002B39EDA303122B3907A303122B397FA255
:104AB00003122B39CCA103122B397B9F03122B3904
:104AC000509F03122B39F19E03122B39629D031262
:104AD0002B39F09C03122B39D79C03122B399A9C4B
:104AE00003122B398C9C03122B39219C03122B3976
:104AF000E69B03122B39579B03122B39099A031299
:104B00002B398F9903122B39CC9803122B39C2976A
:104B100003122B39799703122B39539703122B3930
:104B20008F9603122B39D99403122B3907A903123C
:104B30002B39DDA803122B399FA803122B394AA861
:104B400003122B3992A703122B39D6A603122B3945
:104B50003DA503122B39799403122B394A94031281
:104B60002B39479403122B39329403122B390DA59C
:104B700003122B39EF9303122B39D69303122B39DF
:104B8000DE9203122B399D9203122B39ECE30212B1
:104B90002B396A9203122B39D1A403122B39FE91BF
:104BA00003122B39CB9103122B39709103122B393D
:104BB0003F9103122B39088E03122B391A8D0312E1
:104BC0002B39D48B03122B39808B03122B39748B26
:104BD00003122B39DB8A03122B39A98903122B39D3
:104BE000FA8603122B399D8403122B395184031248
:104BF0002B39368303122B39CB8203122B39F381E5
:104C000003122B39008003122B39AF8103122B3989
:104C10006B8003122B39328003122B39D6D6020057
:104C2000000080FB8F0001001309870001001209BA
:104C3000240002008E1025000200901026000200C1
:104C400092102700020094102800010096102900FD
:104C500001009710840004009810860001009C1049
:104C60002A0001009D102B0001009E102C00010065
:104C7000A2102D000800FA082E000100A3102F003A
:104C80000100A41030000100A51031000100A610A1
:104C90003200010002093300010003093400010061
:104CA000A71036000100040938000100A8103900DF
:104CB0000100A11083000200BA10630001000F0977
:104CC000640001009F1065000100A0106D0001004C
:104CD000100971000800F20866000100B9104300D5
:104CE0000100AA1044000200AB1045000100AD1005
:104CF00046000200AE104700080007094800010006
:104D0000B0104B000100B11004000100BC10A10064
:104D10000100BE1037000100BD1088000100140919
:104D20003C00010005093D000100A91049000200F6
:104D3000B2106700010011094D000200B4104E00CE
:104D40000100B6104F000200B7103E000100060936
:104D500000000000000000013636010100010201E0
:104D6000000103010001040106060502000007011D
:104D700000340801000F090401010D0100FF0E08B5
:104D8000000017020000190100FF1A0100011B01B9
:104D900000FE1C0100081D0200001F01000120018F
:104DA0000001210200002301000F2402000026015F
:104DB000000127010008280200FF2A0100072B013B
:104DC00002402C0100002D0100012E0100012F01E5
:104DD00000FF30010B1C310800003A0100083B01C4
:104DE000000F3C0100013D0100FF3E0400004204B1
:104DF0000000460400004A0400004E040000520473
:104E00000000560400005A0400005E20FFFF360038
:104E10000100060000000F0000000000000000007C
:104E20000000000003FFFF00000403FFFF0000FF7D
:104E3000FF0FF4010005C4040320000100000B0073
:104E40000000000000000003010F0000000000004F
:104E50000000000000000000000000000000000052
:104E60000000000000000000000000000000000042
:104E70000000000000000000000000000000000032
:104E800000000000000000000000000001037103AA
:104E900001030103010301030103220302030103D0
:104EA00010030003000300030003000300030003DA
:104EB0004203000324030603000300030403120358
:104EC0002503230325032303040304030003000332
:104ED00000034403000300032303000365032100D0
:104EE00035038103000305030003000300030003EF
:104EF00025032303030071003001600011007000DE
:104F000031022003500480001000610000001400F2
:104F1000630073007200620043000000130006008B
:104F2000000000000400120000000000000000006B
:104F300004000400370037003C0244000000000079
:104F40000000000065000000350081000000050041
:104F50000000830000000101710101010101110144
:104F600001013101010101018001100161013B00DA
:104F70001400630173017201620143010001130116
:104F800006013D013500040112010001000100018C
:104F9000000104010401330133013C0144013201E9
:104FA00036000001000165010001350081010001AA
:104FB00005018201830100010302710230016002D8
:104FC000110270020102020202028002100261025A
:104FD0003A0041006302730272026202430200025D
:104FE0001302380000020002040212020002000252
:104FF0000002000204020402370037003C024402AF
:10500000000239000002000265020002350281023E
:1050100000020502820283020002030471040204FA
:105020006004110470040204020401040204100468
:1050300061040004140463047304720462044304EE
:105040000004130406040004000404041204000411
:10505000000400040004510464000004000400047F
:105060004404000400040004000465040004350442
:1050700081046400050400048304000400007142FC
:105080001300E141010071420200634103006941E4
:1050900004006F4105007541060081413000A541C3
:1050A00031009F413200B1413300B7413500BD416D
:1050B0003400C3413600C9411100D5411400DB4121
:1050C000150093411F009941FFFF000001A5320622
:1050D000DB3208D5320BF332100F320A053302AB44
:1050E0003205C93207B1320C8D320D99326411305C
:1050F000FF000007ECFDFDFDECDCDCCCBCACAC9CA7
:105100009C8C7C7C6C6C5C5C5C4C4C3C3C2C2C1C0F
:105110001C03EAF5E5D5D5C5B5A5959585857575C5
:105120006565555545453535252515150500160F79
:1051300000000B150B020002220F3300000E0103CA
:105140000507090B0D0F00020406080A0C0D5A6929
:1051500067426565416C6C69616E636530393030FA
:1051600017181921301B1D1F303030161819202335
:105170001A1C1E3000034A49434E181A2505020026
:10518000011916181616182303000C0E020B040B37
:105190000A0708000F00393D3F373C3C362C442DB0
:1051A000020402010101010902E803000000BE043B
:1051B0000A7F003C00000000000E00E8033C0010E5
:1051C0000C0A0C03150900040009FF1E1E0305014B
:1051D0000C0504040810080328C082C08390081C32
:1051E000E4F0A3F07CD57D047A8D7B07124853123E
:1051F0003017124C0112301D026FB474F312258364
:1052000074F5122C1889098A088B0AE9705F7402F8
:105210006508703E9007AC7408F0750C00780C12AD
:105220002B5AECF50C780C122B5AEBF50C780C126F
:105230002B5A90109812298D90109CE0F97C077DD4
:10524000099010BA126FC51230417407122B8402F4
:10525000530D7401650860030253109007AC740885
:10526000F07B00AA0AA90A12308302530D7401656B
:10527000096009740265096003025310EA6006744C
:1052800003650870409007AC7402125331122DFE72
:1052900012302F9007B4E0A2E34010E9700D90089F
:1052A00020E004F06404700312533B74036508703B
:1052B0005C900821E0F8740128F0E8C39405404DA3
:1052C00012533B804874016508704574016509906C
:1052D00007AC702E740AF07401122E2DE4F07402E3
:1052E000122E2D7403F004122E2DE4F0A3F0A3F07F
:1052F000A3F07408122E2DE4F0AA18AB191232B7DD
:105300008025740A125331122DFE123065E96017A0
:105310009080F812298D7A017B009007A9E0F9129C
:105320003F177404122B84740B122B847F05022800
:1053300009F090109CE0F990109822901098E4F0F9
:10534000A374F8F0A374FFF0A37407F02274F612AC
:105350002583E9FFEAFE7AD1F9123DCD8A828B835B
:10536000E5824583702A7A027B00123DAFEA4B70DA
:105370000E7A107B009007A9E0F9123DF180148AA3
:10538000828B8374D1F0EFA3F0EEF9123DBB800362
:10539000EFA3F00255A374F712258389089007063E
:1053A000127681FF90108AE0F47003A3E0F4703667
:1053B00090071DE090108AF0A3E4F080298E828F80
:1053C00083A3A3127A6F60168E828F83A3A3A3E0B8
:1053D000F5838882A3127A6FFAA90812414B8E8254
:1053E0008F83127997FFEE4F70D390108AE0F4709C
:1053F00003A3E0F4600A90108AE0FAA90812414B76
:105400001233BF900777125B141233B90277B97465
:10541000F1122583890A8C08750900750B00740F39
:10542000122E2D12626D7411122E2D125B3B8049CB
:10543000AE0E1254DBF50CA3E0F50DAE0BEE2EFE16
:10544000E433FFEA2EF582EB126826650C7004A3A4
:10545000E0650D7019AE09EE2EFEE433FFEC2EF57B
:1054600082ED3FF583E50CF0A3E50DF00509050E8F
:10547000E50EC3950840B9050BE50BC3950A500529
:10548000750E0080EBA909026ED174F41225838990
:105490000B7D00740C122E2D12626D80010DEDC378
:1054A000950B5032750A008002050AE50AC39C502C
:1054B000ECED25E0FEE433FFEA2EF582EB3F1254DB
:1054C000EBF509AE0A1254DB65087004A3E0650928
:1054D00070D7790180027900026C78EE2EFEE433F9
:1054E000FFE82EF582E93FF583E022F583E0F50839
:1054F000A3E02274F612258312558E7003A3E06D8B
:1055000070177508B27509077808122B56EEFA1253
:1055100042777402122B84801F7508027509807807
:1055200008122B568C088D097808122B56125581BB
:1055300012429B7404122B84806974F61225831224
:10554000558E7003A3E06D70177508BF7509077855
:1055500008122B56EEFA12427D7402122B84801F21
:105560007508037509807808122B568C088D097808
:1055700008122B5612558112429B7404122B848000
:1055800022125EDCF583E0FD7C801268FA2212684C
:105590002F1279A9FCE439FD900777E06C227402A0
:1055A000122B847F0202280974F612258374FE12DE
:1055B0002C18EAFEEBFF851882851983E4F0A3120C
:1055C0005D6B126846E0FCA3E0FBECFA88828983FD
:1055D000A3A3E0F9750900750800600574FF697000
:1055E00005750882803D900777E06A7003A3E06B41
:1055F000701AAA18AB19123983E9F5098518828542
:105600001983126C83701C7508838017900912E04F
:105610006004640170057508818008E0640270030D
:10562000750880851882851983125B3BA908EEFAFC
:10563000EFFB124283E509601185188285198312F8
:105640006C836006126FBF123E5702559E74F212B1
:105650002583EAFEEBFF750A00750B001256BF1298
:1056600033BFEA65087003EB65097012123995E9DA
:1056700014F50A79017AE87B0712399B8003750BD0
:1056800080126820F50C780C122B5A750CE8750DF9
:1056900007780C122B56780A122B5A7808122B56C0
:1056A000E50BF5087808122B5A1266E1126823F907
:1056B0007A057B801242897407122B8402642912B6
:1056C00078E2126271888289831279A8F508E43938
:1056D000F5092274F6122583E9FE7F0080298A826B
:1056E0008B831254EDF8E4C8F9E50828E439F5098C
:1056F000EF25E0F8E433F9EC28F582ED125EE5EAF7
:105700002402FA50010B0FEFC39E40D20255A3743E
:10571000E812258374FB122C188A168B17851882C1
:10572000851983E4F07403122E2DE4F0A3F0041223
:105730002E2DE4F0A3F012625E3517125D3DF50BDD
:10574000850A82F5831279A4FEE439FF850A8285F1
:105750000B83A3A3E0FA850A82850B83A3A3A3E0AE
:10576000F9EAF508E439F509E50A2404F50A5002D6
:10577000050BEEFAEFFB12345BE964016016EEFAFA
:10578000EFFB12345BE9703D900777E06E7003A386
:10579000E06F6031126A3D122B5AE4F508F5097882
:1057A00008122B567808122B5A90077712299575F4
:1057B00008807808122B5A125B1A12428974071259
:1057C0002B84025B0A125B418810602B1275BE129B
:1057D0003E517403122E2D125B147403122E2D12DF
:1057E0006C8360137403122E2D125B33A9101241C7
:1057F0007B8A0A8B0B8003751000125B41880F6057
:10580000271275BE123E517401122E2D125B1474B4
:1058100001122E2D126C83600F7401122E2D125B5B
:1058200033A90F12417B8003750F00900706805D3E
:10583000850A82850B83A3A3A3A3A3A3A3A3E4F058
:10584000A3F0AA0AAB0B851482851583A3A3125B70
:1058500051127A6FF9123DBB851282851383E0C025
:10586000E0851882851983E0F874E828F582E4342D
:1058700007F583D0E0126C8704F0E511A2E0500731
:10588000AA12AB13123E57851482851583E0F514D6
:10589000A3E0F515E51445157003025A77851482C7
:1058A000851583A3A3127A6F60DD85148285158325
:1058B000A3A3A3A3A3A3A3A3E0A2E050CA85148239
:1058C000851583A3A3A3A3126C83851482851583F6
:1058D000A3A3601F127A6FFA79018514828515835C
:1058E000A3A3A3A3126EFA1227698A128B13751150
:1058F00001800F125B51A3A3E0F512A3E0F513752D
:105900001100E5124513700302587A85128285133F
:1059100083A3E065087004A3E06509600F74FF6568
:1059200008700474FF6509600302587A8512828545
:105930001383A3A3A3A3A3A3A312299585128285EE
:105940001383A3A3A3A3A3A3E0FC7405122E2D121B
:105950006FC5A91012415D7402122B84E9703C8559
:105960001282851383A3A3A3A3A3A3A3A3A3A31218
:105970002995851282851383A3A3A3A3A3A3A3A31D
:10598000A3E0FC7403122E2D126FC5A90F12415D06
:105990007402122B84E9700302587AE50F2510C3B4
:1059A00033240AFA7B00123DAF8A0A8B0BEA450BBF
:1059B00070030258588A828B8374D2F085168285D0
:1059C0001783A3A312626D8A828B83A3A3E8F0A33B
:1059D000E912789FA3E5101279B0E50FF0E51060A9
:1059E0003CEA2405FAE4350BFBE50A240AF8E43521
:1059F0000BF98A828B831262777403122E2D125B4D
:105A000056122B52AC10EC2CFCE433FD8A828B83B3
:105A1000126FC5123D8B7403122B84800D8A828B0A
:105A200083A3A3A3A3A3E4F0A3F0E50F700302589C
:105A300030A810E828F8E433F9E50A28F8E50B392E
:105A4000F9E8240AFAE439FB850A82850B83A3A3CB
:105A5000A3A3A3A3A3A3125B147401122E2D125BA4
:105A600056122B52AC0FEC2CFCE433FD123D8B7420
:105A700003122B84025842851882851983E060271F
:105A8000126A3D122B5A7508E87509077808122B1F
:105A9000567403122E2D126A46122B5A9007771253
:105AA00029957508008029EEFAEFFB12345BE97046
:105AB0002F126A3D122B5A7508E8750907780812EB
:105AC0002B567508007808122B5A900777122995E3
:105AD0007808122B5A125B1A1242897407122B840F
:105AE0007403122E2D126C83600B7403122E2D1270
:105AF0006FC5123E577401122E2D126C83600B7409
:105B000001122E2D126FC5123E577405122B847F81
:105B100010022809EAF0A3EBF022E5162402FCE4C7
:105B20003517FDE5161266713517F583E0F97A062B
:105B30007B8022125B3BAA0AAB0B22E0FCA3E0FDB8
:105B400022850A82850B83E0F8A385820A85830B70
:105B500022126EFAA322E0F50CA3E0F50D750E00FB
:105B6000780C2274F112258374F4122C188A088B95
:105B700009ECFEEDFF740B122E2D7403F0122BF2C4
:105B80001248531233B9EAFCEBFD7403122BF212E4
:105B9000484DE9600FEE241312682364036010E09F
:105BA0006401600B8518828519837484025CF58E0C
:105BB000828F83A3A3A3A3A3A3A3A3E06018F4608D
:105BC00015EE241312682364037016EE2414126871
:105BD000236003F4700B8518828519837482025C3C
:105BE000F512776DE064217002A3E06003025CCCE3
:105BF000851882851983748C125D6B6403600302BF
:105C00005CB67401122BFA126411124B83E9600323
:105C1000025CB61240DF8A0A8B0BEA450B70030266
:105C20005CF68E0C8F0D750E00780C122B527C15C5
:105C30007D00123D8B7403122B84850882850983B5
:105C4000A3A3E50A2415FCE4350BFD7409122AB25E
:105C50001273CCC0E0E50A241EF582E4350BF5830F
:105C6000D0E012627DC0E0E50A241FF582E4350B26
:105C7000F583D0E0F0E50A2420F582E4350BF583C6
:105C80007405F0EE240BFE50010FFAEFFB123A3DC3
:105C90007D007C007900EEFAEFFB1242419080F823
:105CA00012298D7A007B109007A9E0F9123F177432
:105CB00004122B848078125D33122B5A125D451228
:105CC0004BA77401122B84E9702C8014125D3312DF
:105CD0002B5A125D45124BA17401122B84E9700DF1
:105CE000851882851983E4F01240AF8009851882F7
:105CF0008519837488F01273CCF50A780A122B5A2E
:105D00007401122BEA880A890B780A122B56E508CF
:105D1000240CF582E43509125D3D4480F50B780AC8
:105D2000122B561267A31242357405122B84740C81
:105D3000026ECEEE12641EE0F50A780A22F583E0C8
:105D4000F50AA3E022EE240BFCE43FFD8E828F8354
:105D5000A3A3A3A3A3A3A3A3A31270028E828F83E2
:105D6000A3A3A3A3A3A3A3A3E0F922F01278E2E0E4
:105D700022C082C08374F3122C188518828519837F
:105D8000E4F004122E2D125B147403122E2DAA823D
:105D9000AB83122F3FAA18AB19122F75740D122B5B
:105DA00084026FB474F612258312682BFAA3E0F90B
:105DB000EAF89007BAE058F508A3E059F509E508B4
:105DC0004509601C7808122B569007771229951206
:105DD0006820FD7C001268F61242957404122B8430
:105DE0000255A374F412258374FF122C18EAFEEBFB
:105DF000FF851882851983E4F0900906E06021EEA2
:105E0000240B126823640160178E828F83A3A31270
:105E1000626DEE2415126823687003A3E0696003C5
:105E2000025ED71266D112626BE8FAE9FB888289BA
:105E300083A3A3A3A3A3A3A3A3E0FC88828983A332
:105E4000A3A3A3A3A3A3A3127949EC28F508E439DB
:105E5000F509EC45096010EC9471E994085008903C
:105E60000912E06402700A851882851983748080A3
:105E700038122FB18A0A8B0BA80AA90BE8496021B6
:105E800088828983A3A3A3A3E06016C3940350115F
:105E9000E82412125EE2E82414125EE21240AF809F
:105EA000098518828519837481F0125EDC126A44B8
:105EB000122B5A7401122BEA880889097808122BD0
:105EC0005675081F7509807808122B561266D7126E
:105ED00042357405122B847401026C75EE127794AE
:105EE0003F22F582E439F583E508F0A3E509F022C5
:105EF00074EA12258374DB122C188A148B15751220
:105F000000751300127A67F50EAC18AD197A007B94
:105F100000799C1230957A047900122F87EAF50CEB
:105F2000851882851983E02AF0F8E50EC3984003AE
:105F300002610FE0C3950EF509C39404400375098F
:105F400003E50975F01AA4FAABF0123E518A128BE0
:105F500013EA45137003026112750D00AE12AF1300
:105F6000850E08807E12617A123D97850A82850B24
:105F700083A3A3A3A3E0702D850A82850B83126CF3
:105F800083700C12710FF0EE24181271128010122F
:105F90006188F0900566E014C0E0126162D0E01202
:105FA00061B3E48034900566E004C0E0126162D021
:105FB000E01261ABC39403EE400302607612641AF0
:105FC00074021261AB64017003026083EE24151247
:105FD000618BF0EE241612618BF0EE241AFE500154
:105FE0000F050DE50DC3950940030260AEE508C33A
:105FF000950C400302608C85080AAA0A7B00122FC8
:10600000F98A0A8B0B0508900553126194124853C4
:10601000850A82850B8312626D126170E8F0A3E934
:106020001261C5850A82850B83A3A3A3A3A3A3A39F
:10603000A3A3A3E0C0E0126158D0E0F07401122ED7
:106040002DE4F0850A82850B8312626D7402122E94
:106050002D1262777401122BF2122F63E964016032
:1060600003025F657404122E2DAC82AD8312618031
:10607000124853025F6B1261891261AB64036003C3
:10608000025FCCEE2415127112025FD2E50CC395AB
:106090000E4005750800801DE50EC3950CF50880BF
:1060A00014126188F0EE241AFE50010F050DE50D63
:1060B000C39509505D740E122BFA85080AAA0A7B53
:1060C00000798712309505087418122E2D126194EC
:1060D00012485312617A123D97EE2412F8E43FF908
:1060E000740E122E2D126FC588828983EAF0A3EBFD
:1060F0001261B374031261C5741D122E2DE0C0E04D
:10610000126158D0E0126F2C709712710F80957544
:106110000900750A00780A122B5A7812122B567849
:1061200009122B5AE50EF5097809122B5A7405123B
:106130002E2DE0FD7C0012665D1242D17405122BFB
:1061400084E51245136007AA12AB13123E5774255B
:10615000122B847F0E022809EE2419F582E43FF504
:10616000832212616622EE2418F582E43FF5832231
:10617000EE2412F582E43FF583227C087D0079FF4E
:10618000EE240AFAE43FFB22EE2414F582E43FF504
:10619000837401221262718E828F83E8F0A3E9F08A
:1061A0007C677D05EE1269113FFB22127904A3A3DF
:1061B000A3E022F0EE1271067402F0EE2416F582CE
:1061C000E43FF58322F0EE2417F582E43FF5837473
:1061D00002F012616674FFF02274F612258374F9DE
:1061E000122C188A088B0912625E3509127A311254
:1061F0003DA3EAF8EBF9ECFAEDFB851882851983EB
:10620000122E16EE2404FE50010F8E828F83E0C002
:10621000E07404122E2DD0E0126F03FA7405122ED2
:106220002D7401F07406122E2D7401F0900781F088
:1062300090078A0412791BA312626D900782126282
:1062400077EA90078B12627D900780F0AA18AB194D
:10625000123035E9600312303B74070255A0EA1290
:106260006263221268402212766A39F583126271E3
:1062700022E0F8A3E0F922E8F0A3E9F022F0127896
:1062800079E02274F212258374FF122C187508002D
:106290007E007F001232E78A0A8B0B1232E78A0CEB
:1062A0008B0DA80CA90D80050508126267E84970DE
:1062B000F7900912E060076401600302638E1232F6
:1062C000E78A0C8B0DA80CA90D8003126267E849C0
:1062D000603688828983126FC5900553E06A700327
:1062E000A3E06B600D12766A39F583126FC5EA4B35
:1062F00070D98882898312626D900553E0687003BB
:10630000A3E069700302638E7A167B00123E518A05
:106310000C8B0DAE0CAF0DEE4F60739005531262F7
:106320006D8E828F83126277900548E08E828F8314
:10633000A3A3F0123443E98E828F83A3A3A3A3A364
:10634000F090109D1278F8F07C677D0512641112B0
:106350004853AA18AB1979411249D9851882851971
:1063600083E0600890077712626D800478FE79FF01
:106370008E828F83A3A3A3A3A3A3A3126277126425
:1063800019E50AF0A3E50BF08E0A8F0B05089007BC
:106390008BE0F8E508C39850047A008022E508C332
:1063A00098FAC3940640027A057900800DE50A1236
:1063B000766B350B125D3DF50B09E9C39840EE7520
:1063C00009007809122B5A780A122B56EAF5097837
:1063D00009122B5A90078BE0F5097809122B5AAD58
:1063E000087C007A827B07900780E0F91242CB7428
:1063F00005122B84900912E060046401700BEE4FCB
:106400006007EEFAEFFB123E5712303B7401025662
:10641000B9EE240BFAE43FFB22EE12641E22127640
:106420006B3FF58322EEFAEFFB7F0602280974EC3E
:1064300012258374FF122C188A0A8B0B7E008E0E95
:106440008E0F12625E350B127A6DFFAC18AD197AA1
:10645000007B00799D123095851882851983E0F8BC
:10646000EFC3984003026509E0C39FFEC3940B404D
:10647000027E0AEE75F007A4FAABF0123E518A08CC
:106480008B098A0E8B0FEA450F607C750C00801A11
:10649000850882850983A3A3A3A3A37403F0E50859
:1064A0002407F50850020509050CE50CC39E505958
:1064B000AC08AD09850C10E5102FFAE43400FB7927
:1064C0008B123095850882850983A3A3A3A3A3E03B
:1064D00014600814601314601F80B5850882850954
:1064E00083A3A3A3A3A3E480B4850882850983A31F
:1064F000A3A3A3A3740180A5850882850983A3A310
:10650000A3A3A3740280967E007508007808122B5E
:106510005A780E122B56EEF5087808122B5AEFF522
:10652000087808122B5A7405122E2DE0FD7C00E528
:106530000A126911350BFBE50A126671350BF583FA
:10654000E0F91242D77405122B84E50E450F60075F
:10655000AA0EAB0F123E577401122B847F0C022837
:106560000974EA12258374FE122C188A148B15758F
:106570000A00750B00127A67F508AC18AD197A009D
:106580007B0079A3124B9B85080C851882851983A3
:1065900012626DC3E50C98E499507D8518828519C7
:1065A00083E0C3950CFEA3E09400FFC3EE9404EFD8
:1065B000940040067E037F008004EE4F605AEEFA9E
:1065C000EFFBEA75F015A4FAA8F075F015EBA42816
:1065D000FB123E518A0C8B0D8A0A8B0BEA450B602D
:1065E00037750900750E00850E10C3E5109EE49FF7
:1065F000502BAC0CAD0D850E12850810E512251040
:10660000FAE43400FB79A2124B9BE50C2415F50C3F
:106610005002050D050E80CF75098B7E00750C00AC
:10662000780C122B5A780A122B56EEF50C780C12B5
:106630002B5A7808122B5A7405122E2DE0FDAC0946
:1066400012665D1242DD7405122B84E50A450B606B
:1066500007AA0AAB0B123E577402026150E51412EE
:1066600069113515FBE5141266713515F583E0F9EE
:1066700022240FF582E42274F612258374FF122C73
:1066800018EAFEEBFF1266D11277B1A3A3A3A3A36E
:10669000A3A3A3E0F9123059E9851882851983F084
:1066A0007508007808122B5A7401122BEA880889A1
:1066B000097808122B567508357509807808122B51
:1066C000561266D71242357405122B847401025596
:1066D000A0EE1262633F2279011266E1FAE43FFB09
:1066E00022EE2402FCE43FFDEE240F2274F4122576
:1066F0008374FA122C188A088B09EA1276711276C2
:1067000081FFEEFAEFFB122F45E960131233B9EA6D
:10671000FCEBFDEEFAEFFB12484DE96401700A74E0
:1067200001122E2DE4F0A380097401122E2DEEF03B
:10673000A3EF127937A3A3A3A3A3E0F8A2E650081E
:106740007403122E2D7401F0E8A2E75008740412AD
:106750002E2D7401F07405122E2DE4F004122BF28C
:10676000123089E9851882851983F07A007B00123E
:1067700033DD750A00780A122B5A7401122BEA884D
:106780000A890B780A122B56750A34750B80780A21
:10679000122B561267A31242357405122B8474060D
:1067A000026C757901E5082402FCE43509FDE50871
:1067B000240FFAE43509FB2274F612258374FF12C4
:1067C0002C1812682BF509A3E0F508A90912304727
:1067D000E9851882851983F0900912E0700B740125
:1067E00065087005A909124385EE240B1268237011
:1067F0002C7508007808122B5A7401122BEA8808AD
:1068000089097808122B56750836750980780812A0
:106810002B561266D71242357405122B840266CCB1
:10682000EE240EF582E43FF583E02212682F22EA7F
:10683000FEEBFF12683F3FF583E0126846E022EE70
:106840002413F582E422F8A3E0F98882898322C028
:1068500082C083900912E0700312438B026FB474FC
:10686000F412258374EF122C18EAFEEBFF1256BFC8
:10687000900777E065087004A3E065097052A818D6
:10688000A919880A890B780A122B56750A11750BFB
:1068900000780A122B567C007D007A817B00123E24
:1068A000DB7404122B84E97027750A00780A122B16
:1068B0005A7401122BEA880A890B780A122B56ACFB
:1068C00008AD091268F612428F7403122B848021DE
:1068D000750A11750B80780A122B567808122B5600
:1068E000126820FD7C841268F612429B7404122BFD
:1068F000847411026C751268FA22EE1269113FFB62
:10690000EE240FF582E43FF583E0F922FCEFFDE58C
:10691000082402FAE42274F112258374EB122C1875
:1069200012682BFCA3E0FAE4CAFBEC2AF508E43B6E
:10693000F509900777E065087004A3E06509600336
:106940000269E588828983A3A3E09410500F8882AE
:106950008983A3A3E085188285198380088518821E
:106960008519837410F0E0C0E07404122E2DD0E07D
:106970001277A2A3A3A982AA83890C8A0D750E009F
:10698000780C122B527407122E2DE0FC7D00740837
:10699000122E2DAA82AB83123D8B7403122B8474AA
:1069A00004122BEA880A890B780A122B56750A11F1
:1069B000750B00780A122B567C007D007A817B00D3
:1069C000123ED57404122B847404122E2DE090070D
:1069D000B26005E0D2E48003E0C2E4F0851882856D
:1069E0001983E480088518828519837484F0E0C0D7
:1069F000E07401122E2DD0E0F07402122E2DE50865
:106A0000F07403122E2DE508F0125EDC126A4412B7
:106A10002B5A7402122BEA880889097808122B561F
:106A20007508147509807808122B5679031266D9F7
:106A30001242357405122B847415026ECEE51612BF
:106A400077943517F583E0F50878082274F4122559
:106A50008374E0122C188A088B09AC18AD19124205
:106A600023900912E0640270337402122E2DAE825C
:106A7000AF831233B9EEFCEFFD12484DE9601D12F1
:106A800033BF8A0A8B0BA80AA90B85188285198344
:106A9000E0687003A3E0697003026C7312357574CB
:106AA00002122E2D126FBB12348BE96401700302A7
:106AB0006C737418122BF21233CB7402122E2DAC9D
:106AC00082AD837418122BF212484DE960321233F2
:106AD000C58A0A8B0BA80AA90B851882851983E041
:106AE000687003A3E06960188518828519831262B3
:106AF0006D9005491262777A497B05794B1249DF1F
:106B0000900912E0600764016003026BB112759096
:106B1000C082C0831233BF8A088B09D083D082E041
:106B200065087004A3E06509605C7402122E2DAA4A
:106B300082AB83122FB18A088B09A808A909E849FA
:106B4000602688828983A3A3A3A3E06401600D88E3
:106B5000828983A3A3A3A3E06402700C7402122EA3
:106B60002DAA82AB83122FBD9005E7126C836016AD
:106B7000900906E06401700E126FBF9005E8E0F521
:106B80008388821227691233BF8A088B09A808A953
:106B900009851882851983E0687003A3E069601194
:106BA0007402122E2D126FBB122F93E96003124054
:106BB000AF7402122E2D126FBB1235637900126F63
:106BC000BF1231D9740B122E2DE4126C87F8A3E09A
:106BD000F9740C122E2D126277740B122BF2122FF5
:106BE00063E9603F7C087D0079007418122BF21273
:106BF0003D97740E122E2DAC82AD837418122BF2B9
:106C000012484DE9601D7402122E2DAC82AD8374C2
:106C10000E122E2DAA82AB83122F3F740B122BF271
:106C2000122F757402122E2DAC82AD83740E122EAB
:106C30002DAA82AB83122F3F740B122BF2122F69F5
:106C4000E96030740C122E2D12626D851882851940
:106C500083E0687003A3E069601985188285198351
:106C600012626D740C122E2D126277740B122BF2BD
:106C7000122F757420122B847F04022809F582E4F8
:106C800038F58312714622F0851882851983E02237
:106C900074F112258374F6122C18EAFEEBFF7508C6
:106CA0000090081E126C8370507A377B00123E51A0
:106CB00090081EEAF0A3EB12747B60197C377D000C
:106CC0007900123D97EEFCEFFD90081E126FC51281
:106CD00041F3E9700B8518828519837488026E3739
:106CE000127775126ED67401F07CFF7D419004D34B
:106CF000126FC5124C07026ECCE0C8126ED6740239
:106D0000F0EEFCEFFD1273D11241F3E9700C85181F
:106D1000828519837488F0750801750AE8750B0778
:106D2000780A122B56126FD51229951277752428DE
:106D30001273C4FC12700812777524141273C4F90C
:106D40001241577404122B84126EE3126F0924311E
:106D50001273C46043127465FAE433FB123E51901F
:106D6000081EE02432126F1E6022750CE8750D07B4
:106D7000750E00780C122B52127465FCE433FD1270
:106D80006FF3123D8B7403122B84800C851882855F
:106D900019837488F0750801780A122B56126FC98E
:106DA00012299512777524111273C4FC126FEA121E
:106DB0007775242B1273C4F91241577404122B8473
:106DC0001277752434126F0924341273C46035129B
:106DD000745CFAE433FB123E5190081EE024351235
:106DE0006F1E6042750CE8750D07750E00780C1269
:106DF0002B5212745CFCE433FD126FE1123D8B7474
:106E000003122B84E508A2E04025126EE31273C43E
:106E1000700890081E12742860157B007A007900B3
:106E20001241F9026ECC8518828519837488F08529
:106E300018828519837486F07409122E2D7402123B
:106E400075D4126EF2122E2DE8F0A3E9126F03F53D
:106E5000087808122B5A7401122BEA8808890978DD
:106E600008122B567508207509807808122B567960
:106E7000017406122BFAEEFAEFFB1242357405127A
:106E80002B8412741770427409122E2D7402F012A2
:106E90006EEC122E2D127482122B5A7401122BEAF0
:106EA000880889097808122B56750820750980789A
:106EB00008122B5679017406122BFA90081E126FD5
:106EC000C51242357405122B841241ED740A122B3F
:106ED000847F07022809126EDA22242EF582E43814
:106EE000F5832290081E1273ED24312290081E12A1
:106EF0006EFAA3A3126271740122E0F8A3E0F58395
:106F00008882221275D4A3E022F582E438F5831238
:106F10006F14C822E9F090081EE0F8A3E022F8A35D
:106F2000E03400F988828983EAF0A3EB1277AB1290
:106F3000714622C082C08390081E126C836075E087
:106F4000C82435126C7D6006126FE1123E5712772D
:106F5000752432126C7D6006126FF3123E57127761
:106F6000752412126C7D6009126FC9126FC5123E32
:106F7000571277752415126C7D6006127008123E48
:106F8000571277752429126C7D6009126FD5126F24
:106F9000C5123E57127775242C126C7D6006126F55
:106FA000EA123E5790081E126FC5123E5790081EF7
:106FB000E4F0A3F0D083D082022B36AC82AD83857F
:106FC0001882851983127002221273EA2412F58244
:106FD000E438F583221273EA2429F582E438F58334
:106FE000221273EA2435126FFC221273EA242C1247
:106FF0006FFC221273EA2432126FFC22F582E4380D
:10700000F583E0FAA3E0FB221273EA2415126FFC69
:107010002274F1122583EAFEEBFF8C088D09750AB4
:10702000018C0C8D0D750E00780C122B527C177D87
:1070300000123D8B7403122B84EE2412127112F095
:10704000A3F0EE2415127112F0A3F0127590E06017
:107050003AEE2412F8E43FF9880C890D1275B91242
:107060003E511271336021E5082412127126122B51
:1070700052E508241112711A126171126FC5123D86
:107080008B7403122B848003750A00E50812759E29
:107090006035EE2415F8E43FF9880C890D1275B9B6
:1070A000123E511271336055E508241512712612F3
:1070B0002B52E508241412711A127102126FC512B4
:1070C0003D8B7403122B84E50AA2E0402BEE2412C0
:1070D000F582E43F126C816009126170126FC51273
:1070E0003E57EE2415F582E43F126C81600AEE12E1
:1070F0007102126FC5123E57A90A026ED1750A00BD
:1071000080CB127106222415F582E43FF58322EE2E
:107110002414F582E43FF583E422127765E025E04C
:10712000FCE433FDEE22127765E0F50CA3E0F50DEB
:10713000780C22850C82850D83125B14850C828568
:107140000D8312714622E0F8A3E0F9E8492274EEBB
:1071500012258374ED122C18890A8A0E8B0F750C78
:1071600000750D00750BFF7510FF7511FF75080098
:10717000750900851882851983E412747B60177481
:1071800003650A60067402650A7010E0C8243012B4
:1071900073C4650F600579000273BA7CFF7D417A84
:1071A000007B00124C077401650A700A85188285FD
:1071B00019837485803DE50A60067403650A7019B9
:1071C00090081E1273F7F07403650A7029E50E60CB
:1071D00029851882851983801A7402650A701BE557
:1071E0000E90081E70051273F780081277781274DB
:1071F0000E7402F08004E50A601E1273FD7019120D
:1072000074216005126EE6800A127428600A1277F3
:107210007524341273C414F012742160221254EDD8
:10722000F509127465F8E433F990081EE0FAA3E05A
:10723000CA2432127439241D1273DE2425802E12C2
:107240007428602E90081EE02417F508A3E034008F
:10725000F50912745CF8E433F990081EE0FAA3E033
:10726000CA243512743924061273DE240E1273C434
:10727000F50B7409122E2D7402126C8760030273D1
:1072800028E508450970030273281273FD70047E17
:107290002280027E21850882850983126EF2122ED9
:1072A0002D126277900822E0C0E01277752430F545
:1072B00082E438F583D0E0F07412122E2D7403F0BE
:1072C000AC0CAD0D740A122BF2124853850882855E
:1072D0000983A3E0F50C780C122B5A780B122B5A69
:1072E000740C122BEA880C890D780C122B5678102E
:1072F000122B56E5082406F50CE43509F50D780C3B
:10730000122B561273CCF97409122BFAEEFA7B0089
:107310001242A77408122B847CFF7D419004D31283
:107320006FC5124C070273B8126EEC122E2D127438
:1073300082122B5A7401122BEA88088909780812E4
:107340002B567508207509807808122B5679017420
:1073500006122BFA90081E126FC5124235740512E0
:107360002B84127417704E1277752419F582E43845
:10737000F583126EF4122E2DE8F0A3126F0F24186D
:10738000F582E438126A44122B5A7401122BEA88EF
:107390000889097808122B56750820750980780825
:1073A000122B5679017406122BFA1273D112423540
:1073B0007405122B841241ED79017413122B847F12
:1073C0000A022809F582E438F583E022127889E080
:1073D0002290081EE02417FAA3E03400FB22F50CEB
:1073E000A3E03400F50D1273EA2290081E1273F127
:1073F00022E0F8A3E0C82212740774012290081E4C
:10740000127407E06401221273F112740E22242F09
:10741000F582E438F583221273EA126EDAE0640230
:107420002212746B90081E2212742C221273F12403
:1074300034F582E438F583E022F582E43AF583E01E
:1074400028F8A3E039F9E824FEF582E934FFF58352
:10745000E0F510A3E0F51190081EE02290081E123E
:10746000742C25E02212746B25E02290081E127302
:10747000F12431F582E438F583E022126F15F9E842
:107480004922E8F0A3126F14F5838882A3E0F5087F
:10749000780822C082C0837B007A8579011241F985
:1074A000026FB474F41225838C088D09EA240F123C
:1074B000793D12789312626D8C828D83A3A3126240
:1074C00077EA240E12793DA3F01276781275C51270
:1074D000778750010FFCEFFDE5082406FAE4350933
:1074E000FB124853EE2408FE50010F8E828F83E07A
:1074F000C0E0127885D0E0127686F8127875E8122E
:10750000778B50010FE5082412127598A3F0E50857
:1075100024151275981275CEA30EAF83C0E01275B4
:1075200090D0E0F06028E50824121275B0123E51A8
:107530001279506019E50824121275A3127592E0B1
:10754000F912417B8A0A8B0BAE0AAF0B8007E50864
:1075500024111275988E828F83E0A3AE82AF83C010
:10756000E012765CD0E0F0601FE50824151275B0DB
:10757000123E511279506010E50824151275A312BD
:10758000759EF912417B800512765CE4F0026C78FE
:10759000E508241112776522127765E4F02212764D
:1075A00062E022127765125B3BEEFAEFFBE5082200
:1075B000F8E43509F9880A890BE01275BE2225E046
:1075C000FAE433FB22FF1278ED8C828D8322A31222
:1075D00075D4E022F08E828F832274F61225838C7C
:1075E000088D09127678FFEEFCEFFDAA08AB0912B0
:1075F0004853EE2408FE50010F8E828F8312799E2D
:10760000127686850882850983A3A3A3A3A3127794
:107610008750010F8E828F83E0F8E508127671E8BB
:1076200012777C7403687026EEFCEFFDE508240BEE
:10763000FAE43509FB1248538E828F83A3A3A3A3D8
:10764000A3A3A3A3E0C0E012765CD0E0800A127886
:107650006912775FE8F0A3E9F00255A3E508127616
:10766000622212766B3509F58322E82414F582E450
:10767000221262631277682212791512767F22F540
:1076800083E0FEA3E0221278B41278F12274F212A1
:107690002583EAFEEBFF750A00EE2410126823C36F
:1076A000940C400D1278DE127778240B1273C4F517
:1076B0000AA80AE828F8E433F9E8240DFAE439FBCB
:1076C000123E518A088B09EA450970030277561267
:1076D00066D11278CD8A828B831278B07078EEFCF6
:1076E000EFFDEA2403FAE43509FB124853EE2408BF
:1076F000FE50010F8E828F831278E98508828509FA
:107700008312778A50010F12775DE4F0E50A604634
:10771000E508240DF8E43509F98E828F83E0C0E096
:1077200012775DD0E0127870C0E012776DD0E01271
:10773000777C850A0B8E828F83E0FCA3E0FBEC88CC
:1077400082898312779A500109EE2402FE50010FBC
:10775000150BE50B70DFAA08AB09026429E50824C4
:107760000B12776522F582E43509F58322E50824BA
:107770000C1277652290081E1273ED221277802278
:107780001278BC0EAF8322A3A3A3A3F0A3E9F0EE6B
:107790002402FE22240EF582E422125B15E8240264
:1077A000F8221277A6221277ABA322F0888289836F
:1077B000221270008A828B83227F0102280974F2D0
:1077C0001225831279111254EB850882F583E0F5B6
:1077D0000DA3858208858309A3A3E0F50C1278C860
:1077E0003400FB123E518A0A8B0BAE0AAF0BEE4FF0
:1077F00060378E828F83E50DF0850882850983E0EE
:10780000FA127924850882850983A3A3A3A982AAF1
:107810008389088A09880A7808122B521278C33F94
:10782000FB123D8B7403122B8402642574F712251E
:1078300083EA2413F8E43BF988828983E0FAA3E021
:10784000F5838A82127943127864126846A3E0FABB
:1078500088828983A3A3E0F9EA8C828D83A31262D4
:10786000780277B91277ABE0221278F1F8E50822B6
:10787000127780E02212787922E508240FF582E45D
:107880003509F5832212788922E5081277943509A3
:10789000F58322127898A322F08A828B83A3221286
:1078A00078A322F08A828B83A3A3A322A3A3A3A3FA
:1078B0001278B4221278BCAE82AF8322F08E828F0F
:1078C00083A322AC0C7D00EE2404FAE4221278D1CA
:1078D00022F583E0FEA3E0FF8E828F83E022127800
:1078E000E22212683F3FF583221278F1228E828FC6
:1078F00083E0FAA3E0F9EA22E08E828F83A3A3A3B8
:10790000A3A3A322F0850A82850B83A3228C088D72
:107910000912791522EA1268403B22F08508828517
:107920000983A322127949EA8E828F83A3F0A3E907
:10793000127937E50CF0221278BCA3A322F582E479
:107940003BF583E08C828D8322A3E0F8E4C8F92222
:10795000850A82850B83125B14850A82850B83124C
:1079600071462274F612258312790DF583127997E8
:107970001275C512778B50010F12690C3509FB1275
:1079800048538E828F83A3A3A3A3A3A3A3A3127997
:107990009EA3A3F00255A3126271E8FEE922127AB7
:1079A00044A3A3221279A822E0FA127949EA2822F4
:1079B0001278A3A3A3A3A32274F612258312790D30
:1079C000127A31123DA3EAF8EBF9ECFAEDFB8508E7
:1079D00082850983122E16EE2404FE50010F8E823A
:1079E0008F83E08508828509831278ACC3940650A2
:1079F00005127A498037850882850983A3A3A3A34A
:107A0000E064FE600E850882850983A3A3A3A3E03A
:107A1000F4701B127A3C12777C850882850983A357
:107A2000A3A3A3E0F47007127A56F0A3E9F002557D
:107A3000A312767FFF7904EEFAEFFB228E828F830A
:107A4000127A4422127A49A322E0850882850983AA
:107A5000A3A3A3A3A3221278ED850882850983A39B
:107A6000A3A3A3A3A3A322EA1262633515F583128D
:107A70006EFAE02274F61225837E00790012442DFE
:107A800075089E7509087808122B567C547D007A7B
:107A9000507B00123EC97402122B84E9F8740A6804
:107AA000600BE8700912443FE9640A70010E027C21
:107AB0004E74F212258374FE122C18E9FE7C547D5C
:107AC0000079007A9E7B08123D97123F3B8A088B13
:107AD000098C0A8D0B90089E7808122DC7EE60580D
:107AE000851882851983E4F0A3F0A818A919880CD9
:107AF000890D780C122B56750C02750D00780C123E
:107B00002B567C007D007A027B00123ED574041255
:107B10002B84750C9E750D08780C122B56750C5421
:107B2000750D00780C122B567C007D007A507B007E
:107B3000123ED57404122B84AA08AB09AC0AAD0B13
:107B40007402122B847F0602280974F61225838A98
:107B5000088B0978081227BD000019000000C27BBD
:107B60000200CD7BC800D27BC900D77BCA00DC7B7A
:107B7000CB00E17BCC00E67BCD00EB7BCE00F07B45
:107B8000CF00F57BD000FA7BD100FF7BD200047CD4
:107B9000D300097C2C010E7C2D01137C2E01187C56
:107BA0002F011D7C3001227C3101277C32012C7C8D
:107BB0003301317C3401367C35013B7C3601407C1D
:107BC0004C7C123F3B90089E122DF2807F9008A2C1
:107BD00080719008C4806C9008C680679008C88047
:107BE000629008CA805D9008CC80589008CE80537F
:107BF0009008D0804E9008D280499008D48044905C
:107C000008D6803F9008D8803A9008DA80359008EE
:107C1000DC80309008DE802B9008E080269008E21F
:107C200080219008E4801C9008E680179008E88086
:107C3000129008EA800D9008EC80089008EE80030E
:107C40009008F0E02401F0A3E03400F08002EEF9A7
:107C50007F0202280974F612258374FC122C188501
:107C60001882851983E4F0A3F0A3F0A3F08A088BAF
:107C70000978081227BD000022000000047D0100E1
:107C8000137D02003E7D6400447D65005C7D6600DE
:107C9000747D67008B7D6800A27D6900B97D6A00F4
:107CA000D07D6B00E77DC800027EC900077ECA0058
:107CB0000C7ECB00117ECC00167ECD001B7ECE004C
:107CC000207ECF00257ED0002A7ED1002F7ED200DC
:107CD000347ED300397E2C013E7E2D01437E2E0161
:107CE000487E2F014D7E3001527E3101577E320198
:107CF0005C7E3301617E3401667E35016B7E360128
:107D0000707E8C7E90089E122E0A851882851983BB
:107D1000027DFCA818A919880889097808122B5631
:107D20007508027509007808122B567C007D007AD0
:107D3000027B00123EDB7404122B84027E8C9008BE
:107D4000A2027E73AA18AB1979E71249D985188265
:107D5000851983122E0A9008A4027DFCAA18AB197B
:107D600079E81249D9851882851983122E0A90085C
:107D7000A8027DFCAA18AB1979E91249D9851882A5
:107D8000851983122E0A9008AC8071AA18AB197954
:107D9000EA1249D9851882851983122E0A9008B0F3
:107DA000805AAA18AB1979EB1249D985188285191E
:107DB00083122E0A9008B48043AA18AB1979EC12EA
:107DC00049D9851882851983122E0A9008B8802C0B
:107DD000AA18AB1979ED1249D98518828519831231
:107DE0002E0A9008BC8015AA18AB1979EE1249D951
:107DF000851882851983122E0A9008C0122E160249
:107E00007E8C9008C4806C9008C680679008C880FB
:107E1000629008CA805D9008CC80589008CE80534C
:107E20009008D0804E9008D280499008D480449029
:107E300008D6803F9008D8803A9008DA80359008BC
:107E4000DC80309008DE802B9008E080269008E2ED
:107E500080219008E4801C9008E680179008E88054
:107E6000129008EA800D9008EC80089008EE8003DC
:107E70009008F0E0F8A3E0F9E8FCE9FD85188285B8
:107E80001983ECF0A3EDF0A3E4F0A3F0851882854C
:107E90001983122DFE7404122B84027C5074F61286
:107EA00025837E0175089E7509087808122B567582
:107EB00008547509007808122B567C007D007A5012
:107EC0007B00123EDB7404122B84E970497AA47B98
:107ED0000879E71249DF7AA87B0879E81249DF7A46
:107EE000AC7B0879E91249DF7AB07B0879EA12495C
:107EF000DF7AB47B0879EB1249DF7AB87B0879EC3A
:107F00001249DF7ABC7B0879ED1249DF7AC07B0821
:107F100079EE1249DF1E027C4E74F21225837A64D8
:107F20007B001244397A657B001244397A667B0003
:107F30001244397A677B001244397A687B00124414
:107F4000397A697B001244397A6A7B001244397AA3
:107F50006B7B00124439123F3B8A088B098C0A8DD7
:107F60000B90089E7808122DC7750C9E750D087829
:107F70000C122B56750C54750D00780C122B567C78
:107F8000007D007A507B00123ED57404122B84AA27
:107F900008AB09AC0AAD0B027B4574F6122583755C
:107FA0002900752A00752B008A2C8B2DEA90620B14
:107FB000F08A088B0974047808122DB8E5089062DD
:107FC00007F08A088B0974097808122DB8E508545F
:107FD0003E906209F0758B00C2E843AC20439A02E0
:107FE0007F020228097409F5D575D4167409F5D3F2
:107FF00075D21E022B36FFFF851A87C2AF022B36C1
:10800000240354004900200043004300320035009F
:10801000330031002000550053004200200043008F
:10802000440043002403540065007800610073009D
:10803000200049006E0073007400720075006D002E
:1080400065006E00740073005D4A153863320D4C94
:10805000672E773F0941BF48A148994400000000BE
:108060000000000000000000000000000000000010
:108070000000000000000000000000000000000000
:108080000030313233343536373839414243444594
:10809000460000000000000000000000000000009A
:1080A0000000FFFFFFFFFFFFFFFFFFFFFFFFFFFFDE
:1080B000FFFF0008000400020001FFFFFFFFFFFFB9
:1080C000FFFF02050200080174000000000000002C
:1080D000000000000082003A003B0002000206029D
:1080E000E71F0300805101003C000000100E00005B
:1080F00019E0FCFF04000000E80300000943388693
:1081000064000000E204000058020000BC0200000D
:10811000F8FF000000F8FF0760EA00000000000020
:10812000300000000B000000010000000200000011
:1081300097511800FEFFFFFF1F000000080000001D
:108140006AAEE7FF965118009F020000E9FFFFFFAB
:108150000000FF0032000000000000FFFA000000F5
:108160000403090400000000000000000A74F71274
:108170002583E99005A0F0900555E4F01248299078
:1081800005B4E4F0A3F09005A1F0A3F012351B9024
:108190000912E0600464017006122F81123143124B
:1081A000482F900516E4F0A3F0124A1B02B1A77401
:1081B000F0122583EAFEEBFF548060689005A0E092
:1081C000F9123DC78A088B09EA4509604F7C008097
:1081D000010CEC75F003A4F8A9F074CC28F58274B6
:1081E0005039F583E493F4602CE493F88508828B8E
:1081F00083E06870DCAA08EC75F003A4F874CD285D
:10820000F582745039F583E493C0E0740193F583EB
:10821000D082122769AA08AB09123DB5EEFAEF64C5
:10822000800284A0EF5420601E12337D8A088B09DF
:10823000EA4509600A123299AA08AB09123DB5EE67
:10824000FAEF64200284A0900912E064027024EE28
:10825000A2E0501F90055AE0640F701179001232AD
:1082600069E9600990108E12D38B123281EE64019D
:108270000283A6EE54207003028377750C007A20E7
:108280007B009005A0E0F9123F29EA4B4C4D701796
:1082900090812C12298D7A207B009005A0E0F912A4
:1082A0003F1D7404122B847C0079047A007B001239
:1082B00033478A088B098018850882850983A3A320
:1082C000A3A3A3A3A3A3A37401F0850A08850B09A4
:1082D000E508450960777C007904AA08AB091233E8
:1082E000478A0A8B0B750C01E5082404F8E435096C
:1082F000F98882898312EF7C12EAD170CD850882D9
:10830000850983A3A3A3A3A3A3A3A3A3A3E06401B9
:1083100070A6850882850983A3A3A3A3A3A3E05421
:10832000047095850882850983A3A3A3A3A3A3A3AF
:10833000A3A37406128BA2700374B7F0E0FA850849
:108340008285098312867E12327B0282CA1233171B
:108350007C0079017A007B001233478B09EA4509DA
:108360007010E50C700C7A207B009005A0E0F912EB
:108370003F23EE6420802FE06007640160030284E5
:1083800076EE5410600812317FEE64108018EE54BF
:108390004060081231F7EE6440800BEE5480600BB1
:1083A00012304DEE6480FAEF0284A0EF54016016A3
:1083B0009005D312CBD1600612C63B122769EEFAA4
:1083C000EF64010284A0EF5408604712314F900916
:1083D00002E064017034900903E0602EF508E4F5D2
:1083E00009F50AF50B9080F8780C122DD6780879EB
:1083F0000C12241E7808122B4E7A007B089005A0E0
:10840000E0F9123F1D7404122B84EEFAEF640802A7
:1084100084A0EF541060129005B2E06005E4F01201
:10842000314FEEFAEF64108077EF544060489005CA
:10843000DD12CBD160399005E312CBD160319009C8
:1084400006E0640170299005DD12C6381227699094
:1084500005E312C63812276990811812298D7A0017
:108460007B409005A0E0F9123F1D7404122B84EEAE
:10847000FAEF6440802AEF5402600A1234E5EEFA03
:10848000EF6402801BEF5404601912CADB12C8EDBE
:10849000790190055312D38B1230CBEEFAEF6404BE
:1084A000FB80047A007B0002C178C082C08374EA3A
:1084B000122C187C167D007900AA18AB19123D9772
:1084C0007408122E2D7402F09005491297C8128478
:1084D000E97409122E2D12C8ED7413122E2DE41218
:1084E000CA37124A097416800EE8F0A3E9F0900525
:1084F0005312D14C227408122B8402C1B074F712AB
:10850000258374DF122C18EAFEEBFFEE4F602DACD2
:1085100018AD191233A17406122E2DE0601E7417C7
:10852000122E2DE0FD7401122E2DE0FCEEFAEFFB71
:108530007900122EFDE9600479A48002790074218B
:1085400002B1A474F4122583EAFEEBFF8E828F83BE
:10855000A3A3A3A3A3A3E054406016128B961234E6
:108560005BE960077AFF7BFF02864512C63402860C
:1085700038900912E060076401600302861E9005CE
:1085800040E0A2E1400302861E8E828F831286782D
:1085900012C9FDA3A3A3A3E0FA88828983A3A3122F
:1085A000D55E8E828F83A3A3A3A3A3A3A3E05410BD
:1085B0006004794080027900750AFE750BFF780A25
:1085C000122B5612B66C122995AC08AD09128B9677
:1085D0001231557404122B84E5086A7003E5096BA7
:1085E000600B12B6716A7003A3E06B704E750A00DF
:1085F000780A122B5A79028E828F8312B25CAA08F3
:10860000AB0912349D7401122B847508CDAA088E13
:10861000828F8312867E12327BE9604C80579009EC
:1086200012E06402600FE06004640170DD900540B8
:10863000E0A2E140D590054912D38B74FE6A700325
:1086400074FF6B60C512C63412DA7F12345BE98E98
:10865000828F83600512AA92800312AAA712AAB081
:10866000124A0FE9F50870A5EE4F60097901EEFA9C
:10867000EFFB12332302BF45E0F812B29E2212EE46
:1086800047E0F92274F6122583E9FEEAFF7A0F7BB0
:1086900000123DAFEA4B601F8A828B83740CF0EEB0
:1086A000A3A3F0EF8A828B8312AEE59005A0E0F9D8
:1086B000123DBB7900802FEEF912334D8A088B09E9
:1086C000A808A909E849601C88828983A3A3A3A3F9
:1086D000A3A3A3A3A3740612E6C1E0F9123209EE24
:1086E000F9123329791002C52474F41225839005F8
:1086F0005AE0640F7030EA4B602C900555E0640836
:108700006005E06404701F8A088B09E4F50AF50B24
:108710007808122B4E7A017B009005A0E0F9123FF9
:10872000177404122B840298B374F2122583EAFEA4
:10873000EBFF8C088D09890A740E122E2D1297E218
:10874000850C82F583E4F0A312C8F3E0F912343704
:10875000E9602612D37E12345BE96402701B8E82BC
:108760008F83A3A3A3A3A3A3A3A3A312B904850CDC
:1087700082850D8312C8ED8003750A0012B096142D
:10878000602514603A14605B14606314603F1460E9
:108790007D24FE700302882814700302883C147044
:1087A0000302884F02885D780C122B56AC08AD0985
:1087B000EEFAEFFB1231677402122B84028858AC78
:1087C00008AD09EEFAEFFB12316D02886712D37E15
:1087D00012345BE9600302885DEEFAEFFB1231BBF5
:1087E000028867A90AEEFAEFFB1234A3806A12BB73
:1087F000AC64027068E50A700A12DB387003A3E00B
:10880000697064EEFAEFFBA90A12342B804A12DB7E
:10881000387003A3E069704512BBAC6402703EEE91
:10882000FAEFFB123413803F9005D512CBD160379D
:10883000EEFAEFFB12C63B122769802B12DB387071
:1088400003A3E0697017EEFAEFFB1234AF8018EE65
:10885000FAEFFBA90A1234BBE9F50A800A750A008F
:108860007AD37B00124433A90A02D15D74F4122535
:108870008374DB122C188A088B098A828B83A3A34A
:10888000E0F912334D8A0A8B0BAE0AAF0BEE4F7034
:108890000302899D850882850983A3A882A983E0B4
:1088A000C0E012C8BBD0E012E6D864F1603385089E
:1088B00082850983A3E064CD6027850882850983CA
:1088C000A3E0641A601B850882850983A3E064E93C
:1088D000600F850882850983A3E064E16003028A52
:1088E00087900912E06007640160030289B68E82F6
:1088F0008F83A3A3A3A3A3A3A3E0540870030289B7
:10890000B68E828F83A3A3A3A3A3A3A3A3A374055B
:10891000F0900912E06004640170538508828509B3
:1089200083A3E064E960479005D912CBD1600612B9
:10893000C63B1227699005DB12CBD1603190054010
:10894000E0A2E1502912CDA9A3A3A312B0AC888262
:10895000898312D38B12354BEA4B601285088285CE
:108960000983A3E0F99005DB12C6381227698E82CD
:108970008F83A3A3A3A3A3A3A3A3A3E06402701064
:108980008E828F83A3A3A3A3A3A3A3A3A37406F0A0
:10899000850882850983A3A3E0F9123329123317CE
:1089A000900912E06402700990109212D38B123277
:1089B0008174250298B07900123323E97003028A8A
:1089C00087900912E0600764016003028A5C9005E9
:1089D00040E0A2E14003028A5C12CBCC607E8E8232
:1089E0008F8312D38B7404122BFA12CDC61233A1CB
:1089F000850882850983A3E064E97020128B8512C3
:108A00002B5A850882850983A3E0F50A780A122B80
:108A10005A12D56F1233D77402122B84740D122E92
:108A20002D12CBC212E9FD12C8ED7409122E2DE0F1
:108A30006004794080027900740F122E2D12B0ACC0
:108A4000740D122E2D12D38B123161E9600E8E82BD
:108A50008F83A3A3A3A3A3A3E04420F0EE2404F5F3
:108A60000AE43FF50B8E828F8312AD3EE0F9850A52
:108A700082850B8312D38B12483B850A82850B8338
:108A8000EAF0A3EB028910850882850983A3E0C080
:108A9000E07402122E2DD0E012A524EEF0A3EF1206
:108AA0008BA2C0E07403122E2DD0E012E2D2E0AA15
:108AB00018AB19702E1230A7900912E060046401FF
:108AC00070247402122E2DE0701C128B9612345BEF
:108AD000E970369005D912CBD1602E12C63B122711
:108AE0006980031234317402122E2DE064E970198A
:108AF000128B85122B5A750AE9780A122B5A12D555
:108B00006F1233D77402122B84900912E06007644D
:108B100001600302896E900540E0A2E140030289F2
:108B20006E8E828F83A3A3A3A3A3A3A3A3A3E064B6
:108B30000270398E828F83A3A3A3A3A3A3E054045E
:108B4000602A128B9612345BE98E828F83700F122B
:108B5000C63874FFF0A312AD59740502898FA3A320
:108B6000A3A3A3A3A3A3A3740302898F850882856B
:108B70000983A3E064E9600302896EEEFAEFFB1259
:108B800034C102896E8E828F8312D14CE8FAE9FBE0
:108B9000750A01780A228E828F8312B277FAA3E0D7
:108BA000FB22F0E50812EE3D3509F583E02274F46E
:108BB000122583EAFEEBFF7508007509008E828F8F
:108BC00083A3A3A3A3A3E0603B75080812D37E7917
:108BD000FF122E738B0BEA450B601075082C8E82EA
:108BE0008F83A3A3A3A3A3E0D2E0F08E828F83A3FD
:108BF000A3A3A3A3E0540364016003028CB8430859
:108C000011028CB8EE241812BBAF6049EE241A1280
:108C1000BBAF6003F4701D12DB387003A3E0697012
:108C200006750822028CB8900555E06404600302C2
:108C30008CB8801CEE241BF582E43F12B694241AF3
:108C400012BBAFFAEE24191298881231CDE9706880
:108C5000750901806312D37E12345BE964027003EC
:108C600075080112DB387003A3E0697006E508D2CD
:108C7000E1F508E50860158E828F83A3A3E07006F6
:108C8000E508D2E58004E508D2E6F50812D37E12A5
:108C9000345BE964017006E508D2E0F5088E828F46
:108CA00083A3A3E0601212B096F9123437E964018D
:108CB0006006E508C2E0F508900912E0600464016E
:108CC0007012E508A2E1400CE509A2E04006E508C3
:108CD000D2E7F50802BF4574EC12258374CD122C3F
:108CE00018EAFEEBFF851882851983129BA4751084
:108CF00000751100750900900912E06402701C8E65
:108D0000828F83A3A3A3A3E0601190109012CBD114
:108D1000600990109012D38B1232817405122BFAD5
:108D20008E828F83A3A3A312CBC412D3891233A143
:108D3000E97003028E5A79017407122E2DE0C39454
:108D4000024001197409122E2DE0C39402400279E9
:108D500000740E122E2DE064F87003A3E0F470038B
:108D6000028E5A740E122E2DE064F97003A3E0F403
:108D70007003028E5A740E122E2DE064FA7003A353
:108D8000E0F47003028E5A740E122E2DE064FB7014
:108D900003A3E0F47003028E5A7408122E2DE0F83B
:108DA000900543E0686003028E5AE9A2E0400302A6
:108DB0008E5A12B8FB7424122E2D12CA26241C12AD
:108DC000B8FE7412122E2D12C8ED740B122E2DE067
:108DD000601D741C122E2DE0FD7406122E2DE0FC79
:108DE0008E828F8312D3897901122EFDE9703D7432
:108DF00005122BF2123293E9F508740B122E2DE0B6
:108E0000702E90053DE06028742255086422602091
:108E100074425508644270147422122E2D12979FCA
:108E2000600E7422122E2D1297A560047ACF802C2A
:108E3000E9A2E6506E900912E0600464017025908A
:108E40000540E0A2E1501D7422122E2D12B09F1297
:108E50002A1A01010A7B8E005A8E7AD37B001244B3
:108E6000330297837422122E2D12B09F24FD600BC3
:108E700014600824FD600424FD70DF7422122E2D7E
:108E80001297EA700E7422122E2D12C63AA3E064D5
:108E90000D60107405122BF2123497E9640170030F
:108EA000029783EE242DF582E43FF583129E7C70B9
:108EB00003A3E069701E750A00780A122B5A780A1B
:108EC000122B5AEE242F1298881297B61233D774A9
:108ED00002122B84740B122E2DE07003028F81126C
:108EE00097B612354B8A0A8B0BEA450B700302903A
:108EF0002A7406122E2DE0F88E828F83A3A3E02819
:108F0000F8A3E03400F9E8240D12978DF88A828BDB
:108F100083A3A3A3E068600FE88A828B83A3A3A343
:108F200012DC1C1297F0F079047406122E2D12A395
:108F300013E02AF8A3E034008882F583A3AA82AB69
:108F400083123DA38A0C8B0D8C0E8D0F850A8285B2
:108F50000B83A3A3A3A3780C122B114003029783C6
:108F6000908128780C122CBF850A82850B83A3A3DD
:108F7000A3A3E50CF0A3E50DF0A3E50EF0A3E50F28
:108F8000F0900912E064026015E06007640160037C
:108F90000290C4900540E0A2E150030290BE90050B
:108FA00055E064046008E064096003029783E50803
:108FB000A2E54003029065EE242F12BBAFC0E0741F
:108FC00002122E2DD0E0129810C0E07403122E2D44
:108FD000D0E0129808C0E07404122E2DD0E0F07496
:108FE00016122E2DE0640170267410122E2D129789
:108FF000AB7003A3E0697017740E122E2D12D38B81
:1090000012345BE9640270077416122E2DE4F0121C
:1090100097FE12298D7406122BFA7409122BF21284
:1090200030AD7404122B8402978390059AE064019A
:109030006003028F817422122E2D12979F7009E512
:1090400008A2E65003028F817412122E2DE0F470F4
:1090500003A3E0F4600CEEFCEFFD7405122BF2129A
:10906000329F029783A2E650527422122E2D12CD07
:10907000C07016741C122E2DE06402703E7405122E
:109080002BF2790012342B80327422122E2D12977B
:10909000A57014741C122E2DE06404701E74051249
:1090A0002BF212341F80147422122E2D1297EA70A4
:1090B0000A79007405122BF21234A30297839009E7
:1090C00012E06013E064016003029783900540E0C2
:1090D000A2E140030297837416122E2DE0601CEE6D
:1090E000240212B65B129D451412AEDB129D45C0E0
:1090F000E07416122E2DD0E0F07006E508C2E7F5F8
:1091000008E508A2E35061751110A2E25018740A34
:10911000122E2DE054E3F0740A122E2DE0131313D7
:10912000541FF8E0802CA2E4502A740A122E2DE07D
:109130001313543F5407F86009740768600B18E86C
:109140007007C3E508C2E7F508E8333354FCF8E0DC
:1091500054E348F0740A122E2DE0C0E08E828F8313
:10916000A3A312AE2BD0E0F0900555E06404600894
:10917000E064096003029244740E122E2D12DB4546
:109180007003A3E069601F740E122E2D12D38B1290
:10919000345BE96402600F740A122E2DE0540364FC
:1091A0000160030297837407122E2DE07041EE24B4
:1091B0002F12BBAFC0E07402122E2DD0E012981017
:1091C000C0E07403122E2DD0E0129808C0E07404A1
:1091D000122E2DD0E01297F912298D7406122BFA57
:1091E0007409122BF21230AD7404122B8480527465
:1091F00022122E2D12CDC07016741C122E2DE0647A
:1092000002703E7405122BF2790012342B803274F6
:1092100022122E2D1297A57014741C122E2DE064AC
:1092200004701E7405122BF212341F801474221263
:109230002E2D1297EA700A79007405122BF212345F
:10924000A302978374615508700302934BE508A24B
:10925000E0506D12B0A37405122BF21231FDE970CB
:109260005C1233D1E9F5097416122E2DE0700F74DB
:1092700010122E2D1297AB7003A3E0696042A9096A
:1092800012B0A37405122BF2123203E96024E50830
:10929000A2E3500C85188285198374FFF0A3800C1B
:1092A000740E122E2D1297C8E8F0A3E9F075100481
:1092B000800EE508C2E5F508750900800353089F94
:1092C000E508A2E5503FEE242F12BBAFC0E07402C8
:1092D000122E2DD0E0129810C0E07403122E2DD063
:1092E000E0129808C0E07404122E2DD0E01297F915
:1092F00012298D7406122BFA7409122BF21230AD5A
:109300007404122B84E508A2E6400302961EA818F6
:10931000A919880A890B780A122B56A9091297965F
:10932000122BF21232877402122B84E9F5097003B2
:1093300002961E7422122E2D12B09F640160030249
:10934000961E74104510F51002961E7407122E2DED
:10935000E06401705D7422122E2D12B09F640570BE
:109360001EA818A919880889097808122B5612977F
:1093700094122BF21232877402122B840297837498
:1093800022122E2D1297EA7029740E122E2D12D34E
:109390008B122F9FE9601BA818A919880A890B78DE
:1093A0000A122B56129794122BF212328774021261
:1093B0002B847416122E2DE070257407122E2DE0CA
:1093C0006401700C7422122E2DE0F81297EA600CE2
:1093D000EEFCEFFD7405122BF212329F02978312FE
:1093E000331DE96003029783741D122E2DE0700374
:1093F0000294997420122E2D12B0AC741F122E2DCF
:10940000E0FA741E122E2DE0F91231CDE9607D7460
:109410001F122E2DE0701E740E122E2D1297C812E0
:10942000BC92FAA3E0FB122FAB8B0BEA450B600357
:1094300002961880517420122E2D12D38B741F1295
:109440002E2DE0F91231C785188285198312DA7F33
:109450007808740D122E2DE060027810740C122E14
:109460002DE06004740828F8740A122E2DE06001C3
:1094700008088E828F83A3A3E028FAA3E034008A31
:1094800082F583E014F07510400296187508007894
:1094900008122B5A790B0295D1740E122E2D12C878
:1094A000E97409122E2DE060030295ECE508A2E3B1
:1094B00050030295EC7407122E2DE06401607A7956
:1094C0000085188285198312D38B1232218A0A8B68
:1094D0000BA80AA90BE849601C88828983A3A3A36F
:1094E000A3A3E06401605288828983A3A3A3A3A3FA
:1094F000E064026044EE242D12B0A685188285191E
:109500008312D38B12354B8A828B83E5824583602D
:109510000FA3A3E0F9123569E96005C39408401967
:109520007410122E2D12D38B122F9FE97003029507
:10953000C77409122E2D7404F0E4F5097809122B72
:109540005A741E122E2DAC82AD83740F122E2D1262
:10955000D38B740A122E2DE0F91232337401122BC0
:1095600084E9600F7510208E828F83A3A312B09FB1
:10957000543FF0741D122E2DE06023740E122E2D18
:1095800012B0AC741E122E2DAA82AB8312339B85AF
:10959000188285198312DA7F74404510F51074071C
:1095A000122E2DE06401601579007410122E2D1218
:1095B000B0AC740E122E2D12D38B1231D3E508A24B
:1095C000E35037794080357508007808122B5A79B6
:1095D00002740F122E2D12B0AC7411122E2D12D354
:1095E0008B12349D7401122B84029783E508A2E349
:1095F0004003029539744002953A79007410122E96
:109600002D12B0AC740E122E2D12D38B123161E9D3
:10961000600674204510F5101233D1E9F50985185C
:1096200082851983E064FE7003A3E0F4700375097A
:1096300000900905E0640160030296D1EE24131244
:10964000BBAFF47003A3E0F470030296D1740E1262
:109650002E2DC3E094F9A3E094FF507512B8FB746B
:1096600010122E2DE0687003A3E06960647410127C
:109670002E2D12D38B122FAB8A0A8B0BA80AA90BA3
:10968000E849604D88828983A3A3A3A3E0640160B5
:109690000D88828983A3A3A3A3E064027033742698
:1096A000122E2D740112DFF5F8A3E0F97431122E99
:1096B0002D12C8ED7426122BF2122F6FE96012746E
:1096C00029122E2DAA82AB83122FBDE9600312400E
:1096D000AFE508A2E74003029783E509700302970C
:1096E000838E828F83A3A3A3A3E0FA7B00123E5153
:1096F0008A0A8B0BEA450B7003029783EE2404F56C
:1097000012E43FF5138E828F83A31297D8122B5247
:10971000851282851383E0FC7D00123D8B74031259
:109720002B847407122E2DE0C0E07402122E2DD06F
:10973000E0F07403122E2DE4F0A3F07402122BEA71
:10974000880C890D780C122B567810122B56E509CF
:10975000F5087808122B5A12CACD12299585128263
:10976000851383E0F97407122E2D12B0ACAA0AAB50
:109770000B12338F7407122B84E96007AA0AAB0B14
:10978000123E577433122B847F0C022809F582E4B1
:1097900012E82222790012CAD112B0B07407221244
:1097A000B27764062212B27D64072212D14CEE24F5
:1097B0001312B6786822EE242BF582E43FF583126B
:1097C000B69A24131298A322E01297CD22F8A3E0B0
:1097D000F985188285198322A31297E2750E007805
:1097E0000C22E0F50CA3E0F50D2212B27D640322F9
:1097F000A3E4F0A3F0A3F0A322F01297FE22EE243C
:1098000025F582E43FF58322F0EE243112B678226A
:10981000F0EE243012B6782274F4122583EAFEEBBF
:10982000FF8C088D09900902E0600F12DB3870038D
:10983000A3E069700512314F804C790012D37E127B
:1098400032218A828B83E58245836032A3A3A3A35E
:10985000A3A3E054186027E508241C12C8D01229DD
:1098600095E508241312C8D0122995EE24181298F1
:109870008812988D1232397404122B848008790072
:1098800012988D123179802B12B678F9228E828F40
:1098900083A3A3A3A3A3A3A3A3A312B69A240B12E7
:1098A00098A322F582E43FF58312E9F8FB227418AD
:1098B000122B847F0402280974F012258374EA12A3
:1098C0002C188A0A8B0BEA2402F50EE4350BF50FEF
:1098D0000A0AFB122FB18A088B09AE08AF09750876
:1098E00001850A82850B83A3E0F509750C01AC0E96
:1098F000AD0F740B122E2DAA82AB83124853741332
:10990000122E2D129BA47415122E2D7402F07408C1
:10991000122E2DE4F0901037E0700EEE4F700AE535
:109920000970067508C3029AF8900555E06408604E
:10993000067508C2029AF4850A82850B83A3A3A345
:10994000A3A3A3A3A3A3A3E0A2E1500EA2E3500507
:10995000750C04800C750C038007A2E35003750C92
:1099600002EE4F7003029A048E828F83A3A3A3A3F7
:10997000E06404600D8E828F83A3A3A3A3E064033D
:10998000700C7404650C602C7403650C60268E8268
:109990008F83A3A3A3A3E06402600D8E828F83A3B1
:1099A000A3A3A3E0640170357402650C6006740122
:1099B000650C701C8E828F8312D38B123479E97000
:1099C000438E828F8312A68F122E2D12C8ED803403
:1099D0008E828F83A3A3A3A3E06402600D8E828F87
:1099E00083A3A3A3A3E06401700A8E828F8312A7CE
:1099F000F6122769E50A2402FAE4350BFB122FBDA3
:109A00007E007F007413122E2DE064FE7003A3E02D
:109A1000F4704E122F7BE97048E50960239005929F
:109A2000E06402701B90103E12D38B123479E970FF
:109A30000F90103E12A68F122E2DE8F0A3E9802081
:109A4000850A82850B83A3A3A3A3A3A3A3A3A3A394
:109A5000E05402F912318B7413122E2DEAF0A3EBAD
:109A6000F07413122E2DE064FE7003A3E0F4700571
:109A70007508C7807FE509F50D780D122B5A850A08
:109A800082850B83A3A3A3A3A3A3A3A3A3A3E0F90A
:109A9000E50A2402FCE4350BFD7414122E2D12D3BA
:109AA0008B1230D17401122B84E97048A90CE50A9D
:109AB0002402FCE4350BFD7413122E2D12D38B12ED
:109AC0002F8D8A0E8B0FAE0EAF0FEE4F601E7402FD
:109AD0006509700D8E828F83A3A3A3A3A3E0D2E3B5
:109AE000F07415122E2DE4F0F50880087413122E70
:109AF0002D129BA4E5097009AA18AB191249EB8035
:109B00000AFCA90CAA18AB19123419E9F8EE4F6037
:109B100053E50960208E828F83A3A3A3A3A3E0D281
:109B2000E6F074026509700D8E828F83A3A3A3A350
:109B3000A3E0D2E5F0850A82850B83A3A3A3A3A3A8
:109B4000A3A3A3A3A3E0A2E6500D8E828F83A3A3B9
:109B5000A3A3A3E0D2E7F08E828F83A3A3A3A3A342
:109B6000A3E004F0E5087003E86034FC7D007A01AE
:109B70007B10124835EE4F600CE50A2402FAE435FA
:109B80000BFB122FBD7413122E2DE064FE7003A385
:109B9000E0F4600B7413122E2D12A7F612276974CD
:109BA0001602C17574FEF0A304F02274F712258327
:109BB00074F7122C18EAFEEBFF900555E064036081
:109BC0000DE064016008E064096003029CD58E82A8
:109BD0008F83A3E06003029CAB7C007D007A027B54
:109BE00000124835129CDA8A828B8312B9049005E0
:109BF0004612C8ED79531249DF790090055312D30C
:109C00008B1230CB900555E0640960099005531222
:109C1000D38B123545851882851983740112CA3792
:109C200079421249DF9005557404F07401122BF249
:109C3000794A1249D97401122BFA7A4B7B051248E2
:109C400053900912E060046401701F900549E064BC
:109C5000FE7003A3E0F4602A79007401122BFA90DD
:109C6000054912D38B122F8D8018E0640270139077
:109C7000054612B0AC7A037B0012483512A5B61225
:109C80004835900540E0A2E35004D2F08002C2F0D3
:109C900012CA2D79521249DF900912E06402703223
:109CA00090108E12D38B12328180278E828F83A3E5
:109CB000AE82AF83FC7D007A037B101248358E8222
:109CC0008F83E0F990055312D38B1230CB9005555A
:109CD000E4F01232ED740902B1A4EE2402FAE43F7A
:109CE000FB22C082C08390051612CBD1701F900555
:109CF00055E014600924FC600A14600C800F900584
:109D00001F803490051B802F90051D802AE8496034
:109D10000890051712A31C700C8A828B83A3E0F9AC
:109D20001230B3801D900516129D45640270051215
:109D300034D9800E9005D712CBD1600612C63B12E3
:109D4000276902C1B0E0F8129D4B22A3E0C82406A7
:109D5000F582E438F583E02274F412258374FB1253
:109D60002C188A088B097A0F7B00123DAF8A0A8B68
:109D70000BAE0AAF0BEE4F7003029E778E828F837D
:109D8000740212CA3779501249D98508828509832D
:109D9000A3E06003029E5A900553E0F47003A3E031
:109DA000F46044900553E064FE7003A3E0F4603770
:109DB000851882851983129E7C7003A3E069602751
:109DC000850882850983A374EAF07A467B05795376
:109DD0001249DF7A497B05794B1249DF7A537B05BB
:109DE00079501249DF807385188285198312DC0946
:109DF00012C8ED7A467B0579531249D9900546126F
:109E0000AD4F12C8ED7A497B05794B1249D97A4892
:109E10007B0579E11249D990055AE0C3940F501D92
:109E2000900548E0C0E07402122E2DD0E0F07404DA
:109E3000122E2D7401F004122BF2124A03750A003F
:109E4000780A122B5A780A122B5A9010C4E0F91291
:109E5000AA3E1233D77402122B84850882850983A7
:109E600012D69EA3F09005557403F0EEFAEFFB9026
:109E700005A0E0F9123DBB74050298B012DC0DE0BC
:109E8000682274F412258374E8122C18EAFCEBFDA6
:109E90008C828D83A3A3A3A37808122DD6780812F1
:109EA0002D689005567808122CF87F7F7E7F790008
:109EB0009005567808122DD6E97808122BB9E508D6
:109EC000A2E0502978009005A180148508828509B8
:109ED00083A3A3E069700108E508241412C8D01216
:109EE000A71970E7E8C39F5004E8FFE9FE09E9C33A
:109EF000941B40BC8C828D83A3A3A3A3122E0AE8DB
:109F0000494A4B607DEC2404F508E43DF5098508D9
:109F100082F583122E0A900556122E167C187D00AB
:109F20007900AA18AB19123D97850882850983121A
:109F30002E0A851882851983122E167404122E2D6E
:109F40007401F090055CE0C0E07405122E2DD0E0A5
:109F5000F07407122E2DE412CA371249F780709060
:109F6000055312D38B1231018A0A8B0BA80AA90B55
:109F7000900553E8F0A3E912CBDE687003A3E06913
:109F8000602D9005A112A719602585088285098397
:109F9000129E7C7003A3E069700C8508828509839A
:109FA000A3A3E06E60B9E508241412C8D080D6EEF1
:109FB000900548F01232CFE96015900555E4F09015
:109FC000052112CBD1600879C412C63B1227690261
:109FD00098AE74F412258374E8122C188A828B834D
:109FE000A3A3A3A3A3A3A3A3A312B904E8FAE9FB21
:109FF00079009005567808122DD6E97808122BB909
:10A00000E508A2E05031EA29F582E43BF583E0F867
:10A0100090103DE0C398501F750801750900750A3E
:10A0200000750B00E97808122AF27808122D689062
:10A0300005567808122CF809E9C3941B40B4900522
:10A0400056122E0AE8494A4B604E7C187D00790072
:10A05000AA18AB19123D97900556122E0A85188240
:10A06000851983122E167404122E2D7401F07407B4
:10A07000122E2D7401F090055CE0C0E07405122EE4
:10A080002DD0E0F07407122E2DE412CA371249F7D2
:10A090009005557406F0801E900555E4F0FCFD7A9D
:10A0A000047B1012483590052112CBD1600879C489
:10A0B00012C63B1227690298AE74F512258374D13B
:10A0C000122C188A088B098A828B8312B908741C97
:10A0D000122BFA8A828B83A3A3A3A3A3A3A312B2F6
:10A0E0005312D3861232FF741C122E2DE0702C8571
:10A0F0000882850983A3A3A3A3A3A3A3A3E0C39476
:10A100000B40188E828F83A3A3A3A3A3A3A3A3E0D2
:10A110006402700712C8BBE0F4600302A30E90054E
:10A1200055E06402700302A1F0E06406700302A12E
:10A13000F090051612CBD1600812A31C700302A286
:10A1400025900555E064086008E06404600302A3FC
:10A150000E741E122E2D12A313A3A3A3A312B908CB
:10A16000900516E0F8496007129D4B6402607790F5
:10A170000553E06E7003A3E06F600302A30E740149
:10A180006A60167423122E2DAC82AD837A677B052C
:10A1900012484DE9600302A30E7A007B029005A0ED
:10A1A000E0F9123F29EA4B4C4D600302A30E9005E3
:10A1B00056122E0A851882851983122E1690055C78
:10A1C000E0C0E07404122E2DD0E0F07405122E2DA4
:10A1D0007401F07406122E2D740212CA3712303533
:10A1E000E9600302A30BEEFAEFFB1234D302A30ED5
:10A1F00090051612CBD1702D7508007808122B5AD5
:10A200007808122B5AEE2410F582E43FF58312CB26
:10A21000C5A3A3A3A3A3A3A3A3A312AE201233D7C2
:10A220007402122B848E828F8312B9047407122E4B
:10A230002DE8F0A3E912AD5912B9047409122E2DBC
:10A2400012CA26240D12BBAFC0E0740B122E2DD003
:10A25000E0F012C8BB12AD32740F7808122DB8743A
:10A260000C122E2DE508F07420122E2DE0C0E074A3
:10A270000D122E2DD0E0F07422122E2DE0C0E074CD
:10A280000E122E2DD0E0F0741D122E2DE0C0E074C1
:10A2900010122E2DD0E0F0741E122E2DE0C0E074AE
:10A2A0000F122E2DD0E0F0EE241012BBAFC0E074E0
:10A2B00011122E2DD0E0F07421122E2DE0C0E0748A
:10A2C00012122E2DD0E0F0742E122E2DE0C0E0746C
:10A2D00013122E2DD0E0F07423122E2DA982AA8302
:10A2E00089088A09750A007808122B527C087D00BB
:10A2F0007417122E2DAA82AB83123D8B7403122B7E
:10A30000847407122BF21230C5800312303B742F75
:10A3100002EF8BE0FA8E828F83A3A322129D4C64FE
:10A32000012274F612258374C9122C189005D112DB
:10A33000CBD1600612C63B122769900555E0640830
:10A34000700302A3DF900592E0640270239051C471
:10A35000E493900537F09051C4E493900535F09064
:10A36000055E7401F01297F004F0A3E4F0A3806C92
:10A37000900566E0F8743128F582E4340AF583E04C
:10A38000FA900537F0743228F582E4340AF583E058
:10A39000F9900535F07508FF7509FFEA7808122D68
:10A3A00044E508F4FCE509F4FD3395E0FE90055E14
:10A3B000ECF0A3EDF0A3EEF0A3F07508FF7509FF34
:10A3C000E9C39A7808122D44E508F4FCE509F4FD88
:10A3D0003395E0FEA3ECF0A3EDF0A3EEF0A3F07C48
:10A3E000237D0079007414122BF2123D97900566BC
:10A3F000E07009741E122E2D74018006741E122E38
:10A400002DE412A524740FF090103C12CA3779463F
:10A410001249DF7401122E2DE4F090109DE0C0E08F
:10A420007402122E2DD0E0F0900543E0C0E07403DA
:10A43000122E2DD0E0F07404122E2DE4F0740512CB
:10A440002E2DE4F07407122E2DE4F0900566E0C383
:10A45000940F500CE0C0E07406122E2DD0E080075F
:10A460007406122E2D740FF07C677D057408122E71
:10A470002DAA82AB831248537C037D0079FF7410B0
:10A48000122E2DAA82AB83123D9790059FE0C0E06B
:10A490007413122E2DD0E012C82F7401122BF21259
:10A4A00032F97AA37B0579451249DF12340790050A
:10A4B0005AE0C0E0741C122E2DD0E0F090055BE055
:10A4C000C0E0741D122E2DD0E0F0900548E0C0E0F1
:10A4D000741A122E2DD0E01284ED7418122E2D1243
:10A4E000C8ED7420122E2DE4F090055DE0C0E074FC
:10A4F0001F122E2DD0E0F07434122E2DE4F07429AA
:10A50000122E2DE4F07A467B0579531249DF7A4901
:10A510007B05794B1249DF7414122BF21249FD743A
:10A520003702C52112A52822F085188285198322B9
:10A53000C082C0838A828B83A3E09005556004E4C7
:10A54000F080707408F0900566E070289005211284
:10A55000CBD16008790012C63B12276990055312CF
:10A56000B0AC7A057B0012483590055312D38B129C
:10A570003545801879001230BF90054612B0AC7A8C
:10A58000067B0012483512A5B61248359005DD123B
:10A59000CBD1601F900906E06401701790811812FA
:10A5A000298D7A007B409005A0E0F9123F177404D2
:10A5B000122B8402C1B090054912B0B07A047B001E
:10A5C0002274F412258374EA122C18EAFEEBFF12AF
:10A5D0009CDA122FB18A088B09EA4509700302A69A
:10A5E0008A8A828B83A3A3A3A3E0640160278A8263
:10A5F0008B83A3A3A3A3E06402601A8A828B83A344
:10A60000A3A3A3E06403600D8A828B83A3A3A3A307
:10A61000E064047075EE2402FCE43FFD740B122E1E
:10A620002DAA82AB8312485385088285098312A61E
:10A630008F122E2D12C8ED7415122E2D7401F07488
:10A6400008122E2DE412CA371249F1890AAC0A7D8C
:10A65000007A077B00124835850882850983A3A309
:10A66000A3A3A3E0C2E012C11CA3A3740112E2E100
:10A670005001097A027B00122326E88508828509A9
:10A6800083A3A3A3A3A3A3A3A3F074160298B01259
:10A69000D14C74132274F212258374F8122C18EA28
:10A6A000FEEBFF8C0A8D0B890C9080BAAC18AD19AB
:10A6B0007408122AB2F50DEEFCEFFDAA18AB1912C0
:10A6C000484DE97003750D019005A1801AEEFCEF6D
:10A6D000FDE508240BFAE43509FB12484DE9702327
:10A6E000E508241412C8D012A7196024E50DA2E0D1
:10A6F00040DB850882850983E0650A7004A3E06574
:10A700000B70DD850882850983A3A3E0650C70D0FA
:10A71000AA08AB09740802D15A12AD36E5084509FA
:10A7200022C082C0839005A102C1AD74F7122583B7
:10A730009005A112E9F8800C12D41712B90B123E41
:10A7400057EEFAEFFBEA4B70EF9005A1E4F0A3F0AF
:10A7500002B1A774F4122583EAFEEBFFEE24131274
:10A76000BBAF6403700CEE240BFAE43FFB122FB175
:10A77000800EE06402707C12C8BB12D38B122FAB28
:10A780008A088B09E508450960698E828F83A3E0FA
:10A79000700F850882850983A3A3A3A3A3A3E480E4
:10A7A0005164F1600A8E828F83A3E064E170278593
:10A7B0000882850983A3A3A3A3A3A3E06401701661
:10A7C00085088285098312A7F6122769EE240BFA01
:10A7D000E43FFB122FBD850882850983A3A3A3A3B1
:10A7E000A3A3E0600E850882850983A3A3A3A3A386
:10A7F000A314F00298B31298A990052F12C9012250
:10A8000074F11225838A088B09ECFEEDFF890A1288
:10A81000D68BEEF8EFF9A30EAF838A828B83A3A3C6
:10A82000E0C454F0FA88828983E04A12A8E112D683
:10A830009F12A8DCE0333354FCF88E828F83E0480B
:10A8400012A8DCA3E033333354F8F88E828F83E010
:10A8500048F0EEF8EFF9A30EAF838508828B83A34F
:10A86000A3A3A3A3A3E0A2E0E4331313FA8882898D
:10A8700083E04AF0E5082407F50CE43509F50D7589
:10A880000E00780C122B527C087D00EEFAEFFB12C2
:10A890003D8B7403122B84EE2408FE50010FE50853
:10A8A000240FF50CE43509F50D780C122B527C03BE
:10A8B0007D00EEFAEFFB123D8B7403122B84E50A48
:10A8C000C3940F4012E5082412F582E412DF158EBE
:10A8D000828F83A3A3A3F07F0702280912A8E1A314
:10A8E00022F08508828B83A3A3A32274F11225830F
:10A8F000EAFEEBFF890A8C088D098E828F83E08C3B
:10A90000828D8312B6AAAE82AF83E012BF4A12C113
:10A9100038C412BF4A12A9B5E054038C828D831249
:10A92000C136A2E2E4338C828D8312C13513131336
:10A93000541F12BF4A12C134A2E7E4338C828D83C4
:10A94000A3A3A3A312A9B58E0C8F0D750E00780CCE
:10A95000122B527C087D00E5082407FAE43509FB38
:10A96000123D8B7403122B84EE2408FE50010F8ECF
:10A970000C8F0D780C122B527C037D00E508240F00
:10A98000FAE43509FB123D8B7403122B84E50AC3EC
:10A99000940F40158E828F83A3A3A3E0C0E0E50847
:10A9A000241212C8D0D0E08008E508241212C8D0C2
:10A9B000E4F002A8D7A3A312B6AE0EAF832274F5BB
:10A9C0001225838A088B098A828B83A3AE82AF8388
:10A9D000E0F91230E98E828F83E064EB6024850811
:10A9E00082850983A3E064E1601885088285098374
:10A9F000A3E064F1600C850882850983A3E0641AF2
:10AA00007009850882850983A3E4F090108E12D323
:10AA10008B123281750A01780A122B5A85088285B9
:10AA20000983A3E0F5087808122B5A790012AA3E90
:10AA30001233D77402122B8412331702EF8E900553
:10AA40005312B0B09005491298A922C082C083E980
:10AA50009005B37003E4800274018065E0F902C1DF
:10AA6000B074F7122583EAFEEBFF8E828F8312C942
:10AA7000FF12DA6412DA7F12345BE98E828F836010
:10AA80000512AA92800312AAA712AAB0124A0F02B4
:10AA9000B1A712AA99E4F0A322E0F8A3E0C8240D1C
:10AAA000F582E438F5832212AA997401F0A3E42216
:10AAB000F07C6F7D328E828F831298A922EAF0A3F8
:10AAC000EBF002C1B074F61225839005B3E0701B61
:10AAD0007C0079017A007B00123347EA4B600C8AD4
:10AAE000828B8312CBD1600312327502C524C082DF
:10AAF000C0837904123341E9F89051D1E493C398AB
:10AB0000401079FF123341E9F89051D0E493C39893
:10AB1000500479018002790002C1B074F0122583DB
:10AB20008A088B09890B750C008A828B83A3A3A3E7
:10AB3000A3A3A3A3A3E0F912334D8A0E8B0FAE0E8D
:10AB4000AF0F750A01EE4F600302ABEB85088285FB
:10AB5000098312AD3EA3A3A3A3A3A312BC8412D363
:10AB60008B1233358A0C8B0DAE0CAF0DEE4F70038C
:10AB700002AD248E828F83A3A3A3A3E4F0A3F0E508
:10AB800008240CFAE43509FB8A828B83E0C0E012CA
:10AB9000E2D7D0E0F0123467EE240D12DA79E5083E
:10ABA00012DF07350912B90212B66C12C8ED750C26
:10ABB00001EE240612BBB3547FF0A3E054FC12E66E
:10ABC000D85404600302AC62901096E0F508750951
:10ABD0000074077808122D448E828F83A3A3A3A349
:10ABE000A3A3E04508F0A3E04509F08E828F83A37C
:10ABF000A3A3A312AD3074077808122DB8E508544A
:10AC000007F508E50B606B8E828F83A3A3A3A3A334
:10AC1000A3A3A3A3740212C13912B01B600B900549
:10AC20004112AD4FA3A312C8EDE508700302ACF0CA
:10AC3000EE240612EE10547FFCA3E054FCFDE50860
:10AC400024FFF508E434FFF50974077808122D4451
:10AC5000EC4508F8ED4509F98A828B8312C8ED02AC
:10AC6000ACF08E828F83A3A3A3A3A3A3E0448002AE
:10AC7000ABEAE5087005750A0080758E828F83A3A4
:10AC8000A3A3A3A3A3E05420600C123DA9EA547F20
:10AC90007900245F80198E828F83A3A3A3A3A3A32B
:10ACA000E05410601A123DA9EA540F7900240A50AA
:10ACB00001098E828F83A3A3A3A3F0A3E9800D8E45
:10ACC000828F83A3A3A3A37401F0A3E412AD5974EC
:10ACD00004F07A207B009005A0E0F9123F29EA4BAE
:10ACE0004C4D700C7A207B009005A0E0F9123DF1EC
:10ACF000E50CA2E050318E828F83A3A3A3A312D3CD
:10AD00008FF9EEFAEFFB12333BE9601B12B19C1294
:10AD1000CBCF600912B28B12D38B123E57EEFAEFF3
:10AD2000FB123E57750A00A90A02C1788E828F83F2
:10AD3000A3A312AD3622E0F508A3E0F50922A3A3F0
:10AD4000A3A3A3A312B0B0850882850983A322120E
:10AD5000D14C8E828F83A3A32212C8DDA3A3A3228A
:10AD600074F412258374F7122C187E0012334DEA06
:10AD70004B700302AE198A828B83A3A3A3A3A3A360
:10AD8000A3A3A3E06406600302AE198A828B83A3A7
:10AD9000A3A3A3A3A3A3E0FF8A828B8312AE2BE01D
:10ADA000C0E07408122E2DD0E012B27012C8EA1260
:10ADB000336BEF5408606085188285198312B0AC3C
:10ADC0007A007B0012332F8B0BEA450B704912EF90
:10ADD00085124A277C007D007A007B0080258E82C8
:10ADE0008F8312B09FF47003A3E0F4602A900553A0
:10ADF00012AE20124A21E9641A601C7C007D00EE2C
:10AE0000FAEFFB12332F8A0A8B0BAE0AAF0BEE4F11
:10AE100070CC7900124A2D7E01EEF974090298B0C7
:10AE200012B0B08E828F831298A92212B8F612AE99
:10AE300032222408F582E438F58322C082C083EAF6
:10AE40004B70059005B480068A828B83A3A312B051
:10AE50004F60258A828B83A3A3A3A3A3A3A3E0545B
:10AE60000860E5EC4D60158A828B8312B09F6C7090
:10AE700003A3E06D70D280047A007B0002C1B0743D
:10AE8000F2122583EAFEEBFF890A8C088D097A11FC
:10AE90007B00123E51EA4B603E8A828B83A3A3A3C0
:10AEA000A3A3A3A3A3A3E412B264A3E50A12DC1C28
:10AEB000A3A3A312F0668A828B83A3A3A3A3E4F0C7
:10AEC000A312B28512AEE512DA6C12B77AE4F01270
:10AED000AEDAA3A3F0A3F002D15DA312AEDF22F09D
:10AEE0008A828B8322A3F012EE3C3BF583E4F022AE
:10AEF00074F4122583EAFEEBFF89088C0A8D0BEEB1
:10AF00004F700302AFA47401650870127901123307
:10AF100041E9F89051D6E493C39850228016740406
:10AF2000650870147904123341E9F89051D1E49323
:10AF3000C398500A7911806E7402650870668E821B
:10AF40008F83A3A3A3A3A3A3A3A3A3E50812BEB5C2
:10AF500012D6838E828F83A3A3E4F0A3F09005B46E
:10AF600012CBD160178003E0F8A312CA06A3A31284
:10AF7000B04F88828983A3A370ED80039005B4123B
:10AF8000DA707A207B009005A0E0F9123F29EA4BA5
:10AF90004C4D700C7A207B009005A0E0F9123DF139
:10AFA0007900800279C10298B3C082C083E9F87940
:10AFB000009005B4801D8A828B83A3A3A3A3A3A3BF
:10AFC000A3A3A3E068600574FF687001098A828BFF
:10AFD00083A3A312B04F70DE02C1B074F7122583B1
:10AFE000EA4B70059005B480068A828B83A3A31276
:10AFF000B04F60208A828B83A3A3A3A3A3A3A3A3A0
:10B00000A3E06970E4EC60108A828B83E012B01BCD
:10B0100070D780047A007B0002B1A712AA9AE0548C
:10B020000422C082C0839005B480068A828B83A3E9
:10B03000A312B04F60128A828B83A3A3A3A3A3A3FE
:10B04000A3A3E06970E580047A007B0002C1B0121E
:10B0500098A9EA4B2274F7122583EAFCEBFD9005D0
:10B06000B480068A828B83A3A312B04F60218A82A8
:10B070008B8312B09F6C7003A3E06D70E68A828BA5
:10B080008312867A12CAECA2E0E43370D680047A86
:10B09000007B0002B1A7EE241DF582E43FF5831288
:10B0A000B27722EE2413F582E43FF58312B0B0228A
:10B0B00012B0B422E0FCA3E0FD2274F21225838AD0
:10B0C0000A8B0B8C0C8D0D750800750900EA450B79
:10B0D00060309005B480068E828F83A3A312B90BD3
:10B0E000EE4F601EAC0CAD0DEEFAEFFB850A8285CB
:10B0F0000B83122769E9640170DDEEF8EFF9880827
:10B100008909AA08AB0902D15D7900022B3674F7D0
:10B110001225839005B412B9047C007D00800DE8EF
:10B12000FCE9FD88828983A3A312B904E849603051
:10B13000EA687002EB6970E79005B412D38BE86A95
:10B140007002E96B88828983A3A3700812B9049006
:10B1500005B4800912B9048C828D83A3A312C8EDB3
:10B16000804574F7122583EAFEEBFFEE4F602B1249
:10B17000336512B291123E578E828F8312D38B1297
:10B180003E5712B19C12CBCF600912B28B12D38BF7
:10B19000123E57EEFAEFFB123E57800BEE240DF5F0
:10B1A00082E43F22122B847F0102280974F71225C2
:10B1B000838A828B8312B25C9005B412B90475083D
:10B1C000007E00803388828983A3A3A3A3A3A3A3C3
:10B1D000A3A3E0640570180E88828983E0FFA3E0D2
:10B1E000F5838F82E06C7003A3E06D700205088820
:10B1F000828983A3A312B904E84970C99051CD1282
:10B20000E42C50089051C912D2CC400F8A828B8313
:10B21000A3A3A3A37401F0A3E4800C900541E0F87C
:10B2200012B253E8F0A3E912B285740512B264E0D9
:10B23000440812B270F47003A3E0F4600E9005535A
:10B2400012D586124A21E9641A70057901124A2D35
:10B2500002B1A7A312B654A3A3A3A32212B277FCF0
:10B26000A3E0FD2212B2682212DC24A3A3A3A3222E
:10B2700012AEDF12B27722E0F812B27D22A3E0F51F
:10B28000838882E02212B268A3A32212B19CF583C4
:10B290002212B2981298A7228E828F83E0F8A3E040
:10B2A000C8241FF582E43822C082C083EAFCEBFD8B
:10B2B000EC4D6017EC24FBF582ED34FF12CBCF7020
:10B2C0000712B302E0F46007123DB57905803090B3
:10B2D00005A0E0C0E012B302D0E0F09051C1E493C9
:10B2E000F97AB67B05123DEBE9640170107A007BB8
:10B2F000209005A0E0F9123DF17900800279040266
:10B30000C1B0EC24FFF582ED34FFF5832274F41212
:10B310002583A2AFE433F508C2AF9005B612B90B8E
:10B32000EE4F603AEE24FBF582EF34FF12CBCF7A7A
:10B33000007B209005A06007E0F9123DF18005E058
:10B34000F9123DF7E4F50AF50B780A122B56EEFCDC
:10B35000EFFD7AB67B05123DE57402122B84E508F9
:10B36000A2E092AFEEFAEFFB0298B374F0122583DD
:10B3700074DB122C18EAFEEBFF750B00750A0075E2
:10B3800008FE7509FF12331DE9600302B647EE247B
:10B390001512BBAF60469010B1E0C43354E0F8E042
:10B3A000333354FC48C0E012D370D0E012B6AA1276
:10B3B000D38A79FF122E738B0DEA450D6011750B40
:10B3C000017508FF12B671440412C90AD2E0F09068
:10B3D0000912E0600464017003750A408E828F8355
:10B3E00012D38912345BE9600312C9DDEE24131213
:10B3F000BBAF700D9051CCE493C0E012CACDD0E049
:10B40000F08E828F83E0A2E7500454038019EE246B
:10B410001412BBAF7012900532E0C0E012EDEED016
:10B42000E0F0900532E004F012EE07701990109FE2
:10B43000E0600D90053DE0700D8E828F83E0700618
:10B44000EE241112C9E0900912E060046401704812
:10B45000900540E0A2E15040E50BA2E040218E8241
:10B460008F8312D38912345BE9602D8E828F83E043
:10B47000600DEE240B12B099F9123437E9601912FD
:10B48000B680700302B5F8EE241312EE0A600302D0
:10B49000B5F812B67154FBF08E828F83E0640170B0
:10B4A0000DEE240B12B0996402700312B68D12B621
:10B4B00080600302B571E50BA2E0500302B5719004
:10B4C0000912E060076401600302B571900540E075
:10B4D000A2E1400302B571E50AF50B780B122B5A75
:10B4E000EE2406FCE43FFD8E828F8312D389EE2486
:10B4F000121298881232337401122B84E9600612FA
:10B50000C9DD12B6868E828F83A3A3A3A3A3A3E073
:10B51000603CEE2402F50CE43FF50D850C8212B67A
:10B52000942407FAE43FFB12339B8A088B09850CAD
:10B5300082850D83E065087004A3E06509700C8EB8
:10B54000828F83A3A3A3A3A3A3E4F012B68D8E825C
:10B550008F83E064016008A90A12B69F1231D3A953
:10B560000A8E828F8312B69F123161E9600312B690
:10B5700086AC18AD19EEFAEFFB1233958A0A8B0BE5
:10B5800074FE6508700474FF6509700312AD2CEA3F
:10B59000450B700302B64B8E828F83E0C0E07401CE
:10B5A000122E2DD0E0F07402122E2D12DA707401DA
:10B5B000122BEA880C890D780C122B5612B66C12DD
:10B5C0002995EE240E12BBAFF50C780C122B5A9075
:10B5D00005461229957407122E2DE0F9AC08AD0925
:10B5E00012338F7407122B84E9FE74106E705EAAFA
:10B5F0000AAB0B123E578055EE241312BBAFC0E0CE
:10B600007415122E2DD0E012EE6B740D122E2D1229
:10B61000CA26240412B65B12B904740F122E2D121E
:10B62000CA26241412BBAFC0E07416122E2DD0E02F
:10B6300012E2CD12B65412B0AC7404122BF21232D4
:10B6400003E9600302B498791180047E10EEF97466
:10B650002502C175E0F98A828B832212B65F22F837
:10B66000E43FF9E8FAE9FB8A828B8322EE12C9F201
:10B670002212B67522EE240FF582E43FF583E02214
:10B6800012B67554402212B6754420F02212B675D7
:10B690004440F022F58312B69A2212B0B4EE22A3EF
:10B6A000A3A3A312D39B1298A92212B6AE22F08EA6
:10B6B000828F83A322C082C08374DC122C188A82FA
:10B6C0008B83A3A3A3A312B904740E122E2DE8F04A
:10B6D000A3E912D143740C122E2D12C8ED12B77AC1
:10B6E000E0C0E0741A122E2DD0E0F012B7843B12A5
:10B6F000B9027420122E2D12C8EDEA12D3783BF550
:10B7000083E0C0E07408122E2DD0E0F0EA241CF58E
:10B7100082E43B12B9027412122E2D12C8EDEA24F3
:10B7200011F582E43BF583E0C0E07409122E2DD0C0
:10B73000E0F0EA2412F582E43BF583E0C0E0740710
:10B74000122E2DD0E012A52474FFF07401122E2DBC
:10B7500074FFF07402122E2D74FFF090811C1229D8
:10B760008D7404122BFA7407122BF21230AD74048C
:10B77000122B84790074240284F7EA240DF582E404
:10B780003BF58322EA12EE3D2274EE12258374EF1C
:10B79000122C188A0E8B0F8C088D09890C750A10D3
:10B7A0007A217B00123E5112D1A3E849700302B8FE
:10B7B000EF750B007C217D00790085188285198347
:10B7C000E0FA123D977426122E2D12B90B90091231
:10B7D000E060046401703EAA08AB09122FAB8A1026
:10B7E0008B11A810A911E849602388828983A3A33B
:10B7F000A3A3E06401600D88828983A3A3A3A3E0CF
:10B8000064037009EE5440700474044FFFEF540455
:10B810006003750B0190055312D38B85188285192F
:10B820008312B8F62409F582E43812DA7D74231203
:10B830002E2D12B904740F122E2DE8F0A3E912B9BF
:10B840001112EE3312B91112AE32740212BC8E1202
:10B85000C639E508F0A3E50912B91112EDFEE50CB1
:10B86000F07425122E2DE0F50885188285198312B3
:10B87000EE43E50812B911241FF582E438F583E59B
:10B880000EF0A3E50FF07406122E2D12DA70740874
:10B89000122E2DE508F07428122E2D12C638C08203
:10B8A000C083740C122E2DAC82AD83D083D08274F1
:10B8B00003122AB2A90BAA18AB19123323E96401A7
:10B8C0007021900912E0600464017012E50BA2E09F
:10B8D000500CA90812334DEA4B6003123371750AFC
:10B8E00000800C85188285198312D38B123E57A9CC
:10B8F0000A741102BEC212D151C822EE2413F5827D
:10B90000E43FF58312D14C22A3A3A3E0FEA3E0FF02
:10B910002212D1B2C82274EE122583EAFEEBFF8C0C
:10B92000088D098E828F83A3740812CA19E06008FB
:10B930008E828F83A37410F012BBAC60098E828F4D
:10B9400083A3E02408F0EE241512BBAF60088E82BA
:10B950008F83A3E004F08E828F83A3A3A3A3A3A36A
:10B96000E060198E828F83A3A3A3A3A3A3A3E0C344
:10B97000332402F88E828F83A3E028F0EE24111284
:10B98000BBAF6005750B0E8003750B008E828F8335
:10B99000A3E0F8EE240D12BBAF28250B8C828D831B
:10B9A000F0EE241112BBAF601190053EE0F9122FAA
:10B9B00003850882850983E029F08508828509834B
:10B9C000E0C39475400975080075090002BBA5E045
:10B9D000FA7B00123E518A088B09EA45097003027E
:10B9E000BBA58E828F83E0FA90054312BBBD740223
:10B9F000780C122D44EA450CFAAB0DEE241212BB62
:10BA0000AF5403F50C750D007406780C122D44EA42
:10BA1000450CFCEBFDEE241512BBAF6004780180F1
:10BA2000027800EE2416FAE43FFBE8F9ED49FDEE5A
:10BA3000241112BBAFF50C7409780C122D44ED459E
:10BA40000DFD8A828B8312BBBD740B780C122D44C2
:10BA5000ED450DFD12BE9212BBBD740C780C122D7B
:10BA600044ED450DFD8E828F83A3A3A3A3A3A31250
:10BA7000BBBD740A780C122D44ECF8ED450DF9E8C5
:10BA8000850882850983F0E9A3F0EE240212BBB396
:10BA900085088285098312BBE1F0EE2404F8E43FB7
:10BAA000F98882898312C0E3A312BBE1A3A3F0EE5D
:10BAB000241312BBC4F0EE241412BBC4A3F0750A05
:10BAC000088A828B83E06015EE241812B0A6E50880
:10BAD0002408FAE43509FB124853750A1012BBAC6E
:10BAE000601BEE241A12B0A6850A0CE508250CFA94
:10BAF000E43509FB1248537408250AF50A8E828F33
:10BB000083A3A3A3A3A3A3E06058EE2407F510E446
:10BB10003FF511851082F583E0C0E012C8C9D0E07E
:10BB200012BBD1E0C0E012C8C9D0E012BBD112975D
:10BB3000D8122B52851082851183E025E0FCE43376
:10BB4000FD850A0CE508250CFAE43509FB123D8B4E
:10BB50007403122B84851082851183E0C333250A78
:10BB6000F50AEE241512BBAF6008C0E012C8C9D0B8
:10BB7000E0F012C8BB1297D9122B52EE240D12BB63
:10BB8000AFFC7D00850B0A8E828F83A3E0F8E50869
:10BB900028F8E43509F9E8250AFAE439FB123D8B67
:10BBA0007403122B84AA08AB0902BEC5EE24171237
:10BBB000B67822F8E43FF988828983E022E0F50C28
:10BBC000750D0022F582E43FF58312BBEAA3A3A31F
:10BBD00022F0050A8E828F83A3A3A3A3A3A3A3A30A
:10BBE00022A3A312DFFB12BBEA2212C0E7A3A32207
:10BBF00074F412258374FD122C188A088B09ECFE4C
:10BC0000EDFF7401122BEA880A890B780A122B5671
:10BC10007402122BFAEEFAEFFB1231AF7402122B00
:10BC200084E97057851882851983E0850882850923
:10BC300083F07401122E2DE0F812BC84A3A312BC71
:10BC400092602914850882850983A312BC8E12D7BD
:10BC5000647401122E2DE028F8A3E039F9E824FEDF
:10BC6000F582E934FFF58312E9F8800C85088285B6
:10BC70000983A3E4F0EEFAEFFB80047AFE7BFF7405
:10BC8000030298B0A3E0F98508828509832212BCDB
:10BC90009A22E8F0A3E912BC9A2212BC9E2212A5B5
:10BCA00028E02274EE1225838A0A8B0BECFEEDFF4E
:10BCB000750F01E9C39408500302BE2A8E828F8358
:10BCC000E912AEDB12C10E1233A7E96003750F0053
:10BCD00012C0F08E828F8312C140EE12B7853F12E0
:10BCE000C12AC0E0EE2411F582E43FF583D0E012D2
:10BCF000C122C0E0EE2412F582E43FF583D0E012C9
:10BD0000B6AA740812BEB5A3A3A3E06018E50A247E
:10BD100008F8E4350BF912CACD12C8ED8E828F8374
:10BD2000A3E02408F08E828F83A3A3A3A3A3A3A3DD
:10BD3000A3E0601C8E828F83A3858208858309120D
:10BD4000C103EE241512E2AFA3E912CBDE2408F002
:10BD50008E828F83A3A3A3A3A3E0600F12BE9C8E49
:10BD6000828F83A3A3A3A3A312BEBCEE241912C97E
:10BD7000E0EE241B12C9E0A3F0EE241812BBAF7052
:10BD80000302BE1A12BE9CFAEE2419F582E43FF5B6
:10BD900083EA12BEBCF8E50A28F582E412E2A6F8AE
:10BDA00012CBE2E812BEBCE8C39AEE506824191226
:10BDB000BBAFF89051C0E493C398500575110C8047
:10BDC00008EE241912BBAFF5118E828F83A3E0F821
:10BDD000E50A28F50CE4350BF50D750E00780C120C
:10BDE0002B52AC11EC2CFCE433FD7AD17B0E123DCE
:10BDF0008B7403122B84EE241BF582E43FF58374CD
:10BE0000D1F0A3740EF0E511C333F88508828509DB
:10BE100083E028800412C9D9E4F08E828F83A3E0E6
:10BE2000F88E828F83E0C398500479008062A3E08B
:10BE3000FAE50A28F8E4350BF9EE241D12E2AFA367
:10BE4000E912C139C39AC0E012BE92D0E012C8D83C
:10BE5000603CEE2417F8E43FF9880889098882F5E8
:10BE600083E024F2F0EE241D12BBB3240EFAA3E00B
:10BE70003400FB8882898312DA7F90053EE0F91254
:10BE80002F03E9F8850882850983E0C398F0A90F9C
:10BE90008033EE2417F582E43FF583228E828F8370
:10BEA000A3858208858309E0F8E50A28F582E43550
:10BEB0000BF583E02212B6AEA3A3A32212CBEC04AF
:10BEC000F022122B847F0A02280974F41225838A37
:10BED000088B09EA12BF51F0EA1313543F12BF4A0C
:10BEE000A3A3A3F0EAC4131312BF51A3A3F0EB1250
:10BEF000BF5C12BF647409780A122DB812BF5A12BF
:10BF0000BF63740A780A122DB8E50A5401C0E0EC48
:10BF10002418F582E43DF583D0E012BF69740B78F4
:10BF20000A122DB812BF5AA312BF63740C780A12FA
:10BF30002DB812BF5AA3A3A3A3A3A3A3A3F0740D68
:10BF40007808122DB8A9080298B3540F8C828D83FB
:10BF50002254038C828D83A3A322E50A54018C8290
:10BF60008D8322A3A3A3A3A3A3F08A0A8B0B22C0D1
:10BF700082C08379008A828B83A3A3A3A3A3A3E0B7
:10BF800090053D600EE070228A828B83A3A3E0704F
:10BF9000198016E060148A828B8312D38290054642
:10BFA000E06A7003A3E06B60010902C1B074F01293
:10BFB00025838A0A8B0B890C8C088D098A828B83D6
:10BFC00012C10E1233A712C0F085088285098312B0
:10BFD000C140E50812B785350912C12AC0E0E5085D
:10BFE000241112C8D0D0E012C122C0E0E50824120A
:10BFF00012C8D0D0E012EE96740812C11CE0601E88
:10C00000E50A2408F8E4350BF9E508241312C8D032
:10C0100012C8ED850882850983A3E02408F085080D
:10C0200082850983A3A3A3A3A3A3A3A3E0601B8585
:10C030000882850983A312C0FFE508241512C8D021
:10C04000E8F0A3E912C1392408F085088285098344
:10C05000A3A3A3A3A3E06019850882850983A3AEE7
:10C0600082AF8312BEA785088285098312C134047A
:10C07000F0AA08AB091233ADE9F50D7061850882AD
:10C08000850983A3A3A3A3A3A312C0E3701AE0FAB4
:10C09000E50A2AF8E4350BF9E508241D12C8D01288
:10C0A000C8EDE50CC39A802A12C0FFE8240EF850B0
:10C0B0000109E508241D12C8D012C8ED90053EE024
:10C0C000F9122F038E828F83E0F8E50CC39824F2D7
:10C0D000C399C0E0E508241712C8D0D0E0F0A90D3C
:10C0E00002C17812C0E722E0850882850983A32275
:10C0F000850A82850B83A3A312C156E0F9EA22AE1A
:10C1000082AF83E0F8E50A28F8E4350BF922E0FA7B
:10C11000A3E0F8E4C8F9EA28E439FB2212EE79A397
:10C12000A32212C169A3A3A3E022F583E812C1628E
:10C13000A3A3E022A3A3A3A3A3F08E828F83E02274
:10C14000A3A3A3A3A3A3A3A3A312C16212C156A333
:10C15000A3E0F9EAF822E0FA850A82850B83A3A31B
:10C16000A322F0A3E912C16922F0850A82850B831C
:10C17000A3A3A3A322122B847F08022809C082C094
:10C18000837AC47B0579E21249D97AC47B05802081
:10C19000C082C0839005468014C082C08390054948
:10C1A000800BC082C083794A1249D9800312D38B95
:10C1B000D083D082022B3674F61225839005CCE012
:10C1C000FE04F0EEF912334D8B09EA450970EDEEED
:10C1D00060EAF902C52474EE122583EAFEEBFF8CB7
:10C1E0000E8D0F890A750B00750C0012354B8A08ED
:10C1F0008B097412122E2DE0F5107413122E2DE0FF
:10C20000F50DEA45097017E50D600302C2FAA90AA7
:10C21000AC0EAD0FEEFAEFFB12356F02C408E50D60
:10C22000700302C2C0900912E060046401700E90B5
:10C2300005D912CBD1600612C63B122769E51070F2
:10C240000B850882850983E4F002C2F5900912E0AB
:10C2500060076401600302C31D900540E0A2E14055
:10C260000302C31D9005DB12CBD1600CA910AA08F4
:10C27000AB0912C63B122769850882850983E0FA5B
:10C2800012E2C2500109C3EA98E499A2D265D03300
:10C290005009850882850983E004F08508828509B4
:10C2A00083E0F89051D7E493687072750B01EEFA51
:10C2B000EFFB12323F850882850983A3E4F0805D9D
:10C2C000E5107021EA2402F582E412DF15850A0EDA
:10C2D000250EF8E4340013E813F070098A828B838A
:10C2E000A3A37401F08A828B83A3A3E0F89010C407
:10C2F000E0C3985028750C0180237401650D701DF2
:10C30000E5106019900912E060046401700F900557
:10C3100040E0A2E15007EEFAEFFB12323F90091223
:10C32000E06402600FE060046401702A900540E060
:10C33000A2E140227401650D701CE5109005EB60D0
:10C3400013E004F0901097E0F89005EBE0C39840FC
:10C3500005750B01E4F0E50CA2E092F0E50BA2E01C
:10C3600072F0400302C408900912E0600464017096
:10C3700041900540E0A2E15039EEFAEFFB122FABFD
:10C380008A088B09A808A909E8496026E50CA2E0FB
:10C39000500D88828983A3A3A3A3A3E0C2E0F0E5A4
:10C3A0000BA2E0506388828983A3A3A3A3A3E0D256
:10C3B000E0F0E50BA2E05050900912E06004640147
:10C3C000701D900540E0A2E15015EEFAEFFB122F30
:10C3D00099E9600BEEFAEFFB79001230E3802990C7
:10C3E0000549E06E7003A3E06F701DEEFAEFFB7974
:10C3F000011230E3900912E06402700C7A017B00B4
:10C400009005A0E0F9123F2302BEC574F412258303
:10C4100074016A4B700E7A017B009005A0E0F9125E
:10C420003DF1803790108E12DA7FEA4B60218A0846
:10C430008B09E4F50AF50B7808122B4E7A017B0084
:10C440009005A0E0F9123F177404122B84800C7A37
:10C45000017B009005A0E0F9123F230298B3C0824F
:10C46000C08390109002AABDC082C0839010920237
:10C47000AABD74F61225837508327509057808126D
:10C480002B567C6E7D007A217B00123EC97402120D
:10C490002B84E9F508122F27E94208900912E06081
:10C4A0000464017006122FD5E9420890070F12CBE1
:10C4B000D1600912C63B122769E94208122E97E99A
:10C4C000FE1243D9E9F8E5084E48F9805774F61290
:10C4D000258312482F7508327509057808122B56E6
:10C4E00075086E7509007808122B567C007D007A5D
:10C4F000217B00123ED57404122B84122F2D90093B
:10C5000012E0600464017003122FDB90071112CB5C
:10C51000D1600612C63B122769122E9D1243E58098
:10C5200003122B847F0202280974F612258374FFFC
:10C53000122C187E007508327509057808122B56E2
:10C540007C6E7D007A217B00123EC97402122B841E
:10C55000E9600302C60C7808122B5675086E8E0926
:10C560007808122B567C007D007A217B00123EDB7E
:10C570007404122B84E9600302C60C900546E06443
:10C58000FE7003A3E0F4700302C60C0E900555E0A4
:10C5900064086005E06404706F851882851983EE75
:10C5A00012CA3779421249DF7A5D7B057943124915
:10C5B000DF7A5A7B0579471249DF7A4B7B05794A46
:10C5C0001249DF7A497B05794B1249DF7A537B05A3
:10C5D00079501249DF7A467B0579531249DF7A5B3D
:10C5E0007B0579541249DF7A487B0579E11249DFEE
:10C5F000900540E0A2E35004D2F08002C2F012CADB
:10C600002D79521249DF800412482F1E122F3390C9
:10C610000912E0600464017003122FED90071312F9
:10C62000CBD1600612C63B122769122EA9EEF9740F
:10C630000102C5218E828F83E0F8A3E0F583888212
:10C640002274F6122583E9FEA2E0502675083275A1
:10C6500009057808122B5675086E750900780812BE
:10C660002B567C007D007A217B00123ED57404128B
:10C670002B84EEA2E35003122F39900912E06004DC
:10C6800064017008EEA2E15003122FF3EEA2E25013
:10C690000E90071512CBD1600612C63B1227690215
:10C6A000C52474F612258374EC122C187401122B15
:10C6B000FA90103CE0F97AA37B051232FF900592C4
:10C6C000E06402707C7405122E2DE4F07407122EC3
:10C6D0002DE4F07A04F9122F878A089051C4E4936C
:10C6E000FAC3E5089AEB9400400302C777122F7B48
:10C6F000E9600302C7779051B712C7D360157A0477
:10C700007903122F879051C4E493FC9051B712C75C
:10C71000DD50087405122E2D7401F09051B512C72A
:10C72000D360157A027901122F879051C4E493FCEB
:10C730009051B512C7DD503F7407122E2D74018041
:10C740003590055E122E0AE8494A4B600474018058
:10C7500001E4C0E07405122E2DD0E0F090056212C5
:10C760002E0AE8494A4B600474018001E4C0E07479
:10C7700007122E2DD0E0F090103CE0F97CA37D054F
:10C780007401122BF21232F97AA37B057945124912
:10C79000DF7407122E2DE070117405122E2DE0703B
:10C7A00009851882851983E4800885188285198394
:10C7B0007401F0901038E0F8901037E058F88518C0
:10C7C00082851983E05812CA3779411249DF7414FF
:10C7D00002C521E493F8740193F9E84922E493F83F
:10C7E000740193F9ECC398F8E499F9C3EA98EB99CA
:10C7F0002274F712258374ED122C18E9FE90059F20
:10C80000F0AC18AD1990103CE0F97AA37B05123218
:10C81000FF7412122E2DEE12C82FAA18AB19123265
:10C82000F97AA37B0579451249DF741302B1A4F0AC
:10C8300090103CE0F97CA37D052274F4122583EA74
:10C84000FEEBFF90103EE064FE7003A3E0F470681E
:10C850007A167B00123DAF8A088B09EA45096058B9
:10C860008A828B83740112C8D88A828B83A3600466
:10C8700074028002740112C8F3A3E08A828B83A33E
:10C88000A3A3A3A3A3A3A3A312C909FCA3E0FDEA46
:10C890002402FAE43509FB124853E508241312C8B0
:10C8A000D0E4F0AA08AB099005A0E0F9123DBB1254
:10C8B000C8BB12D13C12C8ED0298B312C8BF22EE19
:10C8C000240BF582E43FF58322850A0CE508250C4C
:10C8D000F582E43509F5832212C8DDE022F08E826C
:10C8E0008F83A3A3A3A3A3A322E01297CDE8F0A371
:10C8F000E9F022F0EE241DF582E43FF58312C90130
:10C900002212D151F583888222A3F0EE241512B6AB
:10C91000782274F212258374FD122C188A088B0970
:10C92000890A8C0B7401122E2D740412CA3712342A
:10C930003D8A0C8B0DAE0CAF0DEE4F700302C9CECD
:10C94000EE12B7853F12C9FD7407F0A3A882A98330
:10C95000E5082413FAE43509FB8A828B8312CA0E98
:10C960008A828B8312CA0DE50812D37812DF1588EC
:10C9700082898312CA197401F0E508240BF8E435A2
:10C9800009F9EE12C9D912CA2612EE161233B912DB
:10C99000DA76EE241312EE187403650A6006740149
:10C9A000650A700712C9E97404800412C9E9E4F049
:10C9B00090103E12AD4F12C8ED7401650B7006EE7B
:10C9C000241112C9E0EEFAEFFB1230238002791035
:10C9D00090103E129BA402D15812EE6222EE241255
:10C9E000F582E43FF583E4F02212C9F17440F0A32C
:10C9F00022EE12DF073FF5832212EE3C3BF5831255
:10CA0000CA0322E0F8A3E0F98882898322A3E088A0
:10CA1000828983F0A308A98322F0EE2416F582E42C
:10CA20003FF58322A3A3E8F0A3E9F0EE22A2F0E40D
:10CA300033851882851983F0AA18AB192274F41271
:10CA40002583EAFEEBFF7A007B049005A0E0F91253
:10CA50003F2312CADB12C8ED9005557409F012335A
:10CA6000B98A088B09AC08AD0912CACD12D38B1252
:10CA7000484DE9640170537A0F7B00123DAF8A087C
:10CA80008B09EA450960438A828B837402F012CADB
:10CA9000E5FC88828983A3A3E0FBEC8A8285098375
:10CAA000A3A312DA8088828983A3A3A3E08A828564
:10CAB000098312C909FAA3E0FB794A1249DFAA08DF
:10CAC000AB099005A0E0F9123DBB0298B312CAD1A0
:10CAD00022EE2413F582E43FF5832290051812D14B
:10CAE0004C90109222EE241DF582E43FF58312CD86
:10CAF000B6E02274F412258374FD122C188A088B78
:10CB0000097401122E2D740212CA3712343D8A0A9A
:10CB10008B0BAE0AAF0BEE4F700302CBBD12EE8152
:10CB2000700888828983A37420F085088285098330
:10CB3000A3A3A3A3A3E06401700988828983A3E06F
:10CB4000D2E6F0850882850983A3A3A3A3A3A3E06B
:10CB50006401700A88828983A3E0D2E7800312ED22
:10CB6000F812EE727019850882850983A3A312CB8F
:10CB7000D16006EE241612EE1812EE5412C8ED859E
:10CB80000882850983A3A3A3A3A3A3A3E0640170E0
:10CB90000312EE2985088285098312D38B12345B38
:10CBA000E9600312EE2212EE151233B912CBD7123E
:10CBB000CBC312CA24FAEFFB123023800279100291
:10CBC000BC7FE0F8A3E0F98E828F832212B298F541
:10CBD0008312D14CE8492212CBE2EAF0A3EB12CB4C
:10CBE000EC22EE241AF582E43FF58322F0850882D8
:10CBF000850983E02274F512258374F3122C1889B9
:10CC00000AEAFEEBFF7508007509007C0D7D0079CE
:10CC100000AA18AB19123D97EE12D76C3FF583129C
:10CC2000CDA2741F58600C7AD37B00124433790074
:10CC300002CCF4E8A2E55008740C122E2D7401F019
:10CC4000E8A2E75008740B122E2D7401F0E8A2E65A
:10CC5000740A5008122E2D7401F08008122E2DE057
:10CC6000640170138E828F83A3A3A3A3A3A3A3E065
:10CC70006032EE241380128E828F83A3A3A3A3A31A
:10CC8000A3A3A3E0601EEE2415F582E43FF5831212
:10CC9000A7196010AC08AD097402122E2DAA82AB40
:10CCA0008312485312C8BB12C8E9740A122E2DE031
:10CCB0006401703712D37E12345BE97035EE240BB9
:10CCC00012B8FE900549E0687003A3E0697023E59F
:10CCD00008450960161233B9EAFCEBFD7402122E06
:10CCE0002DAA82AB8312484DE96007AA18AB19122E
:10CCF00030DDA90A02EF8974F712258374D2122C51
:10CD000018EAFEEBFF8E828F83129D45A2E040035E
:10CD100002CD9D12CDA9E054FE12E6D0740D122B67
:10CD2000FA12CDC61233B3E97073742A122E2D1283
:10CD3000CDC070697C0D7D007900AA18AB19123D39
:10CD4000977416122E2D12C8E9742A122E2D12CDA8
:10CD5000A2A2E55008740B122E2D7401F0E8A2E790
:10CD60005008740A122E2D7401F0E8A2E6500474E3
:10CD70002080027422122E2D12B0AC7402122E2DBD
:10CD8000AA82AB831248538E828F83A3A3E0C0E0B4
:10CD9000740C122E2DD0E012CA371230D7742E0226
:10CDA000B1A412C901A3E0F8228E828F8312CDB6FE
:10CDB000A3A3A3A3A32212D151F988828983A3221A
:10CDC00012B277640422EA241EF582E43BF583E084
:10CDD000F9EA241FF582E43B1298A722E9F87900CA
:10CDE000740468600A740A68600574036870010955
:10CDF000022B3674F61225838A828B837420F0A36B
:10CE0000A37401F01230298A088B09AE08AF09EE2D
:10CE10004F60168E828F837401F0900593E0700945
:10CE200012EE151233B912DA76EEFAEFFB02C524D0
:10CE3000C082C08390054302AA5CC082C083901068
:10CE40003D02AA5CC082C083E990103D02AAC1C025
:10CE500082C0839005B87401F0E9A2E35003740323
:10CE6000F0E9A2E15004E0D2E2F002C1B074F6129F
:10CE7000258379007C008A088B09780812284FF8EE
:10CE8000FF079ECE9CCE9CCE9CCE9CCE94CE98CEC0
:10CE90009ECE99CE7C0480060C0C80027C08900506
:10CEA000B8E05C6003098003EC60010902C52474EA
:10CEB000F4122583EAFEEBFF8908122FB18A0A8B50
:10CEC0000BA80AA90BE849604188828983A3A3A320
:10CED000A3E06036C39405503174016508601A8878
:10CEE000828983A3A3A3A3E06401600D8882898360
:10CEF000A3A3A3A3E06402700A8882898312A7F621
:10CF0000122769EEFAEFFB122FBD0298B374F612E6
:10CF100025838A828B83E07012A312CBD1600C8AA6
:10CF2000828B8312D38A124B7D80047A007B0002AD
:10CF3000C524C082C083900592E06402700B900506
:10CF400055E06408700312347F02C1B0C082C08310
:10CF50007C00EC12CFFF7003A3E06B70119051C7FF
:10CF6000E493C0E012CFCED0E0F079C580510CEC54
:10CF7000C3940340DD7C00EC75F003A4F8A9F074C1
:10CF8000BC28F582740512979064FE7003A3E0F448
:10CF9000600F0CECC3940340DE7C00EC12CFC27037
:10CFA00015EC12E36912DA7F9051C7E49388828905
:10CFB00083F0790080090CECC3940340DE79C7024A
:10CFC000C1B075F003A4F8A9F012CFCEE02274BB73
:10CFD00028F582740539F58322C082C0837D00ED77
:10CFE00012CFFF7003A3E06B700912CFC960047900
:10CFF0000180090DEDC3940340E5790002C1B075CD
:10D00000F003A4F8A9F074BC28F582740512E82294
:10D010006A2274F212258374DD122C18EAFEEBFFEB
:10D02000750A00900912E060076401600302D136BE
:10D03000900546E06E7003A3E06F701EEE4F700324
:10D0400002D12A9005CD12CBD1700302D12A750AE4
:10D050000112C63B12276902D136122FAB8A088B08
:10D0600009EA4509700302D12A8A828B83A3A3A30C
:10D07000A3E0640160108A828B83A3A3A3A3E0646E
:10D0800002600302D12A851882851983E412D143F4
:10D09000740B122E2DE8F0A3E912CA37122F6FE994
:10D0A000700302D12A85088285098312D13C12C8F7
:10D0B000ED790012318B85088285098312DA7F743D
:10D0C00003122E2DAC82AD837418122E2DAA82ABC2
:10D0D0008312485385088285098312B9047420128B
:10D0E0002E2D12C8ED7422122E2DE4F07C0285083C
:10D0F00082850983A3A3A3A3E0F9740D122BF21276
:10D10000341985088285098312B9047401122E2D01
:10D11000E8F0A3E912CA37122F75750A01E5082451
:10D120000C12C8D01297F1F0800C90055312B696ED
:10D13000FAEFFB123533A90A7423801E12D14C90EA
:10D14000103E2212AEDF12D14A22A3A312D151F90E
:10D1500022E0F8A3E022A90A7403122B847F0602BE
:10D160002809C082C08374FE122C18900912E06056
:10D170000464017029790190052B12C638122769C1
:10D1800012D1A3900546E8F0A3E912CA37795312E9
:10D1900049DF85188285198312D38B12405574029A
:10D1A0000284F7851882851983EAF0A3EB12D1B2C5
:10D1B000F92212BC9EF8A3E02274F512258374F3C1
:10D1C000122C188A088B09ECFEEDFF750A12EA454D
:10D1D000097005790002D2C6900546E06508700422
:10D1E000A3E0650970191233B9EAFCEBFDEEFAEF22
:10D1F000FB12484DE97005750A018003750A008528
:10D200001882851983E4F004122E2DE508F0A3E5B9
:10D210000912CA37122F63E960297403122E2DAA4E
:10D2200082AB83122F45E964017018750A017403FB
:10D23000122E2DAC82AD83EEFAEFFB12484DE97051
:10D240001E801F7412650A7019900592E0640270C6
:10D2500011EEFCEFFDAA08AB09122F93E9600375EC
:10D260000A00EEFCEFFDAA08AB09123551E9F8748B
:10D270000A687005750A01804274A0687037EEFC78
:10D28000EFFDAA08AB091235637E008023EE75F02E
:10D2900017A4F8A9F012E8387004A3E06509700F2C
:10D2A00012E974122F45E9700612E51312353F0E8C
:10D2B00012D2C940D87401650A70097900AA08AB76
:10D2C00009123491A90A02EF899051BFE493F8EE54
:10D2D000C3982274F6122583EAFEEBFF89089009B1
:10D2E00012E060046401701E12347FE508F50978CD
:10D2F00009122B5A790DEEFCEFFD7AFC7BFF1234FC
:10D300009D7401122B8402C52474F7122583EAFE52
:10D31000EBFF8E828F83A3A3A3A3A3A3A3A3E060A9
:10D320001312D37012989A12348BE96401700512AB
:10D33000C8BB802D8E828F83A3A3A3A3A3A3A3E046
:10D34000602912CACD12D38FFAA3E0FB12348BE905
:10D35000640170178E828F83A3A3A3A3A3A3A3A3A7
:10D36000A312D38B12347379018002790002B1A722
:10D37000EE12D3783FF583222415F582E4228E82C3
:10D380008F83A3A3A3A3A3A3A3A3A31298A9221249
:10D39000D39BA3A3A3A3A3A3A3E02212B0B48E8222
:10D3A0008F83A3A32274F212258374FD122C188A92
:10D3B000088B09ECFEEDFF890B750A017401122E32
:10D3C0002D740412CA3712343DEA4B6047741112AF
:10D3D0002E2DE0601AEA2417F582E43BF583E4126F
:10D3E000DC2B8A828B83E0D2E7F012D417E4F012B0
:10D3F000C9F9740312D685EE88828983A3A3F0EF5E
:10D4000088828983A3A312AEDAA3A312F066123036
:10D4100023E9F50A02D156EA2414F582E43BF583A8
:10D420002274F0122583EAFEEBFF890A750B0112C4
:10D43000CAE5F50C88828983A3A3E0FA88828983F0
:10D4400012D55E12BBAC6404600A7AD37B0012442E
:10D450003302D559E50C122A1A0200026ED4030BCE
:10D460000ED5030CF5D40DCDD40E0ED50CD59009E8
:10D4700012E060076401600302D50E900540E0A24F
:10D48000E1400302D50E7900AB09123221EA4B606C
:10D49000318A828B83A3A3A3A3A3A3E054186022A1
:10D4A00012C8BB1229958A828B83A3A3122995796E
:10D4B000008E828F8312D57D1232397404122B8430
:10D4C000802E7901AA08AB091230EF804190091231
:10D4D000E0600464017037900540E0A2E1502FAB9A
:10D4E0000912346DAA08AB09123473E964C5701EC1
:10D4F000750B008019900912E060046401700F90B0
:10D500000540E0A2E150071240798002880AEE242B
:10D5100009F50EE43FF50FAC08AD09A90C850E82A4
:10D52000F58312D38B123107850E82850F8312D3B8
:10D530008B12345BE96022EE241112BBAFC394025C
:10D54000401712C8BB12DB457003A3E069600AE50F
:10D550000BA2E05004A90A8002790002C178A3A3BB
:10D56000A3E0F8E4C8F9EA28F508E439F50922E56A
:10D5700008240CF582E43509F58312B654A3A3A35D
:10D58000A3A3A3A3A3A312B0B08A828B831298A9EA
:10D590002274EE12258374F5122C188A0A8B0B89DB
:10D5A0000C8C0E8D0F7E01EE122E2D740AF0741D60
:10D5B000122E2DE0F50DE9700FE50DC333240AC0DE
:10D5C000E0EE122E2DD0E0F0AA18AB1912343D8AED
:10D5D000088B09EA4509700302D67A12B784350927
:10D5E00012D807740912D813450D12D6A5AC0EAD8A
:10D5F0000FEEFAEFFB124853EE2408FE50010FE540
:10D600000C70247C00741E122E2D12B9048012ECB2
:10D6100012DB31E82AFAE93BFB12D68BA30EAF836B
:10D620000CECC3950D40E8E508241712C8D074012E
:10D63000F01233B9E508241AF582E4350912DA7DCF
:10D640007403122BFAAA0AAB0B122F4BE96019E5EF
:10D6500008241612C8D07401F07403122BEAE508EE
:10D66000241812C8D012C8ED85088285098312D605
:10D6700081AA08AB09123023E9FEEEF9740B02BE51
:10D68000C2A3A3E50AF0A3E50BF0228A828B8312E2
:10D69000D69F12D6A58A828B8312D69EF022A3E053
:10D6A0008E828F8322F0A3AE82AF832274F0122584
:10D6B0008374F8122C188A088B0912D76B3509125B
:10D6C000D88CF50B880AA3AE82AF83EEFCEFFDAADF
:10D6D00018AB19124853EE2408FE50010FAC18ADD8
:10D6E000197A677B0512484DE9607474E0550A7039
:10D6F00067AA0BEA2AFA7B00123E518A0C8B0DEACC
:10D70000450D605B7C00801E8E828F8312C10EEC03
:10D7100012D764E50C28F582E50D3912DA7DEE2486
:10D7200002FE50010F0CECC3950B40DC780C122B61
:10D7300056780B122B5A7403122BFA7900E5082441
:10D740000B12C8D012D38B1234B57403122B84AAD7
:10D750000CAB0D123E5780077AD37B001244337412
:10D760000802C17525E0F8E433F922EA241DF582A8
:10D77000E42274F01225838A0A8B0B890C8C088DA5
:10D78000099007E412CBD1607B7410122E2DE0F5C6
:10D790000D12D764E8240EFAE439FB123DAF8A0E6D
:10D7A0008B0FAE0EAF0FEE4F605A8E828F8374D404
:10D7B000F0A3A3E50AF0A3E50B12BEB5E50CF0ACAF
:10D7C00008AD09EE2405FAE43FFB12485312B28B70
:10D7D000E50DF07411122E2D12DC157808122B5263
:10D7E000AC0DEC2CFCE433FDEE240EFAE43FFB120E
:10D7F0003D8B7403122B84EEFAEFFB9007E412C604
:10D800003812276902C178F583E0FEA3E0FF8E821B
:10D810008F8322F0A3E50CC43354E02274F6122562
:10D820008374F8122C18890812D76B3B12D88CF924
:10D830008809A3AE82AF837401697042EEFCEFFDEC
:10D84000AA18AB19124853EE2408FE50010FAC1869
:10D85000AD197A677B0512484DE9602974E05509D6
:10D86000701C8E828F83A3E0FA8E828F83A312C1F5
:10D87000108E828F83E0F91234CDA90880097AD303
:10D880007B001244337900740802C521F583E0243B
:10D8900001FEA3E03400FF8E828F83E0F8741F58EE
:10D8A0002274F612258374DF122C18EAFEEBFF12A5
:10D8B000CBCC60508E828F8312D38BAC18AD1912F3
:10D8C000CDC61233A17409122E2D12DB457003A3AD
:10D8D000E069603012C6341229957508FE7509FF9B
:10D8E0007808122B56741C122E2DE0F9740D122E8E
:10D8F0002D12B0AC740F122E2D12D38B123239743C
:10D9000004122B84742102C52174F7122583E9FCCB
:10D910007A007B007E00800B12D9ABE02AFAA3E0EC
:10D920003BFB0E9051C412D2CC5029EE75F016A4D8
:10D93000F8ADF0EDF912E827F460E7744328F582BA
:10D94000740A3912CBCF60DAEC60CD12D9ABE4F0B7
:10D95000A3F080CE7E00800B12D998E02AFAA3E0D3
:10D960003BFB0E12D2C9502DEE75F017A4F8ADF0A6
:10D97000EDF912E9857003A3E0F460E6741628F56A
:10D9800082740C3912CBCF60D9EC60CC12D998E4F8
:10D99000F0A3F080CD02B1A7EE75F017A4F8EDF971
:10D9A000741628F582740C39F58322EE75F016A4EE
:10D9B000F8EDF9744328F582740A39F5832274EC82
:10D9C000122583890CEAFEEBFF90059FE0C3950CBE
:10D9D000503B12340D9005CF12DA70900539E0F506
:10D9E00008E4F509F50AF50B9081007810122DD6A0
:10D9F0007808791012241E7808122B4E7A007B02C8
:10DA00009005A0E0F9123F177404122B8402978846
:10DA100074F6122583EAFEEBFF9005B98013888225
:10DA20008983E06E7003A3E06F603688828983A3E8
:10DA3000A312CBD170E87A047B00123E518A088B86
:10DA400009A808A909E84960188882898312DA7050
:10DA50009005B912DA64A3A312DA7F9005B912C84F
:10DA6000ED02C5241298A988828983228A828B8339
:10DA7000EEF0A3EFF022EE241AF582E43FF583EAFC
:10DA8000F0A3EBF02274F41225837E009005B98098
:10DA9000070E88828983A3A312CBD170F4EE12DB28
:10DAA00031123E518A088B09EA4509607E7F009059
:10DAB00005B980218882898312B0ACEF12DB31E591
:10DAC000082AF582E5093BF583ECF0A3EDF00F8819
:10DAD000828983A3A312CBD170DA90059B12DB4518
:10DAE0007003A3E0697808701C122B56EEF50A78D3
:10DAF0000A122B5A7C677D05790090059B12D38B07
:10DB00001234B5801A122B56EEF50A780A122B5AE7
:10DB10007C677D05790090059B12D38B1234A97424
:10DB200003122B84AA08AB09123E5712303B02980D
:10DB3000B325E0FAE433FB228E828F83A3A3A3A351
:10DB4000A3A3A3A3A312D14C900546E06822C082F0
:10DB5000C08380128A828B83A3A312B9049005B973
:10DB600012C8ED123E579005B912B04F70E602C1CF
:10DB7000B074F512258390055312B90B9005CF129E
:10DB8000DC0912C8ED7ACF7B0579501249DF900588
:10DB9000CF12DC15801512E3C765087004A3E06599
:10DBA00009600612E51B12353F050A12DBFE50180C
:10DBB000E50A12E5077003A3E06F70DA740B28F52D
:10DBC00082740C12F06380E19005CF12B90B9007BC
:10DBD000E612CBD160257A067B00123DAFEA4B609E
:10DBE0001A8A828B8374D5F0A3A3E412DC1C04127E
:10DBF000DC2B9007E612C63812276902EF8E90518F
:10DC0000BFE493F8E50AC3982212DC0D2212D15129
:10DC1000F99005532212AD36750A002212DC20223B
:10DC200012DC242212AEDFA3A3A32212DC20A3EE77
:10DC3000F0A3EFF022C082C0839005D174F7F0A367
:10DC40007434F09005D374F1F0A37434F09005D5DA
:10DC5000740FF0A3743502AAC1C082C08390054638
:10DC6000E064FE7003A3E0F4600E900540E0A2E1E2
:10DC700050061235571234FD02C1B074F0122583DC
:10DC8000900594E06053F50CE4F50DF50EF50F905A
:10DC900080F87808122DD6780C790812241E123DCF
:10DCA000A98A088B09A808A9099051B1E49358F5ED
:10DCB00008A3E49359F509E4F50AF50B780C790803
:10DCC000122D0B780C122B4E7A007B019005A0E0F0
:10DCD000F9123F1D7404122B8402C17874EE1225D0
:10DCE000837E007F008E0A8E0B122FFF8E0D803EEA
:10DCF000850D08AA087B00122FF98A088B09A8084D
:10DD0000A909E849602688828983A3A3A3A3E060C8
:10DD1000046404701788828983A3A3A3A3A3A3A385
:10DD2000A3A3A3E0F9123569E960010F050D905135
:10DD3000C4E493F8E50DC39840B612352D8A0E8BD6
:10DD40000F8E0C8023AA087B001235398A088B09B4
:10DD5000A808A909E849600EE8240F12978DF91266
:10DD60003569E960010E050C850C08C3E508950EC0
:10DD7000E4950F40D0EF2EFE700302DE758E08751D
:10DD8000090074027808122D44AA08AB09123E510A
:10DD90008A0A8B0BEA450B700302DE73750C008E4A
:10DDA0000875090074027808122D44AC08AD097991
:10DDB000FF123D97750D00805D850D08AA087B0058
:10DDC000122FF98A088B09EA450960488A828B83F9
:10DDD000A3A3A3A3E06004640470398A828B83A3A5
:10DDE000A3A3A3A3A3A3A3A3A3E0F9123569E960A6
:10DDF00023050C780A122B56EEFD850882850983CF
:10DE0000A3A3A3A3A3A3A3A3A312DF1B123503748D
:10DE100002122B84050D9051C4E493F8E50DC398CC
:10DE20005006E50CC39F4091750C00850C08C3E5B6
:10DE300008950EE4950F503DAA087B001235398AEB
:10DE4000088B09EA45096027EA12DF0712DF15F996
:10DE5000123569E96019780A122B56EEFDE508249F
:10DE60000E12C8D012DF1B1235037402122B840568
:10DE70000C80B87E00750E6290053EE0600CF912D1
:10DE80002F03E9F87454C398F50E75F003E50E847A
:10DE9000F50D94204003750D1F850A08850B097543
:10DEA0000C00E50E6006750C20750E00E50DC39E96
:10DEB0005004AF0D8008EEFFE50CD2E6F50CAC087F
:10DEC000AD09AA0CEFF9123509E9F50FE50CA2E648
:10DED000401A1F7800800BE5082404F5085002055D
:10DEE0000908E8C39F40F0EFCEC39EFEE97006E547
:10DEF0000CA2E650AAE50A450B6007AA0AAB0B1272
:10DF00003E57A90F02BEC5240FF582E422749E2558
:10DF100008F582740F3509F583E022E0FC8508825C
:10DF20008509831298A92274F2122583EAFEEBFF79
:10DF300089088C098D0A7C007D00740E122E2D122A
:10DF4000D38B8C0B800DEAFCEBFDEA2404FA500124
:10DF50000B050BE50BC3950A400302DFF28A828BA7
:10DF600083E0F47003A3E0F46077EC4D600C8C82E6
:10DF70008D83C3E09EA3E09F50CC8A828B8312E303
:10DF800036EE98EF9950BFEAF8EBF988828983E082
:10DF9000F47003A3E0F46010E82404F850010905CC
:10DFA0000BE50BC3950A40E3E8FCE9FDE824FCF827
:10DFB000E934FFF9888289831297E28C828D83E5A8
:10DFC0000CF0A3E50D12DFF58C828D83A3A312E67E
:10DFD000CAE08C828D83A3A3A3F0C3EA98EB994097
:10DFE000C712DA6C8A828B83A3A3E50912DC1CE5D5
:10DFF00008F002D15D12DFFBA3E022F08882898362
:10E00000A32274F212258374FD122C1889088A0940
:10E01000ECFEEDFF750A0175F003E9A42402C0E0EF
:10E020007401122E2DD0E012CA3712343DEA4B6033
:10E030007812C9F97408F0741F55084509A3F0E86F
:10E040002402F8500109750A0080388E828F83E01F
:10E0500088828983F0A3A882A9838E828F8312CAC3
:10E060000D8E828F83A3A3E05407C4FC8E828F831E
:10E07000A3A3A3E054074C12CA0FEE2404FE5001E0
:10E080000F050AE50AC3950840C18A828B83A3A3C2
:10E0900074FCF0A374FFF0EA2413F582E43BF583EB
:10E0A0007401F0123023E9F50A02D15674F11225F9
:10E0B000838A0A8B0B7508007AFE7BFF7CFE7DFF4E
:10E0C000E50A12D76C350B12CAECF509741F550915
:10E0D000F50CE82402F8500109E509A2E7406FE5D4
:10E0E0000A2417F582E412E2A6FE75F003E50CA4FB
:10E0F00024026E7059E50C600B88828983E0FEA3D0
:10E10000E0FBEEFA750D00801DE05407F50EA3A8A4
:10E1100082A983EEFC900546E06E7003A3E06F7069
:10E1200003850E08050DE50DC3950C502B888289DB
:10E1300083E0FEA3E0FCE4CCFDEE2CE43DFFE8240C
:10E1400002F850010988828983E0548860BB7AD341
:10E150007B0012443302E29BE508700BA9091235DB
:10E1600015E9700302E29B12E2B812D38B122FABB7
:10E170008A0C8B0DAE0CAF0DEE4F605A8E828F83E2
:10E18000A3A3A3A3A3A3A3E4F09051D793F88E82F3
:10E190008F83A3A3A3A3A3A3A3A3E0C398402412A4
:10E1A000E2C25001097A027B00122326E88E828F98
:10E1B00083A3A3A3A3A3A3A3A3F0E508C394075039
:10E1C0000205088E828F83A3A3A3A3A3A3A3A3A363
:10E1D000E508F002E29B7CFF7DFF12E2B812D38BD0
:10E1E0001235218A0C8B0DAE0CAF0DEE4F704F1215
:10E1F00035278A0C8B0DAE0CAF0DEE4F700302E28B
:10E200009B7C177D007900123D9712E2B812CBC2B9
:10E210001284E98E828F83A3A3A3A3A3A3A3A31233
:10E22000CA2412B66D74AA12E2E15001097A027B87
:10E230000012232612B28BE812E2CD7401F0905145
:10E24000D7E493F8EE240D12BBAFC398401912E245
:10E25000C25001097A027B0012232612E2ACE508C3
:10E26000C394075002050812E933E50812E2D2E42C
:10E27000F0129CDA122F45E97021850A82850B8302
:10E28000A3A3A3A3A3A3A3A3E06010E50A12D378DA
:10E29000350B12B694129CDB12485302A8D7749E19
:10E2A000250AF582740F350BF583E022EE240DF577
:10E2B00082E43FF583E8F022E50A12EE3D350BF5E6
:10E2C00083229051D7E49379002401F822F012E9D7
:10E2D0003722F012E2D722EE240CF582E43FF583D8
:10E2E00022F09051D7E49379002401F82274F712B8
:10E2F0002583E9FE74FE6A700374FF6B60347460FA
:10E300005E6460602DEEA2E5401CA2E690054650DA
:10E310000DC3E09AA3E09B5019790002B1A7C3E0B6
:10E320009AA3E09B40F390054612E336EC98ED99F2
:10E3300040E7790180E512D14CC32274F71225839E
:10E340007E00800712E51312353F0E12D2C940F449
:10E350007E00EE12E369129BA488828983E4F00EAA
:10E36000EEC3940340EC02B1A775F003A4F8A9F042
:10E3700074BB28F8740539F988828983A32274F75D
:10E380001225837F0080010F9051BFE493F8EFC303
:10E3900098502DEF75F017A4F8A9F012E8136A70E1
:10E3A00003A3E06B70E112E3C76C7003A3E06D6040
:10E3B0000A74FF6C700374FF6D70CC12E51B80044F
:10E3C0007A007B0002B1A712E3CB22740B28F582FE
:10E3D000740C12E8222274F61225837CFF7DFF7AEA
:10E3E000FE7BFF123521EA4B703C7508008032E558
:10E3F0000875F017A4F8A9F0741028F582740C12AF
:10E400009790600512E8087016740128FE740C39A4
:10E41000FF8E828F8312D38B12323FEEFAEFFB0511
:10E420000812E42940C902C5249051BFE493F8E5DD
:10E4300008C39822C082C0837A007B007D008010D0
:10E4400012E97D7003A3E0F460050AEA70010B0D88
:10E450009051BFE493F8EDC39840E502C1B074F465
:10E460001225838A088B09ECFEEDFF800B12353FE5
:10E47000EEFCEFFDAA08AB09123521EA4B70EE0263
:10E4800098B374F61225837D007E0080020D0E1273
:10E49000D2C95018EE12E97E7003A3E0F460EF8D4C
:10E4A00008EA65084B70E612E51B80047A007B00E1
:10E4B00002C52474F7122583EAFEEBFFEE4F601AC3
:10E4C0007C177D007900123D978E828F8374FEF059
:10E4D000A30412AD59A314129BA602B1A774F7129C
:10E4E0002583EAFEEBFF7508008014E50812E507B6
:10E4F0007003A3E06F600612E51B12353F0508129A
:10E50000E42940E702B1A775F017A4F8A9F012E3D7
:10E51000CB6E22EE75F017A4F8A9F0740128FA74F6
:10E520000C39FB2274F41225838A088B09ECFEED6A
:10E53000FF900912E0600464017020900553E06EC2
:10E540007003A3E06F7014122FAB8A0A8B0BA80A1A
:10E55000A90BE8496005E82408801AEEFCEFFDAA43
:10E5600008AB091235218A088B09A808A909E849CE
:10E570006009E8240DFAE439FB80047A007B00028C
:10E5800098B374F41225838A0A8B0BECFEEDFF75A9
:10E5900008007509008034E50912E96D122F45E97C
:10E5A0006027E50975F017A4F8A9F012E8327004A5
:10E5B000A3E0650B700375080AEEFCEFFD12E97429
:10E5C00012484DE960034308A005099051BFE49348
:10E5D000F8E509C3985004E50860BC02BF4574F62D
:10E5E0001225837E00805C8E08AA087B00122FF91A
:10E5F0008A088B09A808A909E849604688828983A6
:10E60000A3A3A3A3E06401603988828983A3A3A3A1
:10E61000A3E06402602CE8240712978DFA74012AA3
:10E62000F0900595E0C39A501988828983A3A3A32B
:10E63000A3A3A3A3A3A3A3E412E6C1A312E6D0124B
:10E64000323F0E9051C412D2CC409C7E008059EED5
:10E6500075F017A4F8AAF0EAF912E9857003A3E0AF
:10E66000F46044740128F8740C39F9E8240C12970A
:10E670008DF8740128F0900595E0C3985029EE7547
:10E68000F017A4F8EAF9740128F8740C39F9E812C3
:10E69000DF0739F583E4F0E8240EF582E439F583E9
:10E6A000E412E6D012323F0E12D2C940A27B00EB38
:10E6B00012CFC2600214F00BEBC3940340F102C509
:10E6C0002412E6CAA3A3A3A3A32212DFFBA3A322BF
:10E6D00012E6D8FAA3E0FB22F088828983E0227454
:10E6E000F31225838A088B09ECFEEDFF750C007B85
:10E6F000007C01740D122E2DE0F50AA3E0F50B80CD
:10E7000010123DA9E50CF5F0EA84ABF0750C007C25
:10E71000007D0080010D9051BFE493F8EDC3985047
:10E720004912E97D7003A3E0F460EA12E83870044E
:10E73000A3E0650960DF12E8136E7003A3E06F6069
:10E74000D412E8327004A3E0650B60C912E80860D7
:10E75000C4C3940750BFEC050C70BAE50CC39B40D2
:10E76000B4740128F582740C80787A0080010A90D4
:10E7700051C4E493F8EAC3985070EA75F016A4F80F
:10E78000A9F012E83E64FE7003A3E0F460E012E832
:10E790003E65087004A3E0650960D312E83E6E7020
:10E7A00003A3E06F60C812E83E650A7004A3E06549
:10E7B0000B60BB743C28F582740A12979060AFC35B
:10E7C000940750AA12E827640160A3E06402609EE7
:10E7D000EC050C7099E50CC39B4093743328F582CB
:10E7E000740A39F58312D38B8019E50C6011EB7034
:10E7F0000E7401650C600302E7017B0102E70C7AED
:10E80000FE7BFF7F05022809740F28F582740C1225
:10E81000E8222212E81722740128F582740C12E80B
:10E82000222239F583E022743728F582740A12E82F
:10E83000222212E817650A2212E8176508227433AB
:10E8400028F582740A12E8222274F51225838A08B8
:10E850008B09ECFEEDFF750A008002050A12DBFE53
:10E860005022EEFCEFFDE50A12E96D12484DE96019
:10E87000EAE50A75F017A4F8A9F0740128F5827486
:10E880000C12F06302EF8EE9F87907C3940D40048F
:10E8900079018019E8C3940740047903800FE8C325
:10E8A0009403400419198005E870027900022B36A0
:10E8B00074F01225838A088B098C0A8D0B890C123F
:10E8C00035278A0E8B0FAE0EAF0FEE4F60627C17AE
:10E8D0007D007900123D978E828F8312F0668E82C2
:10E8E0008F83A3A3A3A3A3A3A3A312D681E50C6044
:10E8F0000712B66CE50C800512B66C7401F0900539
:10E90000D312CBD1601590059AE06401700612E92C
:10E9100033E4800C12E9337407800512E933740183
:10E9200012E2E15001097A027B0012232612E2ACC6
:10E9300002C17812E93722EE240EF582E43FF58316
:10E940002274F71225837E00801BEE12E97E70038D
:10E95000A3E0F4600F12E974122F45E9700612E586
:10E960001312353F0E12D2C940E002B1A775F0175D
:10E97000A4F8A9F0740328FA740C39FB22ED75F0A1
:10E9800017A4F8A9F012E81764FE22C082C0839091
:10E9900005D77481F0A37435F09005D97487F0A37E
:10E9A0007435F09005DB748DF0A3743502AAC17440
:10E9B000F7122583EAF8EBF990051612E9F8CA2454
:10E9C00006F582E43AF583E0702B88828983A3A35D
:10E9D000A3A3A3A3A3A3A312299590051612E9FD4F
:10E9E000122DFE88828983A3E0F91230FB74021293
:10E9F0002B8412303B02B1A7E0FAA3E02212E9F81F
:10EA0000F5838A8222C082C08390059D12EAC8F0F5
:10EA100090059D12CBD1700579011234C702C1B0A7
:10EA200074F612258374FC122C18E9FE9051C8E488
:10EA300093700874E16E600302EAC3EA2408F8E404
:10EA40003BF98882898312EAC812EAD1700E9005D8
:10EA50009DE4F0A3F079011234C78067900914E0B7
:10EA60006061FA90059D12E336EA98E49950547972
:10EA7000001234C78A088B09AC08AD09ECF8EDF92F
:10EA8000E875F064A4F8AAF075F064E9A42AF99096
:10EA9000059D12D38B12232EE8941AE9940040238B
:10EAA0009007DE12CBD1601B90059D12C8E974025D
:10EAB000122E2DECF0A3ED12CA379007DE12C638E5
:10EAC000122769740402C521E02401F0A3E0340098
:10EAD0002212E6D8F8A3E0F9E84922C082C0837484
:10EAE000F8122C1890809AAC18AD197408122AB23A
:10EAF000AC18AD1912484DE9640170047900800228
:10EB000079010284F574F6122583740C122E2D12ED
:10EB1000B90B743A6E7001EF6006743B6E4F702350
:10EB2000740A122E2D1229958C088D097808122B43
:10EB300056EAFCEBFDEEFAEFFB123EDB7404122BFF
:10EB4000848002790A02C524C082C0839005DD74E6
:10EB500005F0A37430F09005DF740BF0A37430F06F
:10EB60009005E174ABF0A37435F09005E374B1F057
:10EB7000A37435F09005E574B7F0A37435F09005F3
:10EB8000E774BDF0A37435F09005E974C3F0A37485
:10EB900035F074AB443560031235AB02C1B074F488
:10EBA00012258374E9122C188A088B097404122E1A
:10EBB0002D7402F004122BF212343D8A0A8B0BAE34
:10EBC0000AAF0BEE4F700302EDE412EE817008887D
:10EBD000828983A37420F0850882850983A3A3A377
:10EBE000A3A3E06401700988828983A3E0D2E6F0E0
:10EBF000850882850983A3A3A3A3A3A3E06401706E
:10EC00000A88828983A3E0D2E7800312EDF812EE2E
:10EC1000727019850882850983A3A312CBD160067F
:10EC2000EE241612EE1812EE5412C8ED85088285F5
:10EC30000983A3A3A3A3A3A3A3E06401700312EE1B
:10EC40002985088285098312D38B12345BE960031E
:10EC500012EE2212EE151233B912CBD7FAA3E0FB53
:10EC60008E828F83A3A312DA7F12345BE9600312D2
:10EC7000C9DDEE241312BBAF700D9051CCE493C0EC
:10EC8000E012CACDD0E0F08E828F83E0A2E750047C
:10EC900054038019EE241412BBAF7012900532E0B9
:10ECA000C0E012EDEED0E0F0900532E004F012EE9C
:10ECB00007701990109FE0600D90053DE0700D8E7B
:10ECC000828F83E07006EE241112C9E0AC18AD19F2
:10ECD000EEFAEFFB1233958A088B09EA45097003B7
:10ECE00002EDD87A217B00123E517406122E2D12AD
:10ECF000DA7F7406122E2D12CBD1700302EDCC9068
:10ED00000912E060046401700812B66CA3E04404C8
:10ED1000F07401122BF279501249D97401122E2D80
:10ED200012B9047406122E2D12E9F8CA2409F582CC
:10ED3000E43AF58312C8ED90054612B90474151231
:10ED40002E2D12C8ED7406122E2D12B8F612EE33C7
:10ED5000F07406122E2D12AE2B740212EE6B740696
:10ED6000122E2D12E9FD12BC92C0E07406122E2D57
:10ED700012B8F612EDFED0E0F0EE240E12EE10C046
:10ED8000E07406122E2D12EE43D0E0F07406122E1F
:10ED90002D12867812F064EE240F12B8FE740C1255
:10EDA0002E2D12C8ED8A828B83E0C0E0740E122EE5
:10EDB0002DD0E0F07406122BF2123311E9F50A742B
:10EDC00006122E2D12D38B123E578003750A10AAFD
:10EDD00008AB09123E578003750A10EEFAEFFB12DA
:10EDE0003E578003750A10A90A74170298B0EE24E2
:10EDF00014F582E43FF5832212CAD1740122241E45
:10EE0000F582E438F58322EE241112B678640122EB
:10EE100012B65FE022EE2417F582E43FF583740119
:10EE2000F02212B6754404F02212C9F17401F0A365
:10EE3000E4F02212EE3D38F583740222EA240BF549
:10EE400082E42212EE472212D151C8240CF582E44A
:10EE500038F5832285088285098312D14AEE12EEA5
:10EE600062222418F582E43FF5832212B6AE12D155
:10EE70004B2212EE79E064012212EE9AA3A3A3A31F
:10EE80002212C8BF12CA037404F0A3E412EE96A3C0
:10EE9000A3A3E064012212EE9A22F085088285097C
:10EEA00083A32274F61225837E00801F7C047D00DC
:10EEB00079FF8E088D0974027808122D44749E25FE
:10EEC00008FA740F3509FB123D970E9051CE12D2FD
:10EED000CC40D902C52474F512258374F7122C187E
:10EEE000750A00801E850A087509007402780812E8
:10EEF0002D4474A02508F582740F12C8D312EF7C3C
:10EF0000F0050A9051CE12DC01506D850A08750992
:10EF10000074027808122D4412DF0DF47003A3E090
:10EF2000F460DE850A0875090074027808122D4421
:10EF300074A02508F582740F350912CBCF70A67422
:10EF400008122E2D7402F0850A087509007808123F
:10EF50002D44749E2508FE740F3509FF8E828F8321
:10EF600012C8E912EF85124A277C047D0079FFEE72
:10EF7000FAEFFB123D9780897409800FE024FFF0BF
:10EF8000A3E034FF2212F0F322740D122B847F03CE
:10EF900002280974F012258374F7122C18EAFEEB8C
:10EFA000FF8C088D09750CFF7408122E2D12F0E5E8
:10EFB000124A21E9641A700302F05F750E00800B9B
:10EFC00074FF650C7003850E0C050E9051CEE49312
:10EFD000F8E50EC3985048850E0A750B0074027848
:10EFE0000A122D4412E29EF47003A3E0F460D1856E
:10EFF0000E0A750B007402780A122D4412E29E6EFE
:10F000007003A3E06F70C2750F007402780E122DAA
:10F010004474A0250EF582740F350FF5838030E41B
:10F0200093650E702D74FF650C602E850C0A750BB0
:10F03000007402780A122D44749E250AF8740F3564
:10F040000BF98882898312DA7088828983A3A312DC
:10F05000F0667901740902C17512EF85124A2779A9
:10F060000080F139F583E508F0A3E509F02274F496
:10F0700012258374F7122C18EAFEEBFF7408122E87
:10F080002D12F0E5124A27750A008002050A9051F8
:10F09000CE12DC01504C850A08750900740278080C
:10F0A000122D4412DF0DF47003A3E0F460DE850A34
:10F0B0000875090074027808122D4412DF0D6E7075
:10F0C00003A3E06F70C67C047D0079FF8D0B740292
:10F0D000780A122D44749E250AFA740F350BFB1220
:10F0E0003D9702AE1B740212A528EEF0A3EFF012BA
:10F0F000F0F32290055312B0B4AA18AB1922C082C3
:10F10000C08374F8122C1885188285198312DA7F4F
:10F110007402122E2DE4F0A3F07404122E2D74014B
:10F12000F07405122E2D7401F07406122E2DE4F0E9
:10F130007407122E2DE412CA371235A50284F57415
:10F14000EE1225838A088B09ECFEEDFF750C00EEAC
:10F1500065087003EF6509600C123ECF8A0A8B0BBD
:10F16000EA450B7006750C0102F1FBEEFAEFFB129B
:10F170003ECF8A0E8B0FAC0EAD0FEC4D6007EEFA52
:10F18000EFFB123EE1E4F50EF50F780E122B56ACB4
:10F190000AAD0BEEFAEFFB123EC97402122B84E9A2
:10F1A0006059AA0AAB0B123E518A0E8B0FEA450F2B
:10F1B0006046780E122B56780A122B567C007D0082
:10F1C000AA08AB09123EDB7404122B84E9701D7887
:10F1D0000E122B56780A122B567C007D00EEFAEFA9
:10F1E000FB123ED57404122B84E96003750C01AA4E
:10F1F0000EAB0F123E578003750C10A90C02BEC552
:10F2000074F612258312F4439051D2E493F508EC7E
:10F210008508F0A4FCA8F08508F0EDA428FD79FF8E
:10F220007AB27B0F123D9790070974C5F0A3743929
:10F23000F090070B74BFF0A37439F090070D74E9D8
:10F24000F0A37439F090070F7401F0A3743AF090B2
:10F2500007117407F0A3743AF09007137419F0A320
:10F26000743AF0900715741FF0A3743AF0900708F1
:10F27000E4F08003122B847F02022809C082C0833D
:10F280007B0080010B9051D2E493F8EBC398500BB4
:10F29000EB12F2D470EE12F6F380047A007B0002D7
:10F2A000F856C082C0837A007B007D008018ED1282
:10F2B000F2D4601174B728F582740F12F718F8EAC7
:10F2C00028FAE43BFB0D9051D2E493F8EDC398404B
:10F2D000DD02F85612F706F42274EC122583890F2A
:10F2E0008A0A8B0B8C108D087E007F00123A37AA99
:10F2F0000AAB0B123A3D8A0C8B0D850A82850B8373
:10F30000A3A3A3A3A3A3A3A3E064017007750E01A5
:10F310008E0980058E0E85100974FE650C700474CC
:10F32000FF650D700302F40E7B007414122E2DE0A5
:10F33000F50AA3E0F50B80010B9051D2E493F8EBB2
:10F34000C3985059EB12F702650F70EC12F6E465A2
:10F350000E70E512F82B650C7004A3E0650D70D8F3
:10F3600074B628F582740F12F718650970CA74B262
:10F3700028FE740F39FF750C00E50CC39508400397
:10F3800002F40E12F4171239D1E9700D12F41712AB
:10F3900039DDE970047E007F00050C80DC1239B98C
:10F3A0008A128B13AE12AF13EE4F60628E828F8380
:10F3B000E50FF0A3E50EF08E828F83A3A3E50CF09A
:10F3C000A3E50DF08E828F83A3A3A3A3E509F0909C
:10F3D00051D3E493C395085004E493F5088E828FCB
:10F3E00083A3A3A3A3A3E508F0850A0C850B0D75E1
:10F3F0000E00780C122B52AC08EC2CFCE433FDEE22
:10F400002406FAE43FFB123D8B7403122B84EEFAC0
:10F41000EFFB7F0C022809A80CE828F8E433F9E593
:10F420000A28F582E50B12F718FCA3E0FDEEFAEFCF
:10F43000FB22C082C08312F44379FF123D97790109
:10F4400002F8569051B9E493FC740193FD2274F7CD
:10F45000122583EA4B60377E0080010E8A828B83FF
:10F46000A3A3A3A3A3E0F8EEC3985022EE25E0F8EF
:10F47000E433F9EA28F582EB39F583A3A3A3A3A328
:10F48000A3E06C7003A3E06D70D179018002790074
:10F4900002F56774F5122583EA4B607B8A828B83C1
:10F4A000A3A3A3A3A3E0606FEA2406F8E43BF98AD0
:10F4B000828B83A3A3A3A3A3E0F509750800800FA3
:10F4C000EA2405F582E412F64B14F0604A0508E5DB
:10F4D00008C395095031AE08EE2EFEE433FF12F555
:10F4E0001E6C7003A3E06D60D7AE08EE2EFE12F521
:10F4F0001EFEA3E0FF88828983EEF0A3EFF0E824EC
:10F5000002F850C90980C68A828B83A3A3A3A3A350
:10F51000E060047901800279007F0302280912F576
:10F520006CE02274F7122583EA4B60399051D3E4E2
:10F5300093F88A828B83A3A3A3A3A3E0C398502547
:10F54000EA2405F8E43BF988828983E025E0FEE4BB
:10F5500033FF12F56CECF0A3EDF088828983E004B0
:10F56000F07901800279007F01022809EA2EF582F4
:10F57000EB3FF583A3A3A3A3A3A32274F4122583D3
:10F580008908EAFEEBFF8C098E828F83A3A3A3A3D5
:10F59000A3A3A3A3E0640170098E828F8312FEB13E
:10F5A000800B123A258A0A8B0BA80AA90B74FE68F5
:10F5B000700374FF69700302F63D7D00801A12F635
:10F5C000446401701274B42AF582740F12F64B6809
:10F5D0007003A3E069605A0D9051D2E493FAEDC331
:10F5E0009A505AED75F00EA4FAACF0ECFB74B22A06
:10F5F000F582740F12F64B650870DC8E828F83A340
:10F60000A3A3A3A3A3A3A3E0640160B212F6447072
:10F61000C674B42AF582740F12F64B687003A3E027
:10F620006970B474B62AF582740F12F64B650970CE
:10F63000A6ECF974B22AFA740F39FB80047A007BC5
:10F640000002F76874B32AF582740F3BF583E02259
:10F6500074F4122583EAFEEBFF8E828F83A3A3A3AB
:10F66000A3A3A3A3A3E06401700D8E828F83E0F5B2
:10F6700008A3E0F5098007123A258A088B0974FE71
:10F680006508700474FF65096057750A008021E5FC
:10F690000A75F00EA4F8A9F012F6E4701112F6FC47
:10F6A0007004A3E06509700612F6F31239CB050A5F
:10F6B00012F76D50258E828F83A3A3A3A3A3A3A3C8
:10F6C000A3E0640170C9E50A12F83A70E112F6FC91
:10F6D0007004A3E0650960D080D4AA08AB09123990
:10F6E000FB02F76812F6E82274B328F582740F1251
:10F6F000F7182274B228FA740F39FB2212F82F651A
:10F70000082212F7062275F00EA4F8A9F074B228A8
:10F71000F582740F12F7182239F583E02274B228AB
:10F72000F8740F39F922122B847F0602280974F429
:10F73000122583890B8A088B097E007F008E0A8040
:10F740001EE50A12F702650B7013AC08AD09AA8218
:10F75000AB831239D1E960050EEE70010F050A1274
:10F76000F76D40DDEEFAEFFB7F040228099051D2DD
:10F77000E493F8E50AC3982274F2122583890C8A6F
:10F78000088B098C0D750A00750B008004050A05AD
:10F790000B9051D2E493F8E50BC3985035E50B7507
:10F7A000F00EA4F8A9F074B228FE740F39FF8E820F
:10F7B0008F83E0650C70D8AC08AD09EEFAEFFB1250
:10F7C00039D1E960CAE50AC3950D40C1EEFAEFFBF5
:10F7D00080047A007B0002F729C082C08374F31290
:10F7E0002C1874FE6A700374FF6B603D7D008015F9
:10F7F000ED12F83A600EE0700B12F82B6A7003A35A
:10F80000E06B60250D9051D2E493F8EDC39840E091
:10F81000E4936D70148518828519837404F0740B59
:10F82000122E2D12FD67122F57802612F82F2274E8
:10F83000B428F582740F12F7182275F00EA4F8A9F7
:10F84000F012F6E8640122740B122E2DE0FAA3E008
:10F85000FB740D122B84D083D082022B3674F612E7
:10F860002583E4F508F5097808122B5612FB2112BE
:10F87000FBF7123EC97402122B84E9FE6003123AB0
:10F8800007EEF902F27774F612258374FE122C1833
:10F89000851882851983E4F0A3F0A818A9198808AF
:10F8A00089097808122B5675080275090078081224
:10F8B0002B567C007D007A417B00123ED5740412E9
:10F8C0002B84740202F27474F212258374EE122CEB
:10F8D00018EAFEEBFF8C088D09750A007A417B005F
:10F8E000123ECF8A0C8B0DAC0CAD0DEC4D6011E5CA
:10F8F000086C7003E5096D60077A417B00123EE1F8
:10F90000E4F50CF50D780C122B56AC08AD097A41D4
:10F910007B00123EC97402122B84E9640A70030250
:10F92000FA6B7402122BEA880889097808122B56A0
:10F930007508027509007808122B567C007D007A44
:10F94000007B03123EDB7404122B84E9600302FA8D
:10F950006B851882851983E4F0A3F0F50802F9F4A9
:10F960007404122BEA880C890D780C122B569051D6
:10F97000B91229C285080C12FC00850CF0A4F8AA63
:10F98000F0850CF0E9A42AF9E82402FCE439FD7AB8
:10F99000007B03123EDB7404122B84E9600302FA3D
:10F9A0006B7404122E2DE0F460487404122BEA8864
:10F9B0000C780C122B569051B91229C27404122ED5
:10F9C0002D12FEB19051B9E493F50C740193F50D2D
:10F9D000E8850CF0A4C8AAF0850DF0A42AFA850CDD
:10F9E000F012FBF0123ED57404122B84E9707C12E5
:10F9F000FCBD0508851882851983C082C08390519B
:10FA0000D2E493F8D083D082C3E098A3E09400506E
:10FA100021851882851983C082C0837402122E2D1D
:10FA200012FEB1D083D082C3E098A3E099500302C4
:10FA3000F960A818A919880889097808122B567541
:10FA400008027509007808122B567C007D007A4167
:10FA50007B00123ED57404122B84E9700EEEFCEF8D
:10FA6000FD7A007B03123EE1E96003750A01A90AF1
:10FA7000741202F72674F212258374FE122C187584
:10FA80000A0012FB21F508E439F5097A417B0012DE
:10FA90003ECF8A0C8B0DAE0CAF0DA818A919880C9F
:10FAA000890D780C122B56750C02750D00780C120E
:10FAB0002B567C007D007A417B00123EDB740412E1
:10FAC0002B847A007B03123ECFEA4B700CE5086E64
:10FAD0007003E5096F700D8041EE4F602B12FEAB95
:10FAE000E84960247C007D037A417B001235C9E936
:10FAF000F8880A7025EEFCEFFD7A417B00123EE1AA
:10FB0000E96009750A018012EAFEEBFFAC08AD0955
:10FB1000EEFAEFFB123A0DE9F50AA90A740202F7B0
:10FB2000269051B9E493F8740193F99051D2E4937B
:10FB3000F508E88508F0A4F8AAF08508F0E9A42AF9
:10FB4000F9E824022274F512258374FE122C18851C
:10FB50001882851983E4F0A3F0123A13E9707EA8A5
:10FB600018A919880889097808122B567508027592
:10FB700009007808122B567C007D007A417B001228
:10FB80003EDB7404122B84E970537E007F008E0AE2
:10FB9000803CE50A12FCCD7808122B569051B91220
:10FBA00029C2850A0812FC008508F0A4F8AAF0858D
:10FBB00008F012FBF0123EDB7404122B84E9700C87
:10FBC000E50A12F2D460050EEE70010F050A12F775
:10FBD0006D500A12FEABC3EE98EF9940B5851882BE
:10FBE000851983E0FAA3E0FB7402122B8402F51955
:10FBF000E9A42AF9E82402FCE439FD7A417B0022D9
:10FC00009051B9E493F8740193F9E82274F1122544
:10FC10008374F0122C18851882851983E4F0A3F000
:10FC2000FE805DEE12FCCD85080CF50D750E00789A
:10FC30000C122B5212F4437405122BF2123D8B74EA
:10FC400003122B847402122BEA880A890B780A1299
:10FC50002B569051B91229C28E0A12FC00850AF067
:10FC6000A4F8AAF0850AF012FBF0123ED574041233
:10FC70002B84850882850983E0F4600312FCBD0EA5
:10FC80009051D2E493F8EEC3984098A818A9198827
:10FC90000889097808122B5675080275090078083A
:10FCA000122B567C007D007A417B00123ED57404F5
:10FCB000122B847410122B847F0702280985188266
:10FCC000851983E02401F0A3E03400F02275F00EE2
:10FCD000A4F8A9F074B228F508740F39F50922C008
:10FCE00082C08374F3122C1812FEC170128A828BA8
:10FCF0008312FE1F122E2D12FEB7122F638017EAF9
:10FD0000FCEBFD7403122E2DAA82AB83122F3FAAA7
:10FD100018AB19122F6902F84774F712258374F390
:10FD2000122C18ECFEEDFF8518828519837404F0FF
:10FD3000740B122E2D12FD67122F6FE9F508601D4E
:10FD40008E828F83A3A3A3A3A3A3A3A37403F01200
:10FD50002E2DAC82AD83EEFAEFFB124853A9087446
:10FD60000D122B8402F567EAF0A3EBF0AA18AB1989
:10FD700022C082C08374F3122C18851882851983DF
:10FD80007404F0740B122E2D12FD67122F6F740184
:10FD900002F84974F612258374F3122C18900708A0
:10FDA000E070778518828519837404F090054612F7
:10FDB000FE1F122E2DE8F0A3E9F01233B9EAFCEB96
:10FDC000FD7403122E2DAA82AB83122F3FAA18AB0B
:10FDD00019122F751233C58A088B09A808A909744E
:10FDE00001122E2DE0687003A3E069602774FE689D
:10FDF000700374FF69601D7401122E2DE8F0A3E9F1
:10FE0000F07403122E2DAA82AB831233CBAA18AB47
:10FE100019122F759007087401F0740D02F274E046
:10FE2000F8A3E0F9740122C082C08374F3122C1885
:10FE300012FEC18A828B83701112FE1F122E2D12A8
:10FE4000FEB7122F63E970608027A3A3A3A3A3A327
:10FE5000A3A3E064037023EAFCEBFD7403122E2DD0
:10FE6000AA82AB83122F3FAA18AB19122F69E9702F
:10FE700037AA18AB19122F75802E8A828B83A3A301
:10FE8000A3A3A3A3A3A3E0640170128A828B8312AD
:10FE9000FEB1740B122E2DE8F0A3E9800A740B1248
:10FEA0002E2D74FEF0A304F002F847851882851900
:10FEB00083E0F8A3E0F922E8F0A3E9F0AA18AB196F
:10FEC000228518828519837404F08A828B83A3A308
:10FED000A3A3A3A3A3A3E064022274F5122583784D
:10FEE000007900880A7F0080010F9051D2E493FCD2
:10FEF000EFC39C5032EF75F00EA4FCAEF0EEFD7433
:10FF0000B22CF582740F3DF583E0F460DCAC0A742A
:10FF1000012CF50A8C08EA65084B70CDEF75F00EE0
:10FF2000A4F8EEF912F71DE8FAE9FB02F519C08210
:10FF3000C0839009157480F0D083D082022B367470
:10FF4000F6122583E9FCEAFD7901ECC39408500E12
:10FF500078008005E9C333F908E8C39C40F6E9421C
:10FF6000F2ED14600814600914600A800C7A0080B5
:10FF70000A7A1080067A2080027A30900915E0F81B
:10FF8000EC4A48F5B6E5B4A2E750FA74FF6952F2BC
:10FF9000E5BAF508E5BBAA08FBC39400A2D265D078
:10FFA0003350047A007B00ED14600814600D146077
:10FFB0001280188A088B09740880168A088B0974C5
:10FFC00006800E8A088B09740480068A088B0974DF
:10FFD000027808122D78AA08AB097F02022809E9E5
:10FFE000F875B60FE5B4A2E750FAE8C395BB500424
:10FFF000790180027900022B36FFFFFFFFFFFFFF30
:020000040001F9
:10000000C082C0837900EA1282053BF583C082C0BA
:100010008390051212D406D083D082C3E09CA3E063
:100020009D500CEA240B12805212803260010902AA
:10003000A385EA75F00BA4FAA8F075F00BEBA428E1
:10004000FB900514E02AF8A3E03B8882F583E05496
:100050000F22F582E43B12B4FE2274F71225838945
:100060000812AB97A3E0F9E875F00BA4F8ACF075B3
:10007000F00BE9A42C1283B6E8FEE9FF74016508D1
:1000800060067402650870228A828B831286E2748D
:100090000265087021EA2403FA50010B122F45E98A
:1000A00070148E828F83E4F0800CEA2403FCE43B1E
:1000B0001286D9122F3F8E828F83E0D2E7F0124052
:1000C0008B02A81074F412258312879C79008E820B
:1000D0008F83E06075890A890B8064E50A75F00BEF
:1000E000A4FAA8F075F00BE50B12803E7049E50A02
:1000F00075F00BA4F8AAF075F00BE50B12833A8E9D
:10010000828F83E085088285098312A203128659B3
:10011000EE2403FCE43F1281F8122F3F12A9D21201
:10012000BF2F1298EAD2E7F012408B7901900512A6
:10013000E0F50AA3E0F50B050AE50A7002050B12CB
:1001400085B5E50A9AE50B9B409102AE8574F512E0
:100150002583EAFEEBFF750A01740B122E2D129017
:10016000A9EC4D6015EC1282053D1287AA790112A7
:100170002F0FE508450960758023E50845096044AF
:1001800012820335091287AA1281F9122F45E964F8
:1001900001701BEEFAEFFB122F15E9F50A850882B4
:1001A0008509831286517902AA08AB09801112864B
:1001B000DA122F45E9640170347903EEFAEFFB128D
:1001C0002F0F80298E828F83A3E064FE7003A3E04B
:1001D000F4700B1286DA122F45E96401700CEEFA06
:1001E000EFFB122F15E9F50A8003750A00028C1443
:1001F000E50A2403FCE4350BFDE5082403FAE435A5
:1002000009FB22E50812C4352274F71225839005F4
:100210001212AAEFEA4B602FEA75F00BA4FAA8F0CD
:1002200075F00BEBA428FBEAFEEBFF123E519005A4
:100230001412AAEF90051412B4E96012EEFCEFFD5F
:100240007900123D978007900514E4F0A3F002A80E
:100250001074F6122583E4F508F5097808122B5678
:100260009005121290A475F00BA4FCA8F075F00B89
:10027000EDA428FD7A237B00123EC97402122B8460
:10028000E9FE6003122F2DEEF9028B2774F612257A
:100290008374FF122C187E007F00803C85188285B5
:1002A0001983E4128E13122B567508017509007814
:1002B00008122B56EEFCEFFDEC75F00BA4FCA8F039
:1002C00075F00BEDA428FD7A237B00123ED5740453
:1002D000122B840EEE70010F1283C240BF74010214
:1002E0008B2474F61225837E007F008039EEF8EFB0
:1002F000F912832E7808122B5675080B75090078B1
:1003000008122B56EEFCEFFDEC75F00BA4FC75F01B
:100310000BEDA42AFD7A237B00123EDB7404122B22
:10032000840EEE70010F1283C240C2028B27E87563
:10033000F00BA4F8AAF075F00BE9A42AF9900514C3
:10034000E028F508A3E039F5092274F61225837E2A
:10035000007F00804AEEF8EF1283A788828983E04D
:10036000A2E75036C2E7F085820885830978081233
:100370002B5675080B7509007808122B56EEFCEF0A
:10038000FDEC75F00BA4FC75F00BEDA42AFD7A23AF
:100390007B00123ED57404122B840EEE70010F12F6
:1003A00083C240B1028B27F9E875F00BA4F8AAF0DC
:1003B00075F00BE9A42AF9900514E028F8A3E039B8
:1003C000F92290051212A7F7C3EE98EF9922C08286
:1003D000C083EC4D600512485380097C087D00798C
:1003E00000123D9702A38574F61225837900EA4B2B
:1003F00060177800EA28F582E412BC4660047901AF
:10040000780808E8C3940840EB028B2774F712259C
:100410008374F3122C18ECFEEDFF85188285198386
:10042000E4F004122E2DEAF0A3EB12A7E9122F63D9
:100430007403122E2DAC82AD83EEFAEFFB122F3F28
:10044000EEFAEFFB122F4502A80B74F71225837406
:10045000F3122C18ECFEEDFF851882851983E4F069
:10046000EAFCEBFD7403122E2DAA82AB83122F3F00
:10047000AA18AB19122F697401122E2D12A2108E18
:10048000828F8312A7DA74FE68700374FF696004B8
:1004900079018002790002A80B74F7122583EAFE25
:1004A000EBFF122F09E9F508740165087011128538
:1004B00002F4FA88828983E05A4480F012408B0269
:1004C000985F74F7122583EAFEEBFF7508008E82B1
:1004D0008F83E0602A122F09E9F50874016508701E
:1004E0001E128502FA88828983E05A70128E828FEA
:1004F00083E04480FA88828983E04AF012408B02CC
:10050000985F12A9D6129A371283A78E828F83E042
:100510002274F41225838A088B097C007D00EA127C
:1005200081FB122F3FE508128673790085088285CA
:100530000983A3E064FE7003A3E0F460757E007F8E
:10054000008066EEFAEFFB1280326058EEFAEFFBA5
:10055000EA75F00BA4FAA8F075F00BEBA428FB9059
:100560000514E02AF50AA3E03BF50B85088285090E
:1005700083A312BC21850A82850B83A3E06A7003E2
:10058000A3E06B701FE50A2403FAE4350BFB122F7E
:1005900045E9640170061281F0122F3F12866879D6
:1005A0000112D23A0EEE70010F1285B5EE9AEF9B52
:1005B000409102AE8590051212B500C32274F31269
:1005C00025838A088B098A828B83128651EA1286D8
:1005D00073750C00EA1281FB122F45E96401706A01
:1005E0007E007F00805FEEF8EFF9E875F00BA4F86D
:1005F000AAF075F00BE9A42AF990051412D2ACE028
:10060000540F603CEEF8EFF9E875F00BA4F8AAF08F
:1006100075F00BE9A42AF9900514E028F50AA3E087
:1006200039F50B1281F012484DE964017012850A08
:1006300082850B83128659128668750C0112D23A94
:100640000EEE70010F1283C2409CA90C7F05022898
:1006500009A374FEF0A304F022A312A7F785088271
:10066000850983A3129F1522E50812867DEEF0A36B
:10067000EFF02212867D74FEF0A304F02212C4393A
:100680003509F5832274F5122583EAFEEBFF8E828D
:100690008F831286517C007D001286DA122F3FEE86
:1006A000FAEFFB122F09E9F50A7401650A702712A7
:1006B000A7F012832E850882F5831286E21281F953
:1006C000122F45E96401700EE5082403FCE43509A6
:1006D0001286D9122F3F028C14FDEE2403FAE43F58
:1006E000FB22A312BC2B129F152274F212258374D5
:1006F000E6122C1812879C750C017508007509000C
:10070000750A00750B00851882851983E4F0EE24C4
:1007100003FCE43FFD7403122E2DAA82AB83122F3B
:100720003FAA18AB19122F69E96401701F740B12EC
:100730002E2D1287AC7401122E2D12BC257003A32E
:10074000E069604AA818A91988088909740D122E51
:100750002D12A202A312A210740E122E2D12A7DACD
:10076000740D122BF2122F63E964017009740D12DB
:100770002BEA880A890B780A122B56AC08AD09EED1
:10078000FAEFFB122F1B7402122B84E9F50CEEFA20
:10079000EFFB122F5DA90C741A02BB81EAFEEBFF7E
:1007A00012A9D674FEF0A304F022F583129A37F949
:1007B00012A9D6129F1522C082C0837800790080CA
:1007C0000508E87001091285B5E89AE99B5029E807
:1007D000FAE9FBEA75F00BA4FAACF075F00BEBA4A8
:1007E0002CFB900514E02AFCA3E03B8C82F583E00F
:1007F000540F70CD79008002790102A385C082C0B8
:10080000839051C4E49375F016A4FCADF079FF7A9F
:10081000337B0A123D9702A38574F6122583EAF80A
:100820007508007D008012ED12BC38C3994009E0C4
:10083000FAE8C39A400205080D9051C4E493FAED1A
:10084000C39A40E3AA087B00028B2774F012258329
:1008500074F3122C188A0C8B0D8C088D09890AEC04
:1008600045096016AA08AB09122FB18A0E8B0FAE8C
:100870000EAF0FEE4F600302893E7B0080010B122A
:10088000BF25500F1289E670F5743328FE740A39BB
:10089000FF80047E007F00EE4F700302899290512A
:1008A000B71289B960217403650A60067404650A89
:1008B00070157A047903122F879051C4E493FC9049
:1008C00051B71289BF50299051B51289B960287467
:1008D00001650A60067402650A701C7A02790112C9
:1008E0002F879051C4E493FC9051B51289BF400703
:1008F0007A007B000289B68518828519837401F01D
:10090000122E2DE50CF0A3E50DF0AC08AD09740333
:10091000122E2DAA82AB83122F3FAA18AB19122FC9
:1009200075740B122E2D129F0E8E828F83A3A3A39C
:10093000A3A3A3E412D402AA0CAB0D1235337800A2
:10094000E50A6007C39405500278048E828F83E520
:100950000CF0A3E50D12C9E6E50AF0E88E828F835C
:10096000A3A3A3A3A312BF365001097A027B0012EE
:10097000232612942AA312BB61A312946EE50A6087
:100980000DC3940350081293F91289D7800312946F
:1009900010F07A047900122F878A089051C4E493EA
:1009A000FAC3E5089AEB94004005901038E4F01281
:1009B0003407EEFAEFFB028D721289CFE84922125A
:1009C00089CFECC398F8E499F9C3EA98EB9922E44B
:1009D00093F8740193F922F9EE2414F582E43FF5BB
:1009E00083E8F0A3E922EB75F016A4F8A9F01294BD
:1009F00063F42274F212258374F3122C188A088B84
:100A000009ECFEEDFF750A00EEFAEFFB122FB18A3A
:100A10000C8B0DA80CA90DE8497003028AB78882D7
:100A20008983E065087004A3E065097003028AB752
:100A300088828983A3A3A3A3E0C394055079888205
:100A4000898312C86612AC53E0603488828983A31C
:100A5000A3A3A3E0C3940350269051B3E493FA7484
:100A60000193FB12974C9051BDE493FA740193FBF0
:100A7000E82414F582E439F583EAF0A3EB800DE86D
:100A80002412128ABEF0E82414128ABEF08518825D
:100A90008519837401F0122E2D12C866F0EEFCEF5A
:100AA000FD7403122E2DAA82AB83122F3FAA18AB1E
:100AB00019122F75750A01A90A740D02BB81F582FE
:100AC000E439F58374FEF0A3042274F61225831230
:100AD0002FAB8A088B09A808A909E8496014888205
:100AE0008983A3A3A3A3E06009C3940550047901FB
:100AF00080027900803174F6122583122FAB8A08A8
:100B00008B09A808A909E849601488828983A3A3EE
:100B1000A3A3E06009C39403500479018002790023
:100B200080057402122B847F0202280974F61225B4
:100B300083122FAB8A828B83E5824583600BA3A34C
:100B4000A3A3E0700479018002790080DAC082C03A
:100B500083EAFCEBFD7A007B0002A382C082C083A3
:100B60007C007D0002A38274F512258374F3122C9D
:100B700018EAFEEBFF8C088D09C3EC94F8ED94FFA6
:100B80004004EE4F606A750A00801974FF650870B2
:100B90000474FF6509600B12CB637004A3E0650960
:100BA000603B050A9051C4E493F8E50AC3985040AD
:100BB000E50A1289E760EBEE4F60D0128BFB122E34
:100BC0002D12A7E5122F6FE960D87403122E2DACF9
:100BD00082AD83EEFAEFFB12484DE960C5E50A7578
:100BE000F016A4F8A9F0743328FA740A39FB8004CB
:100BF0007A007B00740D122B84801B851882851966
:100C0000837401F0743528F582740A39F58312A7CC
:100C1000F7740B22A90A7F0302280974F4122583B2
:100C200074F3122C18750800122FB18A0A8B0BAEC0
:100C30000AAF0BEE4F601F128C7E128C0E122E2DFF
:100C400012A7E5122F577C167D0079FFEEFAEFFB15
:100C5000123D977508017A047900122F878A0A904D
:100C600051C4E493FAC3E50A9AEB9400500990103A
:100C7000387401F0123407A908740D02AE82851889
:100C8000828519837401F08E828F83A3A32274F767
:100C9000122583E9FC74FE6A700374FF6B7D00709B
:100CA00003802C0D128CF05026ED1289E760F412AF
:100CB000D6476A7003A3E06B70E98012ED75F016F9
:100CC000A4F8A9F012D63A6018E0640360130D127C
:100CD0008CF05015EC60E512945760F2C394055007
:100CE000ED12CDA712BC1E80047AFE7BFF02A81075
:100CF0009051C4E493F8EDC39822122FC302A38548
:100D0000C082C083790180F274F01225838A0A8B35
:100D10000B7A047901122F878A0C8B0DEA450D603E
:100D200040EA2AFAEB33FB123E518A088B09AE08DF
:100D3000AF09EE4F60267AFE7BFF122FC974FE6A60
:100D4000700374FF6B601E85088285098312AAEF09
:100D5000E5082402F50850E2050980DE750C0080E4
:100D6000047E007F00850A82850B83E50C12AA238E
:100D70008005740D122B847F08022809E493F8EC97
:100D8000C3982274F6122583E4F508F50978081251
:100D90002B569051C4E493F50874037808122D443F
:100DA000129096123EC97402122B84E9FE740A6EE8
:100DB0006024E4F508F5097808122B569051C4E434
:100DC0009325E0FCE433FD7A3F7B00123EC97402B8
:100DD000122B84EE6003122FDB02828774F6122539
:100DE0008374FE122C18851882851983E4F0A312EF
:100DF0008E13122B567508027509007808122B56AF
:100E00007C007D007A227B00123ED57404122B8474
:100E1000028B22F0A818A919880889097808227479
:100E2000EE12258374E4122C188A0E8B0F8C088D19
:100E300009750C007A227B00123ECF8A0A8B0B7A4E
:100E40003F7B00123ECF8A108B11AE10AF11E50A26
:100E5000450B6017E508650A7004E509650B600B32
:100E6000AC0AAD0B7A227B00123EE17430122E2DBB
:100E7000E0F50AA3E0F50BEE4F6015E50A6E70038E
:100E8000E50B6F600BEEFCEFFD7A3F7B00123EE15D
:100E9000E4F510F5117810122B56AC08AD097A2242
:100EA0007B00123EC97402122B84E9640A700302AB
:100EB000908CE4F508F5097808122B56AC0AAD0BB6
:100EC0007A3F7B00123EC97402122B84E9640A70D7
:100ED0000302908C7404122BEA880889097808129E
:100EE0002B567508027509007808122B567C007D78
:100EF000007A017B03123EDB7404122B84E9600349
:100F000002908C851882851983E4F0A3F0FE02908C
:100F1000037406122BEA880889097808122B567583
:100F200008087509007808122B568E087403780893
:100F3000122D44E5082402FCE43509FD7A017B0307
:100F4000123EDB7404122B84E9600302908C740857
:100F5000122E2DE0F47003A3E0F4700302900274EB
:100F600006122BEA880889097808122B567508089A
:100F70007509007808122B567404122E2D1290A9B0
:100F800074037808122D44129096123ED574041200
:100F90002B84E9600302908C7402122BEA88088982
:100FA000097808122B567508027509007808122B6B
:100FB00056EE25E0FCE433FD7A027B03123EDB743F
:100FC00004122B84E970387402122BEA880889090C
:100FD0007808122B567508027509007808122B56EE
:100FE0007404122E2D1290A42CFCED33FD7A3F7B5D
:100FF00000123ED57404122B84E9600302908C1217
:10100000955F0E851882851983C082C0839051C474
:10101000E493F8D083D082C3E098A3E094005021F9
:10102000851882851983C082C0837404122E2D1204
:10103000A210D083D082C3E098A3E0995003028F1E
:1010400011A818A919880889097808122B5675085B
:10105000027509007808122B567C007D007A227BED
:1010600000123ED57404122B84E97020AC0EAD0F33
:101070007A017B03123EE1E97012742E122E2D12BA
:10108000D4067A027B03123EE1E96003750C01A9E4
:101090000C741C02B14AE5082402FCE43509FD7A0F
:1010A000227B002212D40AEC22E0F508A3E0F50925
:1010B0002274EC12258374FE122C18750A00851810
:1010C00082851983E4F0A3F09051C493F510F508DC
:1010D00075090074037808122D44E5082402F50808
:1010E00050020509E51025E0F510E433F5117A22E8
:1010F0007B00123ECF8A0C8B0DAE0CAF0D7A3F7B7E
:1011000000123ECF8A0E8B0FA818A919880C890DE2
:10111000780C122B56750C02750D00780C122B569C
:101120007C007D007A227B00123EDB7404122B844B
:101130007A017B03123ECF8A0C8B0D7A027B03125D
:101140003ECF8A128B13A812A913E50C450D700A25
:10115000E5086E7003E5096F7025E849700CE5102D
:10116000650E7004E511650F7015E50C450D607B8B
:10117000EE4F604E85188285198312AAF560437C74
:10118000017D037A227B001235C9E9F8880A705B79
:101190007C027D037A3F7B001235C9E9F8880A702A
:1011A0004AEEFCEFFD7A227B00123EE1E9700EACC4
:1011B0000EAD0F7A3F7B00123EE1E96011750A0126
:1011C0008029AE0CAF0DE8496004880E890F7810B5
:1011D000122B56780E122B56AC08AD09EEFAEFFB27
:1011E000122FE17404122B84E9F50AA90A74021281
:1011F0002B847F0C02280974F112258374D9122CD8
:10120000187402122E2DE4F0A3F0122FE7E9600308
:101210000293E87402122BEA880889097808122BD5
:10122000567508027509007808122B567C007D005F
:101230007A227B00123EDB7404122B84E9600302E5
:1012400093E89051C4E493FA7402122E2D12A21066
:10125000C3EA98E49950030293E8750A00750B00FD
:10126000750800803E85188285198312BD0A12CD4B
:101270009A12A7DA851882851983129A371289D7AC
:10128000F07A047900122F878A0C9051C4E493FA03
:10129000C3E50C9AEB94004005901038E4F012344A
:1012A0000705089051C412BB4040030293E8740242
:1012B000122E2D12A210C3E50A98E50B99400302E5
:1012C00093E87411122BEA880C890D780C122B56B6
:1012D000750C08750D00780C122B5685080C7403DC
:1012E000780C122D44E50C2402FCE4350DFD7A2225
:1012F0007B00123EDB7404122B84E970A474131279
:101300002E2DE0F47003A3E0F46096050AE50A7060
:1013100002050B7404122E2D7401F07413122E2D7D
:1013200012A210740F122E2D12A7DA7404122BF2CF
:10133000122F6FE970030292A112D4037411122EBE
:101340002D12BC21123533E50875F016A4F8A9F06A
:10135000743328FE740A39FF7411122BEA880C8941
:101360000D750E00780C122B527C087D00EEFAEF02
:10137000FB123D8B7403122B8412BF3B5001097A80
:10138000027B0012232612942A12946EA818A9191F
:10139000880C890D780C122B56750C02750D00788F
:1013A0000C122B56AC08EC2CFCE433FD7A3F7B008E
:1013B000123EDB7404122B84E960030292818518CB
:1013C00082851983E0F47003A3E0F4600302926560
:1013D000E508129458600BC3940350061293F90267
:1013E000927D1294100292807402122E2DE0F974F4
:1013F00027122B847F070228099051B31289CFEE60
:1014000012CD9E129F159051BDE493F87401932262
:10141000EE241212941EF0EE241412941E22F58271
:10142000E43FF58374FEF0A30422E88E828F83A349
:10143000A3A3A3A3A3A3A312944F740112944FA335
:1014400074AAF0EE2410F582E43FF583E4F0221252
:10145000CA09A3A3A3A322ED75F016A4F8A9F0125C
:10146000946322743728F582740A12D4F622A3F00A
:1014700012A9D6E4F0EE240CF582E43FF583E4F003
:10148000A3F0A3F0A3F02274F312258374FE122CB0
:1014900018851882851983E4F0A3F0F50C029520D5
:1014A000E50C75F016A4F8A9F0743328F50A740A4F
:1014B00039F50B850C82AE82780A122B5675080816
:1014C0007509007808122B568E0874037808122DBF
:1014D00044129096123ED57404122B84E50A24140B
:1014E000F508E4350BF5097808122B5675080275D6
:1014F00009007808122B56EE2EFEE433FFEEFCEFC7
:10150000FD7A3F7B00123ED57404122B84850A823B
:10151000850B83A3A3A3A3E0F4600312955F050CDE
:101520009051C4E493F8E50CC39850030294A0A82A
:1015300018A919880889097808122B5675080275A8
:1015400009007808122B567C007D007A227B00125D
:101550003ED57404122B847402122B8402864C85AF
:101560001882851983E02401F0A3E03400F022C042
:1015700082C0837D008009EA24FF1AEB34FFFB0D53
:10158000128CF05016129457C3940550F2EA4B7027
:10159000E6743328FA740A39FB80047A007B00026F
:1015A000A38574F712258374F3122C187E0002961B
:1015B0003AEF75F017A4F8A9F012D61D12BD077501
:1015C000F016A4FAABF074332AF582740A12BF59EC
:1015D0007003A3E0696040EF75F017A4F8AAF0EA81
:1015E000F912D61D39F58312A2107401122E2DE0C6
:1015F000687003A3E069601FEF75F017A4F8EAF9BB
:10160000740328FC740C39FD7403122E2DAA82ABCE
:101610008312484DE96013EF75F017A4F8A9F07430
:101620000128FA740C39FB12353F0F9051BFE49337
:10163000F8EFC39850030295B10E9051C412D18CAB
:10164000501FEE12D640F47003A3E0F460EB128B4F
:10165000FB122E2D12A7E5122F6FE960DC7F0080B0
:10166000CA02A80B74F712258374F3122C18900584
:10167000E512B4E97003029710750800802BE508A5
:1016800075F016A4F8EAF9744728F582740A12D4A2
:10169000F264FE7003A3E0F4600D744528F58274D3
:1016A0000A39F58312BB7705089051C412BB40502C
:1016B0005FE50875F016A4F8AAF0EAF912945F60E5
:1016C000E6C3940350E1744528F582740A12B4E627
:1016D00070ACE50875F016A4F8EAF9743328F874CC
:1016E0000A39F9E8FEE9FF1297AE1297A4122769AA
:1016F000128C7E128C0E122E2D12A7E5122F6FE97E
:1017000060A57403122E2DAA82AB83122FBD809781
:1017100002A80B74F6122583122FAB8A088B09A836
:1017200008A909E849602088828983A3A3A3A3E0CC
:101730006011C39403500CE82414F582E412BC1E1B
:1017400012974C790180027900028B27E82412F568
:1017500082E439F583EAF0A3EBF02274F7122583D3
:10176000EAFEEBFF9005DF12B4E960309005E51268
:10177000B4E960289005E912B4E9602012CEE812BD
:101780002769E9701712979F122769E96401700CA5
:101790008E828F83A3A312CED512276902A81012BE
:1017A00097AEA3A312B5009005E512CEDF229051AB
:1017B000BDE493FC740193FD8E828F8322C082C0AE
:1017C0008390051B74C3F0A37432F090051D74BDA3
:1017D000F0A37432F090052174B9F0A37430F002D4
:1017E000A385C082C08390051F74B7F0A37432F044
:1017F00002A38574F7122583EAFEEBFF900555E0FE
:101800006408601CE0640460178E828F83E05403D8
:101810006401704112B8D9F8129864E0640670351A
:101820008E828F83A3A3E064FE7003A3E0F460259F
:101830008E828F83A3A312C41B7003A3E069700878
:10184000EE241512C410600512338380031233890D
:10185000E9F50880037508C2EEFAEFFB123E57A9BE
:101860000802A810A3E0F58388822274F41225836D
:101870008A088B09129A33FAE82AFAE43400FB1238
:101880003E518A0A8B0BAE0AAF0BEE4F60558508AE
:1018900082850983E0FC7D007900123D978E828F5E
:1018A00083A31286511233BF8E828F83A3A3A3A377
:1018B000EAF0A3EB1298EAF8EE28F8E43F1287AFBB
:1018C000850882850983A3E0C0E012BF1BD0E0F049
:1018D0001233D112BF11E9129EF1E0C0E0129EE76F
:1018E000D0E0F0EEFAEFFB02AE85F08508828509C4
:1018F00083E02274F412258374E8122C188A088B72
:10190000098C0A8D0BE9FE900555E064046005E042
:101910006408700479C2803CA37808122DC7EE9049
:10192000055C129B76123D9785188285198378088D
:10193000122DC77405122E2DEEF07404122E2D7484
:1019400001F07407122E2DE4F0900555740212A7D1
:10195000E91249F702AE8074F412258374E8122C60
:1019600018EAFEEBFF90051612B4E96003029A2E06
:101970007A077B00123E5190051612AAEF900516C9
:1019800012B4E97003029A2A8E828F83122E0A9073
:101990000516E0FCA3E0F5838C82122E16EE2404DB
:1019A000F50AE43FF50B850A82F583E0C0E0900577
:1019B0001612B4BDA3A3A3D0E0F0EE2405F508E40D
:1019C0003FF509850882F583E0C0E090051612B462
:1019D000CBD0E012A7DFC0E0900516129A37C824DA
:1019E00006F582E438F583D0E0129B76123D978E9F
:1019F000828F83122E0A851882851983122E1685EE
:101A00000A82850B83E0C0E07405122E2DD0E0120F
:101A100098EAC0E07404122E2DD0E0F07407122E64
:101A20002DE412A7E91249F78006791080027901A6
:101A300002AE808A828B83E0F8A3E022C082C0835A
:101A400090051612B4E9601090051612BC21123EE2
:101A500057900516E4F0A3F01232ED1234DF02A322
:101A60008574F412258374E8122C188A0A8B0BEC07
:101A7000FEEDFF89087428122E2DE0FC7429122E29
:101A80002DE0FD740F6C7005740F6D60129010A640
:101A9000E064026005ECC39D500579C1029B73743C
:101AA00024122E2D122E0A900556122E16E508909D
:101AB000055CF0EC90055AF0EDA3F0742A122E2D7F
:101AC000E090055DF074FF650A700474FF650B70AB
:101AD000249010BAE0F47003A3E0F4700C123DA956
:101AE000900553EAF0A3EB80129010BA12CDC4E82F
:101AF000F0A3E9800690055312BF2FF0EE4F601758
:101B0000EEFAEFFB123593E96401700BEEFCEFFD8A
:101B10007A677B05124853900546E4F0A3F09005E0
:101B200049F0A3F0900566F09010A6E064027008FA
:101B300090055A740FF0A3F09005557405129B762A
:101B4000123D977404122E2DE4F0900556122E0AC1
:101B5000851882851983122E1690055CE0C0E0740A
:101B600005122E2DD0E0F07407122E2DE412A7E9F5
:101B70001249F702AE80F07C187D007900AA18ABFC
:101B8000192274F7122583E990051AF07A807B00F8
:101B90009005A0E0F9123F23123053790002A810FB
:101BA000C082C08390051AE070031241CF123053F7
:101BB00002A38574F012258390051AE09010377007
:101BC0000FE06005790012404F901037E4F0804A32
:101BD000E06401600890051AE0F912404F90103758
:101BE0007401F090051AE0F46030E0F50CE4F50DB6
